:020000040000FA
:040000006FD00400B9
:101000006F00907E00000000000000009020002093
:10101000AA220020A9BDF9F56C23002000000000E1
:10102000000000006C230020902000200000000041
:101030000000000090200020000000009020002010
:101040000000000090200020902000209020002030
:101050009020002090200020582F00209424002071
:101060000000000090200020902000201E2400207E
:1010700090200020D22300209020002090200020EB
:101080009020002090200020902000209020002020
:101090009020002001A04111B7170040985F3AC688
:1010A000945F3247E39CE6FE3245410182800111A4
:1010B00013078008F337078093F787083EC20100C3
:1010C0000100B7170040930570052380B70413068D
:1010D00080FA2380C7040100010083C6B70493F699
:1010E000F60DA385D704238007049246F3A6068055
:1010F0000100010093760502D5CEF336078093F602
:10110000860836C4010001002380B7042380C70489
:1011100001000100B70614007D89558D88C70100C4
:1011200001000100010023800704A246F3A6068007
:101130000100010073370780137787083AC6010062
:1011400001002380B7042380C704010001000100CF
:1011500001003727004093061005A303D7802380A2
:101160000704B247F3A70780010001009307800836
:10117000F3B7078093F787083ECE01000100B71749
:101180000040130770052380E704130780FA2380CB
:10119000E7040100010003C7B70413670708A3852C
:1011A000E70423800704F247F3A70780010001004A
:1011B0000561828093760504BDC6F336078093F6F9
:1011C000860836C8010001002380B7042380C704C5
:1011D00001000100B7061400938606047D89558D31
:1011E00088C7010001000100010023800704C246F6
:1011F000F3A6068001000100733707801377870884
:101200003ACA010001002380B7042380C70401000B
:1012100001003727004093062005A303D7802380D1
:101220000704D24781B773370780137787083ACC12
:10123000010001002380B7042380C70401000100DE
:1012400098471367070C98C723800704E24719BF24
:101250000111814601468145114506CE97000000E7
:10126000E780605893078008F3B7078093F78708F3
:101270003EC601000100B717004013077005238028
:10128000E704130780FA2380E7040100010003C785
:101290006704136717002383E70423800704B2471A
:1012A000F3A7078001000100F2400561828041112F
:1012B000814601468145114597000000E780A05214
:1012C00013078008F337078093F787083EC40100AF
:1012D0000100B7170040130670052380C70493066A
:1012E00080FA2380D70401000100FD552396B70240
:1012F00023800704A245F3A5058001000100733790
:101300000780137787083AC6010001002380C704CD
:101310002380D7040100010003C767041367170087
:101320002383E70423800704B247F3A70780010063
:10133000010001A0BD473305F50201007D1575FDD3
:101340008280411122C426C206C6AA8401446317C2
:101350009400B24022449244410182800504130566
:10136000803E420497000000E78000FD4180C5B741
:101370009305000273A04580824573901534924016
:101380002242B2424243D2436244F2440255925551
:101390002256B2564257D2576258F25806499649D9
:1013A000264AB64A464BD64B664CF64C065D965DD1
:1013B000265EB65E465FD65F09617300203041113C
:1013C000B7170040985F3AC6945F3247E39CE6FE49
:1013D000324541018280B71700401307000323887C
:1013E000E702854717170000232EF74673002030C9
:1013F000411122C42D6426C24AC006C637190040D6
:101400001304A4AAB704002023208900976000E0F9
:10141000E780C0379C408297976000E0E780003704
:10142000E5B737370040834747009146BD8B639E41
:10143000D702B73600401306F00F973500009385AA
:10144000651F9737000083D7E72E03C7A6001377E1
:10145000F70F1DE3B7E70400BC4F09468945171590
:1014600000000345A5F7829731A099466394D70001
:10147000834757007300203003C786001377F70FA8
:10148000E365F6FC13851700AE97173800002313A9
:10149000A82A2380E70075B7B787004003C7670015
:1014A000098B6309071003C77700930600031377BE
:1014B0000703630DD70817380000034878771736FD
:1014C00000001306E6730547B30606012380E60015
:1014D00083C577001737000013078774429793F589
:1014E000F50F2300B70003C58700973500009385EB
:1014F0002572C2951375F50F2380A50003470700D9
:1015000089451377F703630CB70C63E7E50A6306B5
:10151000071A8545630CB7129737000083C75771C8
:101520003307F600034707001377F70F19CB85073A
:1015300093F7F70F3D476363F71A17370000A309C6
:10154000F76EB787004009472383E700B78700405D
:1015500083C77700E207E18763DE0704973700005F
:1015600083C7176D17370000130787693E978546B5
:101570002300D700173700001307876A3E979306AA
:1015800000032300D70017370000130767683E9752
:10159000A14685072300D70093F7F70F3D47636403
:1015A000F71417370000A305F768B787004009470D
:1015B0002383E70073002030930610026300D70EE8
:1015C000930620026305D70693060002E316D7F4BC
:1015D00003C727021377C70F13672700D5A803C7D0
:1015E00067001377070465CB03C7A702173800000D
:1015F00013088842173500001305C539134707083B
:101600002385E70203C7A7021377370F1367870005
:101610002385E702814713070004B305F5008C41D9
:10162000B306F80091078CC2E399E7FEF5B503C74E
:10163000A702134707042385E70203C7A70213770E
:10164000C70F136727002385E702F9B503C76700B3
:101650001377070449C303C767021738000013084C
:10166000682F173500001305A526134707082383A5
:10167000E70203C767021377370F136787002383D7
:10168000E702814713070004B305F5008C41B30658
:10169000F80091078CC2E399E7FEBDBD03C767025E
:1016A000134707042383E70203C767021377C70FB3
:1016B000136727002383E70285B503C76700137705
:1016C000070411CB03C727021377370F136787006F
:1016D0002381E70291B5238006003DBD97370000C6
:1016E000A3880754B9BD97370000A383075475BD7D
:1016F0002303048015472303E48001002302A48010
:10170000828083076480E3CE07FE23030480828007
:1017100083076480E3CE07FE03454480828083070D
:101720006480E3CE07FE2302A4808280411126C498
:101730004AC24EC006C61377F50BAD47AA892E895B
:101740009544630CF700194597000000E78080FA84
:1017500097000000E78020FB8D444E859700000035
:10176000E78040F9FD59FD1463983401B240A2446A
:101770001249824941018280135509011375F50F01
:1017800097000000E780E0F92209F1BF011126CCA3
:1017900006CEB704080097000000E780C0F61545A4
:1017A00097000000E78000F597000000E78080F6D2
:1017B00097000000E78000F62AC697000000E78047
:1017C00080F432459377150089EB13651500137586
:1017D000F50FF240E24405618280FD14E9F0014515
:1017E000CDBF397126DC4ADA4ED852D656D45AD2F9
:1017F0005ED006DE62CE66CCB7E700E07D5783AAF6
:10180000070022C603AA470023A0E71823A2E7186F
:10181000B7170040130770052380E704130780FA09
:101820002380E70483C74704930B75FFB684E20760
:1018300093FBFB0F8546AA892E8B32893724004003
:10184000E187015763FA76016308D50089461307DB
:1018500000026313D5000157D98F93F7F70FB71C18
:1018600000402382FC0411472303E4801305F00F9A
:1018700097000000E78000E8094C97000000E7802F
:1018800080E863657C15B7050700DA9537870700A0
:10189000795563FEE504B3879500636AF704370B57
:1018A0000800A94733EB65016395F90881E8814495
:1018B00097000000E78020E5268515A8DA85094510
:1018C00097000000E780C0E605090345F9FFFD1415
:1018D000050B97000000E780C0E481C49377FB0FFD
:1018E000E5F797000000E780A0EA69F17D55B7179A
:1018F0000040130770052380E704130780FA238054
:10190000E70403C74704418B2382E704F250B7E79B
:1019100000E023A0571123A24711E2543244525948
:10192000C259325AA25A125B825B724CE24C21615C
:101930008280A547639BF90685691309F00FB306FA
:101940009900B3742B01B6941349F9FFB37499004D
:10195000856B33796901416B9387F9FFB3F72701F1
:1019600099E363FC340193D94900C147E3E637FFAB
:101970003DBF0569C1697D19D9B71305800D63881D
:101980006901130500026384790113051008CA85F3
:1019900097000000E780C0D997000000E78040DF93
:1019A00031D54E99B38434416DBFDA852D4597000A
:1019B0000000E780E0D7CA94E30B99EE0509970091
:1019C0000000E78020D5A30FA9FEFDB79387F9FF9C
:1019D00093F7F70F636DFC0C83C71C0413073008E3
:1019E0006315F706370708006361EB06B3079B0032
:1019F000B706100063FBD704334BEB0089476399AC
:101A0000F9068980D549E38404EADA850945970017
:101A10000000E780E0D111090327C9FF9147232087
:101A2000E48003076480E34E07FE23033481FD173F
:101A3000EDFBFD14110B81C49377FB0FE9FF9700B9
:101A40000000E780E0D461F155B5B717004003C747
:101A50005704B70708001377070219E3B787070091
:101A60007955E376FBE833079B00E3F9E7F841B5E6
:101A70008547E380F9F0DA852D4597000000E7807F
:101A800020CB9389F4FFE38404E297000000E78011
:101A900060C893F7390091EB83260480032709007F
:101AA00093074900E396E6E03E89CE84D9BFB54767
:101AB0006399F9001305900B97000000E78080C33D
:101AC000FDB3B1471305B00AE388F9FE9947639760
:101AD000F904B7050800B365BB002D459700000069
:101AE000E78000C581448D4BA14997000000E78045
:101AF00060C263967401832704802320F900850463
:101B0000E39534FF8327048013172B0163550700E7
:101B10002312F90069BB2322F90051BB9D47639F43
:101B2000F90281451305B00497000000E78040C02A
:101B3000BD442320090023220900FD59970000001D
:101B4000E78040BD93F77400CA9703C70700FD14F0
:101B5000398D2380A700E39334FF91BBA14763979E
:101B6000F90697000000E780A0C28144630D0B00D6
:101B70008D479304C0036308FB00930400056304CE
:101B80008B01930440041375C507E30295D21945F0
:101B900097000000E78000B697000000E780A0B63D
:101BA000054597000000E780E0B426859700000017
:101BB000E78020B7094597000000E78080B69700CE
:101BC0000000E780E0BCE31405CE0DB39147639FAE
:101BD000F9001305600697000000E780A0B19700A8
:101BE0000000E78040B213059009F9B5E38109CC04
:101BF000F1547DB9BD660147173600001306C620B3
:101C0000938606A685458347060093F7F70F91C391
:101C100082800507E3F9E6FE973700002386B71EAA
:101C2000DDB77D166206618693178601E18763D46E
:101C3000070001458280931726003307F500AE9711
:101C400018439C4363E7E7007D16E37FF7FC7D556F
:101C5000828005458280FD15E205E18513978501A7
:101C6000618793F7F50F63480700FD15139725006B
:101C70002A97584365D713851700620561858280CE
:101C80003308B5021C4283A80600B335B502C297DB
:101C900033B50701AE98469585486367B5006394F0
:101CA000A50063E3070181480C43C6950CC388C2B5
:101CB0001CC2828081471397870161876343B70005
:101CC0008280139727002A97232007008507E5B70E
:101CD0008147014793968701E18663C5B6001335B6
:101CE0001700828093962700AA9694428507558F05
:101CF000D5B793D755408A07AA979C430545331516
:101D0000B5007D8D828017F3FFDFE702833D2A84D3
:101D100097000000E78060F405C5931725003E9406
:101D20000327C4FF814711EB7D1516053E9542053B
:101D3000418517F3FFDF6700033D05838507E5B79E
:101D40000145C5BF81471397870161876343C7007A
:101D5000828013972700B386E50094422A9785076F
:101D600014C3D5B77D1662066186014793178601B5
:101D7000E18763D50700133517008280931726008B
:101D8000B306F500AE9794429C437D16B58F5D8FE8
:101D9000F1BF8A05AA9501476363B500828083A6D7
:101DA000C5FFF11593D71600D98F9CC11397F60183
:101DB000E5B72A830148014701456343D700828084
:101DC000B387050183A80700B30706019C43C697A4
:101DD000AA976384F80033B517010507B308030118
:101DE000620723A0F80061871108C1BF2A83014759
:101DF0008147014563C3D70082803388E50083288B
:101E00000800330EE600032E0E003388A840330886
:101E1000C8416384080133B508018507B308E300AE
:101E2000E20723A00801E1871107E9B717F3FFDFF5
:101E3000E702232B0111B286B2842E86AA850A8579
:101E400097000000E780C0FA2A84A6850A859700DB
:101E50000000E78020E833348000060413351500C5
:101E6000018D056117F3FFDF6700E32917F3FFDF3B
:101E7000E702A3244111AA89AE8A328BB68402C23A
:101E800002C402C60144131C8401135C8C416349E3
:101E90009C02939B1400FD1B0549138CF4FFF15C1D
:101EA00033048901620461846340740792478E049D
:101EB000CE9423AEF4FE410117F3FFDF67006323E6
:101EC00013192400B30B2B01014A93172A00D6974C
:101ED00083A50B0088437800340050009700000071
:101EE000E78040DA050A93178A01E187F11BE35E78
:101EF000FCFC92474E9905042320F900A2473EC2FC
:101F0000B24702C63EC441B7131A8901135A8A4127
:101F1000131D240093178A01E18763CF970092472E
:101F20000A044E941CC0A24705091379F90F3EC25A
:101F3000B24702C63EC4ADB7B3079A0313152A00D1
:101F400056950841780034005000050AEA97DA9760
:101F50008C4397000000E780E0D26DBF197106C284
:101F600012C416C61AC81ECA22CC26CE2AD02ED219
:101F700032D436D63AD83EDA42DC46DECAC0CEC2C9
:101F8000D2C4D6C6DAC8DECAE2CCE6CEEAD0EED2F9
:101F9000F2D4F6D6FAD8FEDA971500009385058CB0
:101FA0008841E700050092402242B2424243D243B8
:101FB0006244F244025592552256B2564257D257C5
:101FC0006258F25806499649264AB64A464BD64BBD
:101FD000664CF64C065D965D265EB65E465FD65F45
:101FE0000961730020300000972100209381810156
:101FF000175100201301018117F5FFFF1305C500DC
:102000009705002093850500171600201306C6FDCE
:1020100063FAC5008322050023A055001105910530
:10202000E3EAC5FE170502001305C5F69715002063
:102030009385C5FB171600201306C66563FAC50015
:102040008322050023A0550011059105E3EAC5FE92
:1020500017150020130505649745002093858526F4
:102060006377B500232005001105E36DB5FEFD4241
:10207000739002BC8D4273904280B722000093821D
:10208000828873900230970200209382A2F793E235
:1020900032007390523097520000938202897390FD
:1020A00012346FB0F47573002030397101436EC67D
:1020B00019A0397141536AC866CA62CC5ECE19A0B4
:1020C000397101535AD056D252D44ED64AD826DA54
:1020D00022DC06DE33016140828241114AC026C201
:1020E00022C406C68282B24D4101024D924C224C5E
:1020F000B24B4101024B924A224AB2494101024984
:1021000092442244B240410182803D432A87637356
:10211000C3029377F700BDEFADE5937606FF3D8AE6
:10212000BA960CC34CC30CC74CC74107E36BD7FE30
:1021300011E28280B306C3408A0697020000969699
:102140006780A6002307B700A306B7002306B700E1
:10215000A305B7002305B700A304B7002304B70005
:10216000A303B7002303B700A302B7002302B700FD
:10217000A301B7002301B700A300B7002300B700F5
:10218000828093F5F50F93968500D58D9396050182
:10219000D58D61B7939627009702000096968682A8
:1021A000E78086FA9680C1171D8F3E96E374C3F8C8
:1021B000A5B73367B500FD530D8B79E7B7877F7FF0
:1021C0009387F7F710419441B372F6003363F6003A
:1021D000BE92B3E262006397720C6318D606504158
:1021E000D441B372F6003363F600BE92B3E26200EC
:1021F0006398720A631BD60410459445B372F600C7
:102200003363F600BE92B3E262006391720A631E0A
:10221000D6025045D445B372F6003363F600BE9241
:10222000B3E26200639A72086311D60210499449BE
:10223000B372F6003363F600BE92B3E262006393BA
:1022400072085105D105E30FD6F6131706019397CF
:102250000601631CF7001357060193D706013305E7
:10226000F7409375F50F91E982804183C18333056F
:10227000F7409375F50F91E182801377F70F93F78D
:10228000F70F3305F74082800346050083C605003B
:10229000050585056313D60065FA3305D6408280AF
:1022A00011059105E312D6FE014582802105A105A5
:1022B000E31CD6FC014582803105B105E316D6FC4E
:1022C000014582804105C105E310D6FC01458280AD
:1022D000B717004003C777051377E70FA38BE70411
:1022E000130700F8A38DE7043D47238CE704130789
:1022F0005003A38CE70403C7A7051377D70F238DDB
:10230000E7048280B717004003C7E7020D89411137
:102310001377C70F498F93068008F3B6068093F6AC
:10232000860836C601000100930670052380D70495
:10233000930680FA2380D704010001002387E70277
:1023400023800704B247F3A7078001000100410181
:10235000828041112A83014E930E407E130F001993
:10236000930F400663E56E129308001913034006AD
:10237000B3781503854E0D4FA14F337365020D8958
:102380001335150063EFBE121308F6FF79467298F5
:102390004208135808013307C70213D61700BE07B7
:1023A00032976146B3F6C60213068070B386C60242
:1023B0003697A166F58F42075D8FB716004083C739
:1023C000F60293F70708A303F1000346710083C7E1
:1023D000F60293F70708E394C7FE83477100B71628
:1023E000004093F7F70F6388071293078008F3B74D
:1023F000078093F787083EC401000100B71700402B
:10240000930670052380D704930680FA2380D704AF
:102410000100010023AA070383C6170393E60608F9
:10242000A388D70223800704A247F3A707800100EF
:1024300001001166B71700407D16D45BC85F938515
:102440004703A98EF18EF5FA93068008F3B606804D
:1024500093F6860836C601000100930670052380B6
:10246000D704930680FA2380D7040100010098C1A5
:1024700003C7170313670704A388E7022380070431
:10248000B247F3A7078001000100410182807D135C
:102490003368E3039308E016630E08003368F30320
:1024A0009308D016630808009378330093B8180097
:1024B0009388D81633081E01131E0801135E0E01FF
:1024C00055B56393E5030548638608000148630337
:1024D00003002A8871087298FD15131E0801C205B1
:1024E000135E0E01C18179BD13F8150063F4BF00BE
:1024F0007908D5B713381800E5BF83C7F60293F7FC
:102500000708A303F1000346710083C7F60293F79F
:102510000708E394C7FE8347710093F7F70FF1DFD5
:10252000E9B531714AD966CB06DF22DD26DB4ED70D
:1025300052D556D35AD15ECF62CD6AC96EC7AA8C26
:1025400002D897100000E78020B12A8993078008FD
:10255000F3B7078093F787083EDA01000100B71749
:102560000040130770052380E704130780FA2380D7
:10257000E7040100010003C7F7021377770FA38771
:10258000E70203C7F70213678700A387E7022380E8
:102590000704D257F3A70780010001000545970003
:1025A0000000E78060D6130780C13347E902116A53
:1025B00093070AE893065002BD69930BA004814A71
:1025C000014B13048008930470057D1AB347F90288
:1025D0003307D7023EC0FD873ECC938709A69309F7
:1025E000803E3347F7023AC27D873AC43347390306
:1025F0008549B399990193D93940B306D702B30BF2
:102600007703B3C6F602B3CBFB0236C6FD8636C8E7
:1026100093D6FB4136CEB7460F0093860624334946
:10262000D9028566938606FAB3969601B389E902C4
:10263000130760553309D90293060010B389E902E4
:102640003349D902B3C9F9029316390036CA37198A
:102650000040FD8636D0930D090493D7F9413ED250
:10266000F336048093F6860836DC010001009307F8
:1026700070052380FD00930680FA2380DD000100B1
:1026800001008346390593F6860FA309D9048346D2
:10269000390593E61600A309D90423800D00E256FC
:1026A000F3A6068001000100130C80FA116DF336C9
:1026B000048093F6860836DE01000100930770055A
:1026C0002380FD0023808D01010001008346390530
:1026D000216693E60602A309D90483560905B3E6E9
:1026E000A6012318D90483560905D18E2318D904CD
:1026F00023800D00F256F3A60680010001008346F8
:10270000390593F606026381061A03463905218AC4
:102710006DDE081897100000E7800098733604807B
:1027200013768608B2C20100010023809D00238039
:102730008D0101000100B717004003C6370513766D
:10274000F60DA389C70403C6370513660602A389DD
:10275000C704835609052166B3E6A6012318D904E8
:1027600083560905D18E2318D90423800D0096467F
:10277000F3A60680010001008346390593F60602A0
:10278000638B061483463905A18AEDFE970000206D
:10279000E7806090AA8636D497000020E780A08F5B
:1027A000A256E30AD5FE835609054255B3E6A601B3
:1027B0002318D90497100000E780C08F834639059D
:1027C000A18AEDDE03560905834629058247337643
:1027D000CA00B306DA0293D5F641B296B388F64042
:1027E000E24733B8C6002E983308F840A247B3B684
:1027F00016013308D84063C70701631DF8009247EC
:1028000063FA1701C247634FF80E63950701B24799
:1028100063EAF80E894663E9660FF24693151800DD
:1028200013D3F8015E8613951800B365B30042D642
:1028300046D497C00100E78040DE3258050B137B79
:10284000FB0F63470001631A0838A25863870838F2
:1028500013081500B336A800B69513D6F5013298C3
:10286000B336C800AE9613581800FE06B3E606014C
:102870007336048013768608B2C6010001002380F7
:102880009D0023808D01010001000356C902B2960C
:10289000C206C1822316D90223800D00B646F3A6D4
:1028A00006800100010021B5F336048093F6860806
:1028B000B6C00100010023809D0023808D0101002E
:1028C00001008346390593E60602A309D904238053
:1028D0000D0086460DB5F336048093F68608B6C41F
:1028E0000100010023809D0023808D010100010073
:1028F0008346390593E60602A309D90423800D0017
:10290000A646BDB5E30B0BF0F336048093F68608BC
:10291000B6C801000100930680FA23809D00238041
:10292000DD00010001008346390593F5FC0F93F6A5
:10293000860FA309D90483463905CD8EA309D9048E
:1029400023800D00C646F3A6068001000100130592
:1029500080FA03463905930639051D8A631C9629BA
:102960007336048013768608B2CC0100010013068A
:1029700080FA23809D002380CD000100010003C662
:1029800006001376F60D2380C60003C60600136604
:1029900006022380C600835609051166D18E2318CE
:1029A000D904835609052166D18E2318D9042380C2
:1029B0000D00E646F3A6068001000100130680FA2A
:1029C0008346390593F60602638006268346390559
:1029D000130C3905A18AFDDA081897000000E7807A
:1029E000A06BF336048093F68608B6D00100010090
:1029F000930680FA23809D002380DD000100010002
:102A000083460C00116693F6F60D2300DC00834626
:102A10000C0093E606022300DC0083560905D18EE4
:102A20002318D904835609052166D18E2318D904A9
:102A300023800D008656F3A60680010001001306D0
:102A400080FA8346390593F60602638A0620834698
:102A50003905A18AEDFE97F0FF1FE780C0632A8C3D
:102A600097F0FF1FE7802063E30C85FF835609057D
:102A700011664255D18E2318D90497000000E780D3
:102A800060638346390513063905A18AFDDAF336FA
:102A9000048093F68608B6D401000100930680FAFC
:102AA00023809D002380DD00010001008346060095
:102AB00093F6F60D2300D60023800D00A656F3A64C
:102AC0000680010001008356090503462905D24707
:102AD000B376DA003306CA021305800C9355F6412B
:102AE0003696330DF6408257333CD6002E9C333653
:102AF000A601330CFC40330CCC40330885039256BE
:102B00004E86B335A5033305A503C29597C00100D2
:102B1000E780A0B063468001631E0C16630C0D169F
:102B2000130615003335A6002E959356F5013696FB
:102B3000B335D600AA959396F50105828585D18E89
:102B40006346B000639D051A638B061A0356C902DB
:102B500015823305D6003336C500B2956348B00000
:102B6000639105241306F00F637DA622894663F363
:102B7000561593078008F3B7078093F78708BED6EA
:102B80000100010037170040930770052300F70488
:102B9000930780FA2300F704010001008356C7025F
:102BA00089678117D58FC207C1832316F7022300D7
:102BB0000704B657F3A7078001000100FA506A54D2
:102BC000DA544A59BA592A5A9A5A0A5BFA4B6A4C49
:102BD000DA4C4A4DBA4D296182801308F5FF33352E
:102BE000A800FD152E951356F5013298B336C8008E
:102BF000AA9695B9F336048093F68608B6CA010002
:102C0000010023809D002380AD0001000100834668
:102C10003905CD8EA309D90423800D00D646F3A62D
:102C200006800100010035B3F336048093F6860870
:102C3000B6CE0100010023809D002380CD0001005D
:102C400001008346390593E60602A309D9042380CF
:102C50000D00F646F3A606800100010095B3F33699
:102C6000048093F68608B6D20100010023809D00FF
:102C70002380CD00010001008346390593E606025A
:102C8000A309D90423800D009656F3A606800100FF
:102C9000010045BB9306F5FF33B5A600FD152E9543
:102CA0009355F501AE96B3B5B600AA951396F50106
:102CB000858269B5F336048093F68608B6D801009C
:102CC0000100930680FA23809D002380DD0001002F
:102CD00001008356C9020566011693F6F60FD18EE0
:102CE000C206C1822316D90223800D00C656F3A660
:102CF000068001000100850A93FAFA0F95B233E6C7
:102D0000B60045C20356C9023305D0403338A0008F
:102D1000B305B040B385054115826345B000D1E1EC
:102D20006371A608894663F0560593078008F3B7D8
:102D3000078093F78708BEDA01000100B71700404B
:102D4000130770052380E704130780FA2380E70444
:102D50000100010003D7C7027D8B2396E702238081
:102D60000704D65781BDF336048093F68608B6DC97
:102D700001000100930680FA23809D002380DD007E
:102D8000010001008356C9020566011693F6F60F8D
:102D9000D18EC206C1822316D90223800D00E656C9
:102DA000B9B793078008F3B7078093F78708BEDEAB
:102DB0000100010037170040930770052300F70456
:102DC000930780FA2300F704010001000356C702AD
:102DD00093975600B297C207C1832316F7022300C8
:102DE0000704F657C1BB914763EEB70217D701003E
:102DF000130707208A05BA959C41BA978287B717AF
:102E0000004003A7470B1345F5FF698F23AAE70A84
:102E100003A7070B698F23A8E70A03A7070A798D81
:102E200023A0A70A8280B717004083A6470B134749
:102E3000F5FFF98E23AAD70A83A6070B558D23A881
:102E4000A70A83A6070A758F23A0E70A8280B7170F
:102E5000004003A7470B498F23AAE70A03A7070BE4
:102E60001345F5FF45BFB717004083A6470B13472F
:102E7000F5FF758F23AAE70A03A7070A598D4DB7F7
:102E8000B717004003A7470B498FEDB7914763EE93
:102E9000B70217D701001307E7168A05BA959C41B8
:102EA000BA978287B717004003A7470D1345F5FF70
:102EB000698F23AAE70C03A7070D698F23A8E70CE6
:102EC00003A7070C798D23A0A70C8280B7170040B9
:102ED00083A6470D1347F5FFF98E23AAD70C83A6C7
:102EE000070D558D23A8A70C83A6070C758F23A06B
:102EF000E70C8280B717004003A7470D498F23AA2C
:102F0000E70C03A7070D1345F5FF45BFB7170040B2
:102F100083A6470D1347F5FF758F23AAE70C03A778
:102F2000070C598D4DB7B717004003A7470D498FC0
:102F3000EDB7797122D43714004026D24AD0035914
:102F400024028354040206D64209C2044ECE52CC57
:102F500056CA13590901C1802DE11379F9F793F489
:102F6000F49F4209C20413590901C18093078008E4
:102F7000F3B7078093F787083EC401000100930769
:102F800070052300F404930780FA2300F404010081
:102F90000100231124032310940223000404A247F8
:102FA000F3A7078001000100B25022549254025945
:102FB000F249624AD24A45618280B7F507008146EC
:102FC0003000B105194597000020E7808081A247B5
:102FD00013972701E34A07FC1369090893E40440A7
:102FE00093098008F3B7098093F787083EC0010072
:102FF0000100930A700523005405130A80FA230088
:10300000440501000100231124032310940223002E
:1030100004048247F3A7078001000100294597F0C7
:10302000FF1FE7802031F3B9098093F989084EC268
:1030300001000100230054052300440501000100A4
:103040008357040293E707202310F40223000404AB
:103050009247B9B7B7170040884742054181937737
:10306000050491EB9377F5013755E80113050580C9
:103070003345F50282809377050C130700046397AC
:10308000E7009377F50137459C1CCDB72165130503
:1030900005D0828037E700E01C435443A183E20659
:1030A000D58F1CC1FD572320F7182322F7188280E3
:1030B00013178500B7E700E023A0E710618123A282
:1030C000A7108280B7F700E08847CC47828081470D
:1030D00037370040A14663C4C7003285828003456C
:1030E000B740E38EA6FE3385F5000345050085074E
:1030F0002304A740CDB797070020938727EF9C4371
:10310000173700201307071C3E95636EE50017373D
:1031100000201307274F6368A70017070020232705
:10312000A7EC3E858280FD57EDBF8280411122C40D
:1031300006C62A8497000000E78000F22947B307FB
:10314000E502B2408D83B3D7870222449507B3D7F7
:10315000E70237370040C207C1832316F700410159
:103160008280411137150E0006C697000000E780E7
:1031700020FCB7370040130770F82381E7000D47A4
:10318000A381E70013070004A380E7000547238716
:10319000E700B24041018280373700408347270073
:1031A0001A0593F7F703C98F93F7F70F2301F70079
:1031B0008280B737004003C7170019C9D98DA38093
:1031C000B70003C70700136787002380E7008280EA
:1031D00093C5F5FFF98DA380B7008280AE872A875B
:1031E000B736004021463738004089E71703000012
:1031F0006700E3F383C8B600E30916FF05078348B9
:10320000F7FFFD17C20723041801C183F9BF41115D
:1032100022C406C62A8497000000E780E0E329471D
:10322000B307E502B2408D83B3D7870222449507E6
:10323000B3D7E70237370040C207C1832316F740F0
:1032400041018280716541111305052006C6970072
:103250000000E78000FCB7370040130770F82381B7
:10326000E7400D47A381E74013070004A380E74030
:1032700005472387E740B24041018280CC4141119C
:1032800006C6328503C6150083C5050022064D8E8D
:1032900042068D654186138875A2630C0611634B47
:1032A000C804138845A26300060D634AC8009385CD
:1032B00035A26301B6082390060029464DA0138865
:1032C00055A26305060D938565A2E316B6FE8D45EE
:1032D0001D4663E6E5081146198E63F3C7003E8676
:1032E000B7E704002390C600FC4797D501009385FB
:1032F000A5D39DA0138895A263030611634E060D06
:103300001388A5A263000613938505A5E315B6FAF5
:1033100099451D4663E5E504198E63F3C7003E86B3
:10332000B7E704002390C600FC479705002093856B
:1033300025D61DA09D451D4663E3E5022146198E55
:1033400063F3C7003E86B7E70400FC472390C6003E
:103350009705002093858534BA9582970146B2403F
:10336000328541018280AD451D46E3EAE5FE3146E6
:10337000198E63F3C7003E86B7E704002390C600AA
:10338000FC4797D501009385A5CCF9B7B1451D46FB
:10339000E3E7E5FC3546198E63F3C7003E86B7E7E1
:1033A00004002390C600FC4797D50100938545CBC8
:1033B00065B78D451D46E3E4E5FA1146198E63F3C2
:1033C000C7003E86B7E704002390C600FC4797D5A8
:1033D0000100938525C649B78D451D46E3E1E5F813
:1033E0001146198E63F3C7003E86B7E704002390A9
:1033F000C600FC4797D50100938545C8B1BFA545D8
:103400001D46E3EEE5F42946198E63F3C7003E86B8
:10341000B7E704002390C600FC4797D501009385C9
:1034200025C21DBFB5451D46E3EBE5F23946198EB1
:1034300063F3C7003E86B7E704002390C600FC474D
:1034400097D50100938545BD01BFB7E7040003A3ED
:103450000713970600209386A6C24146A545170587
:1034600000201305E5B802832D455DE703C505007F
:103470000947631FE50803A84500411106C6034735
:10348000180032850346080022074168518F9308CF
:1034900028FE6307170563E9E800051863030703BF
:1034A00023900600294591A8130648FE630AC70425
:1034B0001518E31707FF15463E87637BF60015478F
:1034C00001A8130600023E876374F600130700028A
:1034D000B7E704002390E600FC471316070111A884
:1034E0003E8691C30546B7E70400FC472390C6001B
:1034F0004206CC45418282970145B240410182801B
:10350000130600083E87E375F6FC13070008C9B7E9
:103510002390060005458280828041677917630405
:10352000E504411122C406C685472A84639FF5003D
:10353000B7E7040022852244B24003A3871397050E
:1035400000209385E52F4101028389476399F500A7
:10355000B7E7040083A7070B8545829771D9B2406E
:103560002244410182808280797126D252CCAE847D
:103570002A8A97D50100938565B217D501001305F6
:1035800065B406D63AC622D44AD0368432894ECEA5
:1035900097B00100E780A053A28517D5010013055D
:1035A00065B397B00100E7808052294597B00100CC
:1035B000E780C05683C7840093F70702F9E383C905
:1035C00004008947054532476396F908D44083C70C
:1035D000160083C60600A207D58FC166138616FEA5
:1035E000638CC7028D16638FD7068D6693862690EF
:1035F00029456391D706B7E70400A286225403A3A6
:103600004714B250F2494A86A6850259925452850F
:10361000624A8547456102832D450DEF93070002FD
:10362000354563E98702B7E70400FC47C844130641
:103630000002CA8582978149970700209387072156
:103640009C43014581CB9C4391C74E852286CA8508
:1036500082970145B250225492540259F249624A6B
:10366000456182802D457DF79307700F3545E3E373
:1036700087FEB7E70400FC47C8442286CA858297C4
:1036800065BF2145C1BF411122C437E4040083272F
:10369000841326C2AA84416506C697050020938537
:1036A000251A7D1582978327C40A17050000130584
:1036B00005E78588829795C0032304132244B2400E
:1036C000924497060020938626AE4146C5451705CD
:1036D00000201305659C41010283B24022449244BC
:1036E00001454101828019C59707002023A0A71634
:1036F00001458280454582801147636AA70A97D6B3
:103700000100938666980A0536951841411106C650
:103710003697AE87B2850287130700026145639D25
:10372000E700B7E70400FC47130600021705002076
:10373000130545F782970145B24041018280054754
:103740006145E39BE7FEB7E70400FC470546170524
:103750000020130525F7F9BF1307700F6145E39D9E
:10376000E7FCB7E70400FC471306700F17050020BD
:10377000130585F5C1B7130700086145E39EE7FA15
:10378000B7E70400FC4713060008170500201305DF
:1037900025034DB715476145E390E7FAB7E7040005
:1037A000FC471546170500201305C50961B70945F3
:1037B0008280411126C2B7E4040083A7C41322C447
:1037C0004AC006C62E8497050020938565072A897E
:1037D0008297058905C5970700209387E78B83D7D4
:1037E000A70BA28503A3440D2310F4002244B2408A
:1037F00092444A850249014641010283B240224473
:103800009244024949454101828097070020238163
:1038100007049707002023AF0702B717004003A74C
:10382000070CB706C0FFFD16758F23A0E70C03A792
:10383000070DB7064000558F23A8E70C03A7070C18
:103840003D9B23A0E70C03A7070D1367070123A8DF
:10385000E70C8280B717004003A5470C83A7470CED
:10386000598113451500C18B058999E3136525001E
:103870009707002083C7C7FD6380A7029707002032
:103880002388A7FC11C9970700209387A7FC03A3EF
:1038900007006303030002838280114517F3FFFFD3
:1038A000670063C8011122CC06CE3714004026CA37
:1038B0004AC84EC652C483447405034AB4058349BA
:1038C00084050349940597F0FFFFE780A0A0834794
:1038D000A40593F4F40F137AFA0F93E71700230D5E
:1038E000F40493F9F90F1379F90FB717004003C7E0
:1038F000A705058B6DFF03D5C705A38D4705238C51
:103900003705A38C2705A38B9704F2406244D24469
:103910004249B249224A05618280411193970501CB
:1039200022C406C626C2C1872E8463DC0700B7E422
:103930000400FC54829719C1BC5482972165218DE3
:1039400015A893F7150013C515008DE793F725000B
:103950009DC797000000E78020F0B7E70400BC4F48
:103960001306000A894517050020034525EF8297B5
:1039700013452400B240224492444101828093972F
:10398000250163D80702B7E4040083A7C41E829709
:1039900097000000E780A0F0BC4C375607001306E4
:1039A0000630896517050020034545EB82970965B8
:1039B00079B7939715010145E3DE07FA17C50100B2
:1039C0001305457997B00100E7804028B7E7040068
:1039D000BC4F13060064916517050020034505E8F8
:1039E00082971165A9BF1D71A2CC37E404005C5C0D
:1039F000485886CE494697C5010093852571829720
:103A000011E917C501001305A57197B00100E78002
:103A1000E02301A0B7F600E0795798CAFD57DCCA49
:103A20000567B7E700E023A0E7101306F00290C295
:103A300023A0E718010001003707002018471306EC
:103A4000000481459706002023A8E6E04157A38A99
:103A5000E7403C4408088297970700209387077D3A
:103A60003EC8856713870740938757D1231AE10023
:103A70002312F1021307B00F97F7FFFF9387C76474
:103A80002310E1023ED81547970700009387C7E14E
:103A9000B7F50700A30FE1003EDC054797070000DC
:103AA0009387E7DF81463000E10519452301E102F4
:103AB0003EDE97F0FF1FE780C0D218088147994685
:103AC00030003E960346060085070507A30BC70096
:103AD000E398D7FEC24791C70357410185676373D7
:103AE000F70001A0B7E7040083A7470A08088297F8
:103AF000AA8511C917C501001305C56397B0010058
:103B0000E780E0FC01A0F640664425618280411117
:103B100026C2B7E4040083A7040806C622C417051A
:103B200000001305C5DF829717040020130404D397
:103B30002300A40097000000E780800297000000A7
:103B4000E780E0CC03450400224403A38405B2408F
:103B5000924413060032896541010283797106D6C9
:103B600022D413078008F337078093F787083EC2F3
:103B700001000100B7170040930570052380B704CA
:103B8000130680FA2380C7040100010083C6F702F0
:103B900093F6A60FA387D702238007049246F3A6C5
:103BA00006800100010073370780137787083AC445
:103BB000010001002380B7042380C7040100010035
:103BC00003C7F70213672700A387E70223800704D0
:103BD000A247F3A7078001000100054597E0FFFF1A
:103BE000E780807297000000E78060CB0147814644
:103BF0008147054685451305407E97E0FFFFE78036
:103C0000807537E404003C44680051468145829742
:103C1000B707C0A83EC8B787E803938707D03ECA56
:103C200097E7FF1F9387A7793EC67C586800829765
:103C3000B250225445618280411197D5010093858D
:103C4000A5B317C501001305E54706C697B00100E7
:103C5000E780E0E717D501001305C5CA97B001005A
:103C6000E780E0E6B2402945410117B30100670053
:103C7000E3EA411197D50100938545B117C50100CD
:103C80001305454406C697B00100E78040E417D508
:103C900001001305E5C597B00100E78040E3B2409D
:103CA0002945410117B30100670043E7411122C4D0
:103CB00006C6834705002A849DC797D501009385D2
:103CC000A5B217C501001305E53F97B00100E780D5
:103CD00000E04C4017D50100130505D597B0010051
:103CE000E780E0DE3DA058410DEF97D501009385B8
:103CF000A5AF17C501001305E53C97B00100E780AB
:103D000000DD17D501001305A5D397B00100E780AA
:103D100000DC2244B2402945410117B3010067008D
:103D2000E3DFA1679386D7036313D70297D501001A
:103D3000938585AB17C501001305C53897B0010001
:103D4000E780E0D817D50100130585D07DBFED07CA
:103D500097D50100938545A917C501001305853640
:103D6000631BF70097B00100E78060D617D501000C
:103D7000130545CF59BF97B00100E78040D54C40AF
:103D800017D50100130505D091BF411197D501004A
:103D9000938505A117C501001305C53206C697B066
:103DA0000100E780C0D2B2402945410117B30100AC
:103DB0006700C3D6797122D426D24AD02E842A89AC
:103DC0008145B2844800714606D697E0FFFFE78040
:103DD000003497F7FF1F9387275EDC4783D70700E0
:103DE000231421012313F10097500000E780C0E75E
:103DF0008547A305F1009307401F3EC6FD572305E5
:103E0000A100230AF10097500000E78020FA2686DF
:103E1000A285480097500000E780E0E7B2502254A6
:103E2000925402594561828097270020239307907E
:103E300097170020238C077EB7E70400BC47411189
:103E400006C641468145170500201305A52C82971B
:103E5000170700200347072E9307F00A6315F702A0
:103E60009307F0F88945170500201305A52C1707BF
:103E700000202301F72C97070020A38D072A9760C5
:103E80000000E78080A197600000E780E0CC9760A9
:103E90000000E78060CF81453705040097070020C8
:103EA00023A80726970700202392072697070020BC
:103EB000238F072497070020239E071C97070020C5
:103EC000239C071A970700202391072497070020B7
:103ED000239A072497300000E780402C0145976023
:103EE0000000E78080A497D501009385E58D17C574
:103EF00001001305251D97B00100E78040BD17D5CF
:103F00000100130565BE97B00100E78040BCB240D8
:103F10002945410117B30100670043C041118146A3
:103F200017F6FF1F13068646854517050020035523
:103F3000651406C697C00000E780202B15C997D5E9
:103F400001009385258917C501001305A51797B0B2
:103F50000100E780C0B717D501001305E5A897B0A9
:103F60000100E780C0B6294597B00100E78000BB9B
:103F700097D501009385058617C5010013058514A3
:103F800097B00100E780A0B417D50100130505A77D
:103F900097B00100E780A0B3294597B00100E78002
:103FA000E0B797F7FF1F93872741DC47054797D571
:103FB0000100938525822390E70017C501001305B2
:103FC000651097B00100E78080B017D50100130598
:103FD00025A497B00100E78080AFB2402945410198
:103FE00017B30100670083B3011122CC06CE26CAA5
:103FF0004AC84EC693F715002E84B5CB9700000033
:10400000E78000F2930710F8170700202304F71247
:104010009707002083D7C70517070020A30CF710C8
:104020009145A183170500201305C510170700202F
:104030002303F71097070020A38F070E9760000057
:10404000E780A085B7E70400BC4F13060014930572
:104050000010170500200345E580829713451400E2
:10406000F2406244D2444249B2490561828093F7EA
:104070000510B1C3054597600000E780008B171558
:1040800000200355056B97500000E780805697206D
:104090000000E780A0269707002083C7F71889E76C
:1040A00097600000E78040AB97600000E780C0ADFC
:1040B0001345041075B793F72500E9CF17070020C3
:1040C0000357C70469C7AD64B71900409384A4AA15
:1040D00023A099009706002093868603944297D7E1
:1040E0000100938767A21706002003464602814518
:1040F000170500201305050297700000E780A02A2D
:1041000023A0990097F7FF1F239CA71A2A8941C172
:1041100097C501009385C57217C50100130585FA7F
:1041200097B00100E780A09ACA8517C50100130562
:10413000251197B00100E7808099294597B00100CB
:10414000E780C09D97070020239207FC930710F893
:10415000170700202300F7FE9707002083D747F1B9
:1041600017070020A308F7FCA183170700202304EA
:10417000F7FC91458D47170500201305A5FB170790
:104180000020A30AF7FA97500000E780007113455A
:104190002400F9B593F74500D1C397C50100938575
:1041A000256A17C501001305E5F197B00100E78006
:1041B000009217C501001305650A97B00100E7805A
:1041C0000091294597B00100E7804095930720F8BA
:1041D000170700202300F7F69707002083D787EB07
:1041E00017070020A308F7F4A18317070020230472
:1041F000F7F4854717070020A30FF7F29750000048
:10420000E780C0BA170500201305C5F29145975005
:104210000000E78080681345440099B593F7850056
:10422000A9C797C501009385A56117C501001305AE
:1042300065E997B00100E780808917C50100130583
:10424000250397B00100E7808088294597B00100D9
:10425000E780C08C97070020239A07EA9770000038
:10426000E780402413458400E5BB93F70501D1C3E3
:104270008545170500200355E5E197600100E780BB
:1042800000DA97C501009385A55B17C501001305EA
:1042900065E397B00100E780808317C5010013052F
:1042A00065FE97B00100E7808082294597B0010044
:1042B000E780C086930730F817070020230CF7E645
:1042C0009707002083D707DD17070020A304F7E630
:1042D00017050020130505E6A1838D45170700206B
:1042E000230BF7E497500000E780205B134504019F
:1042F00085BB93F70502D1C797C501009385455447
:1043000017C50100130505DC97A00100E780207C9C
:1043100017C50100130545F997A00100E780207B30
:10432000294597A00100E780607F930740F81707B1
:1043300000202301F7E09707002083D7E7D3170772
:104340000020A309F7DEA183170700202305F7DE6D
:10435000854717070020A300F7DE97070020239D5D
:1043600007D097500000E78060A4170500201305D0
:1043700065DC914597500000E78020521345040208
:10438000C5B193F70504FDC397C501009385454B5F
:1043900017C50100130505D397A00100E78020731E
:1043A00017C501001305C5F197A00100E780207231
:1043B000294597A00100E78060769707002083C712
:1043C00067D71307700A6386E7061307800A638CB2
:1043D000E7081307600A6393E704930760F8170779
:1043E00000202309F7D49707002083D707D21707A7
:1043F0000020A301F7D4A18317070020230DF7D2D3
:10440000854717070020A30CF7D2B14517050020F8
:10441000130545D297500000E780204897500000D0
:10442000E780C0981345040497070020239F07CC1A
:1044300005B9930770F817070020230DF7CE9707EB
:10444000002083D787CC17070020A305F7CEA183D0
:10445000170700202301F7CE854717070020A30D7B
:10446000F7CC994565B7930780F8F1B793F705083E
:104470000145E38707BE97C501009385653C17C5D5
:104480000100130525C497A00100E780406417C50B
:104490000100130565E497A00100E780406329450A
:1044A00097A00100E78080679307A0F81707002016
:1044B0002302F7C89707002083D7C7C61707002035
:1044C000A30AF7C6A183170700202306F7C685476E
:1044D00017070020A301F7C697070020239407C4FD
:1044E00097500000E780808C17050020130585C4D5
:1044F000914597500000E780403A134504088DB677
:10450000411122C497C501009385452F2A8417C500
:104510000100130525BB06C697A00100E780205BBC
:104520004C4017C501001305A54997A00100E7807D
:10453000005A294597A00100E780405E0347040028
:104540009307F00F631FF70297C501009385052BB2
:1045500017C50100130505B797A00100E780205794
:104560004C4017C501001305A54697A00100E78040
:1045700000562244B2402945410117A301006700BB
:10458000E359B240224441018280411122C426C233
:104590002A84AE8417C501001305C5B297C5010072
:1045A0009385852106C697A00100E780405217C574
:1045B00001001305E55197A00100E780405129450E
:1045C00097A00100E780805597C501009385C51E1F
:1045D00097070020239087AA17C50100130585AE11
:1045E000054497070020239597A89707002023925A
:1045F00087A897170020239E971297A00100E780B5
:10460000004D9715002083D5C51217C5010013056D
:10461000A54C97A00100E780804B294597A0010099
:10462000E780C04F971700202382870097F7FF1F6E
:10463000938787D8DC4717F5FF1F0345A52203D7CB
:104640000700C167FD17631EF700B7E7040003A367
:1046500087051306000A85452244B2409244410171
:104660000283B7E7040003A387051306001493052C
:104670000010DDB7B1C1411122C417C501001305F7
:1046800065A42E8497C501009385451206C697A0A0
:104690000100E780C043A28517C5010013058542CC
:1046A00097A00100E780A0422244B2402945410181
:1046B00017A30100670083468280011122CC37E4F2
:1046C00004005C5C06CE354697C501009385C52481
:1046D00017D501001305C5F1829711E917C501002F
:1046E000130505A497A00100E780405601A097F7A5
:1046F000FF1F9387E7173EC4B7F5070085679387C9
:104700000780814617F6FF1F13060616E1051945B7
:104710003EC697E0FF1FE780C00C7C44194697F522
:10472000FF1F93856514170500201305E5968297F2
:10473000340017F6FF1F1306261397C50100938553
:10474000A56D17C501001305A56E97700000E780E1
:10475000809A2A841DCD97C501009385650D17C5E4
:1047600001001305259697A00100E7804036A28539
:1047700017C501001305451B97A00100E7802035F0
:10478000294597A00100E7806039F2406244056145
:10479000828097E00000E780800017C501001305C4
:1047A000A50F97600000E780C08E97A00000E7800B
:1047B000C05497600100E78040B917F5FF1F13054B
:1047C00025BC97600100E780E0A117C50100130533
:1047D000A50D97600100E780C0B92A8497600000AA
:1047E000E78000F597100100E78020919780010095
:1047F000E780402A97700000E780E0509760000053
:10480000E780006B97300100E780805297C5010078
:104810009385050217C501001305C58A19C897A01D
:104820000100E780C02AA28517C501001305051203
:10483000A1B797A00100E780802917C501001305E3
:10484000251397A00100E7808028294597A0010043
:10485000E780C02C97300100E780602E97F00000C1
:10486000E780204D7DC58545370504009730000061
:10487000E780C09297C50100938585FB17C50100AD
:104880001305458497A00100E780602417C5010047
:104890001305850F97A00100E7806023294597A0A5
:1048A0000100E780A02797F7FF1F938767A083D7B2
:1048B000070017170020231EF7E68547171700206B
:1048C0002306F7D697F7FF1F938707AFDC4703D779
:1048D0000700C167FD176316F70097F0FFFFE78039
:1048E000206497700000E78020CC1305C5149770F2
:1048F0000000E78020CC97200000E780E0B39720FD
:104900000000E780A09F17150020035585E297500F
:104910000000E78000CE054597500000E780E000EA
:1049200097500000E780402697C50100938545F029
:1049300017B501001305057997A00100E78020193C
:1049400017C501001305850697A00100E780201810
:1049500005BD97C501009385A5ED17B501001305A9
:10496000657697A00100E780801617C50100130542
:10497000A51797A00100E7808015294597A00100A1
:10498000E780C019014597500000E78000FA69BF31
:10499000411122C437E404008327041A06C6829713
:1049A00097500000E780A0C88327040817F5FFFF91
:1049B0001305C563829797F7FF1F2385A7EA17F5AD
:1049C000FF1F1305659F97400000E780C0702244D9
:1049D000B240410117030000670063CEB7E704004F
:1049E000FC471171A2DDCAD986DFA6DBCED72E84A3
:1049F00032892E86AA8517F5FF1F1305A5738297A6
:104A000017F7FF1F130707738347070093068002FA
:104A10009387E70793F7F70FE3ECF610BA898A0755
:104A200017B7010013074773BA979C43BA97828759
:104A30008D4797C501009385E5E117B50100130582
:104A40006568630FF40097A00100E780400817C570
:104A500001001305E59E97A00100E7804007BDA473
:104A600097A00100E780A00617C501001305C59EA9
:104A700097A00100E780A005294597A00100E780E5
:104A8000E009930720F8114697F5FF1F9385856A83
:104A90004A8517F7FF1F230FF76897F7FF1FA38CAF
:104AA000076897F0FFFFE78020312A841DC997C56A
:104AB0000100938525DA17B501001305A56097A0BD
:104AC0000100E780C000A28517C501001305859C81
:104AD00097A00100E780A0FF294597A00100E7808B
:104AE000E00397C501009385E5D617B501001305CE
:104AF000655D97A00100E78080FD17C501001305E3
:104B0000A59A97A00100E78080FC294597A00100A5
:104B1000E780C0004165930730FA054697F5FF1F0F
:104B2000938545617D1517F7FF1F2305F76097F003
:104B3000FFFFE78060282A841DC997C5010093857F
:104B400065D117B501001305E55797A00100E7806F
:104B500000F8A28517C501001305C59397A00100B1
:104B6000E780E0F6294597A00100E78020FBB7E742
:104B70000400BC4F0566130606C8A14517F5FF1FC4
:104B8000034545CE8297FE506E54DE544E59BE59B1
:104B90001161828091476303F40297C501009385F8
:104BA00065CB17B501001305E55197A00100E7801B
:104BB00000F217C501001305659271BDB7E7040047
:104BC000FC4F914517F5FF1F0345C5C9829797C54F
:104BD0000100938525C817B501001305A54E97A0C0
:104BE0000100E780C0EE17C501001305E59097A00E
:104BF0000100E780C0ED294597A00100E78000F2A1
:104C000097400000E780801A914535A485476303EB
:104C1000F40297C501009385E5C317B5010013059C
:104C2000654A97A00100E78080EA17C501001305D7
:104C3000258E15B597F7FF1F239E2745B7E704007C
:104C40000566BC4F130606C8C1450DBF8D476303FB
:104C5000F40297C501009385E5BF17B50100130560
:104C6000654697A00100E78080E617C5010013059F
:104C7000E58BD5B3930740F8114697F5FF1F938551
:104C8000654B4A8517F7FF1F2306F74A97F7FF1F63
:104C9000A383074A97F0FFFFE78000122A84E3040A
:104CA00005EE97C501009385E5BA17B50100130518
:104CB000654197A00100E78080E1A28517B501005A
:104CC0001305457D97A00100E78060E0294597A086
:104CD0000100E780A0E445BD9147E31CF4F6B7E787
:104CE0000400FC4F9305000217F5FF1F034585B72D
:104CF000829797C501009385E5B517B501001305A7
:104D0000653C97A00100E78080DC17C50100130512
:104D10006583F1BD894763E3870297C501009385E9
:104D200065B317B501001305E53997A00100E780C9
:104D300000DA17C501001305258231BB97F4FF1F68
:104D400083C4643F97F7FF1F83C7D73E97C5010011
:104D5000938545B0A20417B501001305A536DD8C77
:104D600097A00100E780A0D6A28517B50100130522
:104D7000E57F97A00100E78080D5C204294597A070
:104D80000100E780A0D9C1849305D4FF9396040164
:104D9000C1824A8693F5F50F17F5FF1F1305B53944
:104DA00097200000E7804043E35F90DC930750F8D2
:104DB00017F7FF1F2300F73883C73900228697F5BE
:104DC000FF1F9385253785074A8517F7FF1FA30423
:104DD000F73697F0FFFFE78020FE2A84E30505DA27
:104DE00097C50100938505A717B501001305852D0B
:104DF00097A00100E780A0CDA28517C5010013058B
:104E000065CBC9B5894763E3870297C501009385E0
:104E100065A417B501001305E52A97A00100E780F6
:104E200000CB17B501001305257635B1974000007A
:104E3000E780C0F7A28517F5FF1F1305A52F975030
:104E40000000E78080A581B38D476303F40297C516
:104E50000100938525A017B501001305A52697A08D
:104E60000100E780C0C617B501001305A573E5B6BC
:104E7000B76602000146B7750200054597E0FF1FBF
:104E8000E7802096930760F817F7FF1F2304F72A9F
:104E900097F7FF1FA381072A9307000617F7FF1F45
:104EA000230CF728894717F7FF1FA307F72897F761
:104EB000FF1F2384072897F7FF1FA3800728C147F8
:104EC00017F7FF1F230CF726930720F917F7FF1F8B
:104ED000A306F726314697F7FF1FA382A72697F56B
:104EE000FF1F938525254A8597F7FF1F23890724F0
:104EF00097F0FFFFE78040EC2A84E30605C897C5DA
:104F000001009385259517B501001305A51B97A0F2
:104F10000100E780C0BBA28517B501001305056A33
:104F200055B3B1476303F40297C501009385859299
:104F300017B501001305051997A00100E78020B9F6
:104F400017B501001305456939B6B7E70400FC4FF2
:104F50009305000417F5FF1F0345C59082979740FE
:104F60000000E780A0E4B145F9B5914763E387020B
:104F700097C501009385058E17B5010013058514AB
:104F800097A00100E780A0B417B50100130585665E
:104F9000D9B497F4FF1F83C4241A97F7FF1F83C760
:104FA0009719A204DD8C8E04B77702006D14BE94AD
:104FB0002286A68517B501001305056597A0010097
:104FC000E780E0B0B7E70400FC47228697F5FF1FB3
:104FD000938595162800829793160401C1823000AC
:104FE000A685094597D0FF1FE780A07F2A8409C9BD
:104FF00017B501001305056397A00100E78000C500
:10500000930770F8194697F5FF1F9385A5124A85F7
:1050100017F7FF1F2300F71297F7FF1FA38E8710C4
:1050200097F0FFFFE78040D92A84E30E05B497C5C7
:1050300001009385258217B501001305A50897A0E7
:105040000100E780C0A8A28517B501001305855EA1
:1050500095B99947630BF41297B501009385857F45
:1050600017B501001305050697A00100E78020A6EB
:1050700017B501001305855DF9BA914763E387020F
:1050800097B501009385057D17B5010013058503CC
:1050900097A00100E780A0A317B501001305855C68
:1050A0005DBA97F4FF1F83C4240997F7FF1F83C7D6
:1050B0009708A204DD8C8E04B77702006D14BE94AD
:1050C0002286A68517B501001305055B97A0010090
:1050D000E780E09FB7E70400FC47228697F5FF1FB3
:1050E000938595052800829793160401C1823000AC
:1050F000A6850D4597D0FF1FE780A06E2A8409C9B9
:1051000017B501001305055997A00100E78000B409
:10511000930780F8194697F5FF1F9385A5014A85E7
:1051200017F7FF1F2308F70097F7FF1FA3868700D5
:1051300097F0FFFFE78040C82A84E30605A497B5EF
:1051400001009385257117B501001305A5F797A0F8
:105150000100E780C097A28517B501001305C5546B
:1051600095B699476303F40297B501009385856E60
:1051700017B50100130505F597A00100E7802095FC
:1051800017B501001305C553F9B0B7E70400FC4F8C
:105190009305000417E5FF1F0345C56C82979740F0
:1051A0000000E780A0C0994579B18D476303F40200
:1051B00097B501009385056A17B50100130585F0C1
:1051C00097A00100E780A09017B501001305C55016
:1051D00059B017B501001305255197A00100E780CC
:1051E000E0A61305C01297D0FF1FE7808015014588
:1051F00097E0FFFFE78040EA0D4597100000E78049
:10520000E09F294597D0FF1FE780A01397D0FF1F8D
:10521000E78000048DBA99476303F40297B5010053
:105220009385456317B501001305C5E997A00100F3
:10523000E780E08917B501001305C54B29B817F7BA
:10524000FF1F034777EF97F7FF1F83C7E7EE22079C
:105250005D8F9166BA96C2061166C1821306F6EF9B
:105260008D476365D60297E7FF1F9387E7149C4B32
:1052700017F6FF1F034636EC9386C7002DC203D6F0
:10528000070069CA8907E39CD7FE89471307A0F87E
:10529000114697F5FF1F9385E5E94A8597F6FF1FAD
:1052A000238AE6E817F7FF1FA307F7E897F0FFFF49
:1052B000E78080B02A84E308058C97B501009385C8
:1052C000655917B501001305E5DF97A00100E780D8
:1052D0000080A28517B5010013050543E5B203D68A
:1052E0000700630EE60A8907E39BF6FE8D4779BF48
:1052F00091476304F40297B501009385A55517B54E
:105300000100130525DC97900100E780407C17B56C
:1053100001001305E5406FF00FF4B7E70400FC4F00
:105320009305000817E5FF1F0345C5538297C9B8C9
:1053300097B501009385055217B50100130585D86F
:1053400097900100E780A07817B501001305C53ECE
:105350006FF06FF02390E70017E5FF1F1305C505F9
:1053600097300100E78020A397B501009385854E13
:1053700017B50100130505D597900100E78020754A
:1053800017B501001305453C97900100E780207494
:10539000294597900100E78060788147C5BD23903B
:1053A000070017E5FF1F1305250197300100E7806F
:1053B000809E97B501009385E54917B50100130557
:1053C00065D097900100E780807017B50100130544
:1053D00025395DBF411122C406C6834705002A84D2
:1053E0009DC797B501009385A54217B50100130528
:1053F00065CD97900100E780806D4C4017B50100A6
:105400001305857197900100E780606CE1A0584119
:10541000B707CF009387777D631DF70697B5010027
:105420009385053F17B501001305C5C99790010085
:10543000E780E0691C448356E4008355C40003C63A
:10544000070017B501001305A56E97900100E780CE
:105450000068294597900100E780406C0357E400FD
:105460009707002083D7E72C6309F7008355C40012
:10547000084497E0FFFFE780A0D60356E400835579
:10548000C40008442244B240410117F3FFFF670003
:105490002355B707CC009387777D6315F70497B53D
:1054A00001009385E53617B501001305A5C1979056
:1054B0000100E780C0611C448356E4008355C400AA
:1054C00003C6070017B50100130585669790010014
:1054D000E780E05F2244B240294541011793010073
:1054E0006700C363B707CE009387777D6304F70235
:1054F00097B501009385C53117B50100130585BC2B
:1055000097900100E780A05C4C4017B5010013059F
:105510006557CDBDB240224441018280B7E7040007
:10552000FC4741112E8606C622C426C24AC02E84DC
:105530002A89AA8517F5FF1F1305C5BF829797B55E
:1055400001009385E53217B501001305A5B79790C3
:105550000100E780C05797F5FF1F83C5A5BD17B5AC
:1055600001001305E5D897900100E78040562945D2
:1055700097900100E780805A97F4FF1F938484BBC3
:1055800083C7040041479387070693F7F70F636EBD
:10559000F75A17B70100130767C68A07BA979C43E3
:1055A000BA9782879D476307F40297B501009385F8
:1055B000252C17B501001305E5B097900100E78091
:1055C000005117B50100130525D397900100E7801E
:1055D00000508DA497F7FF1F83C7D7B5DDCB17F712
:1055E000FF1F034757B597F7FF1F83C7C7B42207AD
:1055F0005D8F97F7FF1F83C727B4C2075D8F97F7AB
:10560000FF1F83C777B3E207D98F17F7FF1F232147
:10561000F7B083C7640097B501009385652517B57A
:105620000100130525AA17F7FF1F2302F7AE979075
:105630000100E780C04997F7FF1F938767AD8C4350
:1056400017F6FF1F0346A6AC17B50100130585CC5E
:1056500097900100E780A047294597900100E780D7
:10566000E04B97F7FF1FA38707AC2244B240924458
:105670000249930700F817F7FF1F230DF7AA9D456E
:1056800017F5FF1F130505AB410117430000670025
:10569000C32097600000E78060F097F7FF1F238C1E
:1056A000A7A89357850017F7FF1FA306F7A89357DE
:1056B00005012A8417F7FF1F2300F7A893578501D8
:1056C000014517F7FF1FA309F7A697600000E780C1
:1056D00040F197F7FF1F2382A7A697B50100938596
:1056E000251917B501001305E59D97900100E78086
:1056F000003E17F6FF1F034646A4A28517B501001A
:105700001305C5C2B1B7CD476303F40297B50100D5
:105710009385051617B501001305C59A97900100EA
:10572000E780E03A17B501001305C5C179BD37E43C
:1057300004007C44414697F5FF1F9385B59F17F5FC
:10574000FF1F1305259D829797F7FF1F83C7A79F0C
:1057500017F7FF1F0347179FA20703238405D98F5D
:1057600017F7FF1F2314F79A1306000A89452244EE
:10577000B2409244024917E5FF1F0345A50E4101BF
:1057800002838D476303F40297B501009385450EAC
:1057900017B501001305059397900100E7802033AA
:1057A00017B501001305C5C90DB517F4FF1F034454
:1057B000849897F7FF1F83C7F79797B501009385E4
:1057C000250B220417B501001305C58F5D8C97903A
:1057D0000100E780C02FA28517B50100130505B8A9
:1057E00097900100E780A02E294597900100E7805F
:1057F000E0320D4697F5FF1F9385C593228597E00C
:10580000FFFFE780605BAA8421C197B50100938503
:10581000250617B501001305E58A97900100E7807A
:10582000002BA68517B50100130585B497900100DC
:10583000E780E0292244B2409244024929454101CF
:10584000179301006700832D97F7FF1F2394878428
:10585000B7E70400116603A38705130606E8914520
:1058600039B78D476303F40297B50100938545006E
:1058700017B501001305058597900100E7802025E5
:1058800017B50100130585CA89B317F4FF1F034438
:10589000848A97F7FF1F83C7F78997B5010093851F
:1058A00025FD220417B501001305C5815D8C979075
:1058B0000100E780C021A28517B50100130585AC62
:1058C00097900100E780A020294597900100E7808C
:1058D000E0240D4697F5FF1F9385C585228597E047
:1058E000FFFFE780604DAA841DC197B50100938535
:1058F00025F817A501001305E57C97900100E780C6
:10590000001DA68517B50100130505A905B797E782
:10591000FF1F23938776B7E70400116603A387056B
:10592000130606E89305000299B5894763E38702E9
:1059300097B501009385C5F317A501001305857878
:1059400097900100E780A01817B501001305C5C0A6
:10595000ADB997E4FF1F83C4047E97E7FF1F83C799
:10596000777D97B501009385A5F0A20417A50100E6
:1059700013054575DD8C97900100E7804015A685DD
:1059800017B501001305C5A297900100E780201408
:10599000294597900100E7806018228697E5FF1F50
:1059A00093854579268597E0FFFFE780E0402A84CC
:1059B000630E051A97B50100938585EB17A50100C5
:1059C0001305457097900100E7806010A28517B518
:1059D00001001305259F99BD854763F98718834505
:1059E00019002244B24092440249B335B00097E70F
:1059F000FF1F238BB76A17B501001305E59D410111
:105A0000179301006700A30CA2852244B240924480
:105A10004A85024941011703000067006324994742
:105A20006303F40297B50100938585E417A501008F
:105A30001305456997900100E780600917B50100DB
:105A4000130545CB59B617E4FF1F0344C46E97E70F
:105A5000FF1F83C7376E97B50100938565E1220468
:105A600017A50100130505665D8C97900100E7807E
:105A70000006A28517B501001305859797900100D0
:105A8000E780E004294597900100E7802009194646
:105A900097E5FF1F9385056A228597E0FFFFE78062
:105AA000A031AA841DC197B50100938565DC17A5B7
:105AB00001001305256197900100E7804001A6854C
:105AC00017B501001305C59395B397E7FF1F239BF7
:105AD0008764B7E70400116603A38705130606E889
:105AE0009305000869B1854797B50100938545D8AE
:105AF00017A501001305055D630BF40097900100E5
:105B0000E780E0FC17B501001305C5907DBC9790B8
:105B10000100E780C0FB17B50100130525919790A0
:105B20000100E780C0FA294597900100E78000FF57
:105B30002244B2409244024997E7FF1F2398075C32
:105B40004101176300006700E39597B50100938555
:105B500025D217A501001305E55697900100E780AF
:105B600000F717B50100130525BD85B4B2402244E6
:105B70009244024941018280411106C622C497E045
:105B8000FFFFE780602321CD97E7FF1F83D7E75111
:105B900085072A8417E7FF1F2319F75097B50100DF
:105BA000938585CE97E7FF1F2392A75017A5010085
:105BB0001305455197900100E78060F1A28517B564
:105BC0000100130525EF97900100E78040F0224483
:105BD000B2402945410117930100670023F497E77C
:105BE000FF1F83D7C74CB2402244850717E7FF1F2A
:105BF000231FF74A41018280411122C491462A8421
:105C000017E6FF1F130606619D652D4506C697D052
:105C1000FF1FE78000BDB7F7070003C70701A547CF
:105C20006313F70001A09306001001469D6525450A
:105C300097D0FF1FE780E0BA97E7FF1F238C875CB0
:105C40002244B240914617E6FF1F1306A65C9D65ED
:105C50002945410117D3FF1F6700A3B81171CED7A3
:105C6000B7E9040083A7C904CAD917E9FF1F1309BC
:105C7000694CA2DD2E8686DFA6DB2E84AA854A85A6
:105C8000829797E7FF1F83C7E74A1307700A638568
:105C9000E710636DF7001307600A6385E704FE50A1
:105CA0006E54DE544E59BE59116182801307800A2A
:105CB0006385E7161307900AE393E7FE8D476306B3
:105CC000F41C97B50100938525F217A50100130573
:105CD000653F97900100E78080DF17B5010013054D
:105CE000E5ED25A08D47630CF40297B5010093857F
:105CF000A5EF17A501001305E53C97900100E7808B
:105D000000DD17B501001305A5E497900100E780B9
:105D100000DC294597900100E78040E049B78547BE
:105D200017B50100130585E417E7FF1F230EF736AB
:105D300097900100E78080F1B7750200B766020016
:105D40000146054597D0FF1FE780A0A9930760F89B
:105D500017E7FF1F2300F73E97E7FF1FA38D073CC0
:105D60009307002617E7FF1F2328F73CE577938763
:105D7000072117E7FF1F2313F73CB14597E7FF1FE4
:105D8000238F073A97E7FF1FA38BA73A4A8597000F
:105D90000000E780E01621B7914763E3870297B5DB
:105DA0000100938565E417A501001305A5319790BF
:105DB0000100E780C0D117B50100130525DDB1B79B
:105DC00097E4FF1F83C4443797E7FF1F83C7B736A5
:105DD000A204DD8C83A7C9046D14228697E5FF1FFA
:105DE00093859535280082978E0493160401B77524
:105DF0000200C1823000A695094597D0FF1FE780B9
:105E0000409E930770F817E7FF1F2305F732994567
:105E100097E7FF1FA382A73295BF914763E38702ED
:105E200097B50100938545DC17A501001305852969
:105E300097900100E780A0C917B50100130585D62A
:105E4000E9B597E4FF1F83C4242F97E7FF1F83C79B
:105E5000972EA204DD8C83A7C9046D14228697E5D2
:105E6000FF1F9385752D280082978E0493160401D9
:105E7000B7750200C1823000A6950D4597D0FF1F6F
:105E8000E7802096930780F8BDBF17B50100130582
:105E900025D497900100E78060DB930790F82304F6
:105EA000F100834719008D452800A304F1008347C2
:105EB00029002305F10097000000E7806004130526
:105EC000C01297C0FF1FE780C047014597D0FFFF72
:105ED000E780801C0D4597000000E78020D229450F
:105EE00097C0FF1FE780E04597C0FF1FE78040365F
:105EF0007DB397E7FF1F23A7A732828097E7FF1F95
:105F00009387473203A30700630303000283174309
:105F100000006700839841114AC09706002083D68D
:105F20004681328917D6FF1F0356264B22C426C24C
:105F300006C62A84AE8497000000E780205B35C146
:105F40002DC0994763FF970483471400034704005B
:105F5000A207D98F13978700A183D98FC207316712
:105F6000C1831307C755639EE70297D7FF1F83D7E7
:105F7000C746A301F400A1832302F40097F7FF1F93
:105F800083D7277B91C7A302F400A1832303F400E6
:105F9000A68517B50100130525C997900100E78074
:105FA00000B397F7FF1F83C76768A5C797D5FF1F83
:105FB00083D5A54217B501001305C5C89790010008
:105FC000E780E0B02686A28517D5FF1F0355E54080
:105FD00097000000E78080BA6306090497F7FF1F67
:105FE00083C7C764A1E397E7FF1F83C7E7239DCB60
:105FF00095C897E7FF1F83C7270B8DE722852244AB
:10600000B2400249A685924441011743000067004F
:10601000C38817B501001305E5C397900100E78019
:10602000E0C25DBFB24022449244024941018280F5
:10603000834755008345450017B50100130585BD0D
:10604000A207DD8D17930100670063A817B5010053
:10605000130545BB17930100670043BF8D4763F6E7
:10606000B708011126CA06CE22CC0344350097E4B6
:10607000FF1F83C4741B97B50100938565BEB337BA
:10608000800017E7FF1FA301F71A09C497B50100A5
:106090009385C5BD17B501001305C5BD97900100D7
:1060A000E780E0A297E7FF1F83C717186386970072
:1060B00097000000E780402C97400000E780C0ACCC
:1060C0009967938757EE2316F1006800854791453D
:1060D000A30781002307F10097000000E78040E25A
:1060E000F2406244D244056182808280894763F72E
:1060F000B708011122CC06CE26CA83442500854765
:106100002A84639DF404914763F5B7040345450071
:106110008347340022055D8D97D7FF1F239FA72A51
:1061200097000000E78060459967938767EE231426
:10613000F1008347340023059100A305F100834754
:106140004400954528002306F10097000000E780F1
:1061500020DBF2406244D24405618280FDF89967F9
:10616000938767EE2314F10097D7FF1F83D7E726A5
:10617000A305F10023050100A183E1B7828001118D
:10618000996722CCD51717F4FF1F1304244A231450
:10619000F1008347040026CA97F4FF1F93846459D3
:1061A0002305F10083D7040028009545A305F100DD
:1061B000A18306CE2306F10097000000E78040D4BB
:1061C00003D604008345040017B50100130585AB11
:1061D00097900100E780A08FF2406244D2440561AD
:1061E00082809D677971D9172316F10097F7FF1FF9
:1061F00083C7C74306D62307F100A9C3B7E7040046
:10620000FC47414697E5FF1F9385C5F01305F10054
:1062100082976800CD4597000000E78060CE97F533
:10622000FF1F83C5A54017B501001305A5A89790CA
:106230000100E780C089B25045618280B7E7040061
:10624000BC47414681451305F1008297D9B745C542
:10625000411106C622C4930750FA2300F5009307A4
:10626000A005A300F50089472301F5009147A3018C
:10627000F5009307B003A302F50097F7FF1F93877C
:10628000E73A83C70700230205002A842303F500A9
:1062900097E7FF1F938757F983C70700414697E5A4
:1062A000FF1F938525E7A303F50097F7FF1F83D70B
:1062B00047482304F500A183A304F50097D7FF1FE7
:1062C00083D7A7112305F500A183A305F500B7E740
:1062D0000400FC47310582972285F14597000000B4
:1062E000E780C01C230EA4002181A30EA400B240AD
:1062F00022444101828082805D710A8586C6A2C4E3
:1063000097000000E780E0F437E404007C448A85CD
:106310000810794682973C441305E10309468145FC
:106320008297101093050002014597D0FFFFE78088
:10633000E03CB640264461618280411122C426C2FD
:106340004AC02A84AE843289AA85856601462545DD
:1063500006C697C0FF1FE780C048A2852244B2400E
:10636000CA862686024992442945410117C3FF1F68
:10637000670023470111B7C7A55A22CC9387C733BB
:1063800017E4FF1F130454EA3EC4834704002C00A3
:106390002146196506CE3EC697000000E78020FA28
:1063A0008345040017B501001305C59F97800100C0
:1063B000E780E071F2406244056182800111A146EC
:1063C000300099652D4522CC06CE97C0FF1FE7808F
:1063D0004041A24737C4A55A1304C43363958702CA
:1063E000B24517B501001305258FB335B00097E707
:1063F000FF1FA38BB7E297800100E780406DF2405A
:106400006244056182809165A1463000938505F064
:106410002D4597C0FF1FE780C03CA247E38287FC61
:1064200097E7FF1FA38207E0814517B50100130519
:10643000E58CD1B77971D146700091652D4522D494
:1064400006D697C0FF1FE780C039B24737C4A55AA8
:106450001304F43563988702B7E70400FC4717E597
:10646000FF1F130525CB41460C08829717B5010085
:106470001305C58E97800100E780407DB2502254FD
:10648000456182809165D1467000938505E82D4570
:1064900097C0FF1FE780E034B247E38F87FA17B554
:1064A00001001305A58DF9B7C16769768146FD170F
:1064B00005061397060141836364B7003E85828019
:1064C0003307D50003470700B98F214713F817009A
:1064D000858363050800B18FC207C1837D171377D9
:1064E000F70F6DF78506F1B741C5A547054763F27C
:1064F000B70883471500034705003168A207D98F05
:1065000013978700A183D98FC207C1831308C85589
:10651000054763900707411106C622C426C20344FB
:106520002500914763F087049307540063ECF5025C
:10653000A301C50021822302C5009304340091C643
:10654000A302D500A1822303D5002A84A685970043
:106550000000E780A0F526942300A4002181A30079
:10656000A4000147B240224492443A85410182800E
:1065700005473A8582800111B7C7A55A22CC938777
:10658000E7342A842AC621462C00156506CE3EC46F
:1065900097000000E780A0DAA28517B50100130577
:1065A000658297800100E780805297000000E780B5
:1065B000E0D4F2406244056182800111A1463000BE
:1065C00095652D4522CC06CE97C0FF1FE780602140
:1065D000A24737C4A55A1304E43463958702B24531
:1065E00017A501001305857397D7FF1F2397B7DE03
:1065F000C205C18197800100E780604DF24062448E
:10660000056182809165A1463000938505EE2D4598
:1066100097C0FF1FE780E01CA247E38287FCD147B9
:1066200017D7FF1F231BF7DAD14517A50100130564
:10663000E570C9B721C1411126C206C622C4AE8485
:106640008DC52A8497000000E780806697E7FF1FCA
:1066500083C787BD99CB22852244B240A685924448
:1066600041011733000067004323B24022449244A3
:1066700041018280828001114AC806CE22CC26CAFE
:106680004EC693F715002E899DCBAD673717004096
:106690009387A7AA1CC3B7E70400BC4F13060019D1
:1066A000854517D5FF1F034525D38297134519004C
:1066B000F2406244D2444249B2490561828093F774
:1066C0002500638A071C17F7FF1F035767069547C6
:1066D00063F9E70C014417F6FF1F130666F59306EE
:1066E000300513055004130810049308B004130375
:1066F0009005930764006374F7043A84FD5997F496
:10670000FF1F83C4E4F297F7FF1F83C777F2A20449
:10671000DD8CAD679387B755638BF41463E3970AF9
:10672000A9679387A755638EF414A28517F5FF1FF9
:10673000130505F097000000E78000F031A2B307D1
:10674000860083C50700639AD50483C51700639646
:10675000A50483C527006392050583C53700639EA2
:10676000D50283C54700639A150383C75700639614
:106770006702A2890DE897F5FF1F83D565FBB385F6
:106780003541C20517F5FF1F130585EAC1814E95F6
:1067900097000000E78040EAE1A005044204418040
:1067A00089BF3A84FD598547E3EB87F45DC485458D
:1067B00017F5FF1F1305C5E797000000E780C0E746
:1067C00069A8B1679387C7556380F404B567938759
:1067D000D755E39CF4F4A28517F5FF1F130545E593
:1067E00097300000E780600B8947630FF40493053E
:1067F000E4FFC205C18117F5FF1F130585E397006C
:106800000000E780E04A89A097200000E780C0F7F9
:1068100097000000E780204911C9A28517F5FF1FE6
:10682000130505E197000000E78080480546A28532
:1068300017F5FF1F1305C5DF97F0FFFFE780E06D39
:1068400097200000E78040F4A68517A501001305F6
:10685000255997800100E7808027FD57E39DF9F0D7
:1068600097F7FF1F239607EC1345290091B5A285E2
:1068700017F5FF1F1305C5DB97F0FFFFE780807B4F
:10688000E1B7A28517F5FF1F130585DA97F0FFFF23
:10689000E780007C55BF93F745000145E38A07E098
:1068A00017A501001305055597800100E780003A00
:1068B00097300000E780002C13454900D5BB4111FB
:1068C00022C437E404005C5C06C6354697A5010087
:1068D0009385850417B50100130585D1829711E9C9
:1068E00017A501001305C55197800100E780003608
:1068F00001A08327041C82972A84054597C00000C5
:10690000E78040E997600100E780606E97600100D2
:10691000E780604397B00000E780C0FA2285B2406C
:106920002244410182804111054506C622C426C287
:1069300097C0FFFFE78020601305A00497B0FF1FFA
:10694000E780E076757585457D1597C0FFFFE78088
:10695000C0497D7585451305F53697C0FFFFE78073
:106960002053371400408327840A8D4513050020E7
:1069700093E707202324F40A97C0FFFFE780E0464F
:10698000B7E4040097D0FFFFE780008CC8589780D9
:106990000100E780A02B17B50100130565C597809E
:1069A0000100E780A02A8327840C8545414593E7B1
:1069B00007082324F40C97C0FFFFE780604D8D4546
:1069C0001305000897C0FFFFE780804C97C0FFFFCA
:1069D000E780607937A507001305051297C0FFFF10
:1069E000E7800075014597C0FFFFE780207B954554
:1069F0000545894717F7FF1F230EF7D297C0FFFF02
:106A0000E780607BB7E700E013070006238DE740CF
:106A10003707000423A0E71097D0FFFFE780E0FCD2
:106A200097D0FFFFE780E00E97000000E78060E965
:106A300097000000E780C09897000000E78020B82A
:106A400097E0FFFFE78000F597000000E7808027D0
:106A500097000000E780801083A704081705000056
:106A60001305A5C1829797D7FF1F2387A796BC4C14
:106A7000130600648545829797C0FF1FE780409703
:106A800001458280AD67371700409387A7AA1CC3D2
:106A9000B7E700E03707400023A0E7180100010036
:106AA000B7F7070003C70701A5476316F7009397D9
:106AB000450191C301A04111AE860146AA85254535
:106AC00006C697C0FF1FE780C0D1B240B7E700E01D
:106AD0003707400023A0E710410182804111B286B0
:106AE0002E86AA852D4506C697C0FF1FE78060CF7A
:106AF000B2400145410182809307000463ECC70462
:106B00001D71A2CC2A840808A6CACAC886CE32C67D
:106B100097800100E78040F0AD673717004093870A
:106B2000A7AA1CC3B7E400E03709400023A024193A
:106B300001000100B2461008A285294597C0FF1F39
:106B4000E78020CAF640664423A02411D644464973
:106B5000256182803955828041110D658D4506C6BB
:106B600097C0FFFFE7806028B71700408D6623A617
:106B7000D70A17F5FF1F130525BC1387C70A93878C
:106B8000870A1CC15CC5856689675CC958C114C584
:106B900018C9B7E70400B24003A3871E410102836E
:106BA0008145B307B5008387070089E717230000F5
:106BB000670023C48505C205C181E5B797A7010019
:106BC0009387073E1357C5003E97034707000111FF
:106BD00006CE2304E100135785003D8B3E97034703
:106BE000070023060100A304E100135745003D8B75
:106BF0003D893E97AA970347070083C707002800EF
:106C00002305E100A305F10097000000E78080F96B
:106C1000F24005618280411126C2E97797F4FF1F97
:106C2000938404C222C49387A7552E842381B40081
:106C30002E86AA8517F5FF1F1305C5C006C623902B
:106C4000F400A381040097800100E780E0DC930555
:106C50002400C205C18117F5FF1F130585BE9700EB
:106C60000000E780A084B38784002382A7002181ED
:106C7000A382A700930564002244B2402685924473
:106C8000C205C181410117230000670083B609C90D
:106C90009307800263E6B700170300006700E3F77D
:106CA000828017F5FF1F0345A5AA828097F7FF1F73
:106CB00083C7C7B889E717230000670083B38280C2
:106CC00097F7FF1F83C7A7BA99EF411106C6972010
:106CD0000000E780E0A9B240854717F7FF1F2308AF
:106CE000F7B84101828082806307054A6385054ABF
:106CF0005D71CAC04EDE86C6A2C4A6C252DC56DA98
:106D00005AD85ED662D466D26AD0B9472A89AE898B
:106D100063F9B706394697A5010093852516978034
:106D20000100E78000CD31ED8347E9001307100330
:106D30006394E702854717F7FF1F2301F7B017A5F4
:106D400001001305A51497F7FF1F239807AE9700BE
:106D50000000E78020E571A01307000317A50100DC
:106D60001305C515E395E7FE97F7FF1F238807ACCA
:106D700097F7FF1F239307AC17A501001305851292
:106D8000F9B797F7FF1F83C767AB63870722BD6A11
:106D9000B96B938CFA55014A17FBFF1F130B8B9BA2
:106DA000138CEB65938AFA6605A8B307490183C67D
:106DB000070097F7FF1F83D747A8B1E39307A00504
:106DC000639BF600854717F7FF1F2318F7A697F771
:106DD000FF1F2381D798050A93170A01C183E3E6B1
:106DE00037FDB640264496440649F259625AD25AB3
:106DF000425BB25B225C925C025D61618280054D08
:106E0000639BA7039307500A639EF600894717F711
:106E1000FF1F2314F7A2930750FA17F7FF1FA30BC6
:106E2000F79255BF9307A005E387F6FA97F7FF1F80
:106E3000239507A04DB7138717004207DA974183C0
:106E40002380D70017F6FF1F2319E69E8D47E3F432
:106E5000E7F817F4FF1F0344149097F7FF1F83C749
:106E6000878F22045D8C9307F4FFC207C1839306CA
:106E7000F00DE3EDF6FA93076400C207C183E31C4B
:106E8000F7F493052400C205C18117F5FF1F130510
:106E9000858C97F0FFFFE780606133078B008347A5
:106EA000570003474700A207D98F17F7FF1F231684
:106EB00007986318F50E8144630CA40197F4FF1F33
:106EC00083C48489A20497F7FF1F83C7F788DD8CEA
:106ED000170500001305E5DB97F0FFFFE780A00131
:106EE00063878407636D9C029387EB556382F40488
:106EF00097F7FF1F83C7478605476389E70681CB5E
:106F00001387A7051377F70F8D4663F2E60813077B
:106F1000F0072300E100A300F10089459DA06382F2
:106F20009405E39754FD97F0FFFFE780C02B11A86D
:106F3000A28517F5FF1F1305258297F0FFFFE78055
:106F40002012014597F0FFFFE780E0FA69B5A285BE
:106F500017F5FF1F1305458097F0FFFFE7804019E5
:106F6000CDB797F0FFFFE780C021E1BF930710F88E
:106F7000130511002300F10097F0FFFFE780602D5B
:106F8000FD450A8597000000E78020C95DBFA28506
:106F900017E5FF1F1305457C97F0FFFFE78040CC06
:106FA0004DB79307F00789450A852310F100970034
:106FB0000000E78080C605B5BD4763F83717414636
:106FC00097A501009385C5F14A8597800100E78068
:106FD00040A2631C051417A501001305A5F1970035
:106FE0000000E78020BC17E5FF1F0355857497005C
:106FF0000000E780E0BC97E7FF1F83C7276317A562
:1070000001001305A5E689E717A50100130585E62C
:1070100097000000E78000B917A50100130505EFF0
:1070200097000000E78000B817C5FF1F035585389B
:1070300097000000E780C0B817A50100130545EDD3
:1070400097000000E78000B617C5FF1F0355E5381D
:1070500097000000E780C0B617A501001305C5EB37
:1070600097000000E78000B417D5FF1F03552504E3
:1070700097000000E780C0B417A50100130545EA9A
:1070800097000000E78000B217D5FF1F0355E50108
:1070900097000000E780C0B217A501001305C5E8FE
:1070A00097000000E78000B017D5FF1F03550500CB
:1070B00097000000E780C0B017A50100130505E7A1
:1070C00097000000E78000AE17C5FF1F0355451F5E
:1070D00097000000E780C0AE17A50100130585E505
:1070E00097000000E78000AC97D7FF1F83C7870297
:1070F000A20717D5FF1F0345F5015D8D970000001E
:10710000E78000AC97D7FF1F83C7E700A20717D51A
:10711000FF1F034555005D8D97000000E78040AAE2
:10712000179501001305C5561DB1C14763FE37050C
:10713000414697A50100938525E04A859780010087
:10714000E780208B31E18347090113071003639C1B
:10715000E700854717E7FF1F230CF75E17A501001F
:107160001305C5DEEDB61307000317A501001305CF
:10717000E5E0E39EE7BC97E7FF1F238B075C17A5BD
:107180000100130525DEE1B6CE854A8597C0FFFFD5
:10719000E7800005B9B18280411126C2AE848D45D9
:1071A00022C406C62A8497C0FFFFE78060CEB717C7
:1071B000004099C803A5C70C418D23A6A70CB24077
:1071C000224492444101828003A5870C418D23A46F
:1071D000A70CF5B78347050003471500A207D98F11
:1071E000C2076177C18713072720639AE7008345A9
:1071F00025003705040017030000670023FA82808A
:1072000017E6FF1F130606678147B2861303F00FC8
:10721000A9483308F6000348080013F7F70F63077F
:10722000A80C630668008507E39517FF2947B38715
:10723000E6002380A70097E7FF1F938767645DA898
:10724000411113D765001347170006C693F63500A2
:10725000058B954791CA054699476387C60009463D
:107260009D476383C600A14713F645003336C0002F
:1072700093F68503050685C2A145638BB604E145F7
:10728000638AB604930580026388B604930580037D
:107290006393B600914697F5FF1F2388F58497F511
:1072A000FF1F2383C58497F5FF1FA38FD582BE855B
:1072B00017A501001305C5D297800100E780208142
:1072C000B240854717F7FF1FA301F7824101828073
:1072D0008546D1B78946C1B78D4675BF17A5010050
:1072E000130585D2177301006700637E17E7FF1F40
:1072F00013070759BA972380B700E147E302F5F473
:1073000093077002E30CF5FC82802A872380050036
:10731000814717E5FF1F1305E5551308F00F2946B0
:10732000B306F50083C606006396E60297E6FF1FE4
:1073300093860655B69783C7070005452380F50059
:107340009947636EF7029D4763FDE700E147630DD0
:10735000F7008280638506018507E393C7FC01453A
:10736000C5B7238005008280B737004003C73700C8
:1073700083C7050093F70704D98F2380F500828027
:107380005D7152DC56DA5ED6716A97FBFF1F938BF4
:10739000EB868D6AA6C24EDE62D486C6A2C4CAC07F
:1073A0005AD866D26AD06ECEC1495E8C97E4FF1F70
:1073B0009384C44D130A0A20938A7ADC17F9FF1FBD
:1073C0000349C986B3872B0183C7070093F7F70FDB
:1073D000C9EFB787004003C76700058BE310077C40
:1073E00003C76700118BE30D077E83C75700918B9E
:1073F00099E36F10200317F7FF1F03474783854763
:107400006304F7006F10400197E7FF1FA38FE76C3D
:1074100097E7FF1F238C075297E7FF1F238A075E1A
:1074200097E7FF1F2388076A97E7FF1F2385076AEF
:1074300097E7FF1FA38C075097E7FF1FA38A075CFE
:1074400097E7FF1FA388076897E7FF1FA3850768D3
:1074500097E7FF1FA38C076897E7FF1FA389077CA7
:10746000B787004011476F0070779307190093F7B3
:10747000F70F3D476364F70617E7FF1F2308F77A06
:1074800097E7FF1F93878779CA9783C7070013077A
:10749000100293F7F703638EE71E6366F704054453
:1074A0006385871CE38C07620947638EE710130727
:1074B0000002E384E74EB7E700E03707400023A06F
:1074C000E71801000100629923000900FD1923A0BB
:1074D000E71093F9F90FE39309EEE5BD97E7FF1F76
:1074E0002386077471BF130730026388E70C63E8D3
:1074F000E71613074002638CE70A13070003E39CB7
:10750000E7FA97E7FF1F93876770CA9703C70700DB
:10751000A1471377F70FE31BF71483C7640097E6BF
:10752000FF1F238BF65A97E7FF1F83C7973691C734
:10753000FD5797E6FF1F2381F65A97E5FF1F83C586
:10754000F53497E7FF1FA389B75897E7FF1F83C755
:10755000E73313FB07089306000493F70706639FBE
:10756000D74C9307A009638DF51663EAB71293070A
:10757000F0056386F54A930750096384F52A0144B0
:1075800097E7FF1F83C757551547E392E736B7E7DD
:1075900000E03707400023A0E71801000100B7868C
:1075A000004023808602130680FC6F00500EFD57BA
:1075B00017E7FF1F2301F752FDBDFD5717E7FF1F18
:1075C000230AF750CDBD17A50100130565B59770C7
:1075D0000100E780A06797E7FF1F93872763CA979B
:1075E00003C40700014B97ECFF1F938CAC4213744C
:1075F000F40F17AD0100130D2DB363478B0429451C
:1076000097700100E7808051854717E7FF1FA301AE
:10761000F74017E7FF1F230E873E17E7FF1F2307DB
:10762000F74C37E700E0B70640002320D7180100E9
:107630000100378600408347A60293F7370F2305E2
:10764000F6022320D71085BDB3876C0183C50700E0
:107650006A85050B97700100E780604779BF854711
:1076600017E7FF1F2306F73AB9B517E7FF1F130700
:10767000E7594A970347070097E6FF1FA388F62CB0
:1076800097E6FF1F2385E62C17E7FF1F2300F74629
:107690001DB5854717E7FF1F230AF72A29BD930762
:1076A000400A6389F5349307200B6384F53693070A
:1076B000100AE396F5EC838724000144E3D207EC3B
:1076C00097E7FF1F83C7B71C93F63700638A061A34
:1076D0000546638AC62209466395C61A1D4755A208
:1076E00017E5FF1F0345A51AC94797ECFF1F83CC79
:1076F0001C1A97E5FF1F83C5A51917E4FF1F034454
:1077000034196315F510CD476392FC109307700888
:10771000639CF5021307300FB7170E006308E400EF
:107720001307900DB7B704006314E40817E7FF1FB1
:10773000232AF73ABE8517A501001305659F9770A8
:107740000100E780C03825BD93078008639DF500E0
:10775000B307804013F4F70FB7774600938787CDC0
:10776000B3D78702E1B793079008639AF500B30790
:10777000804013F4F70F91679387C766D5B79307D7
:10778000A008639BF500B307804013F4F70FB71709
:107790003D0093870790E9B79307B008639AF50017
:1077A000B307804013F4F70F9167938797D04DBFCD
:1077B00093F5F5078D47639BF500B307804013F4FD
:1077C000F70FB7975B00938707D859BF8947639B2B
:1077D000F500B307804013F4F70FB7770B009387DA
:1077E000071BBDBF8547639AF500B307804013F4BC
:1077F000F70FDD67938767E3A5B7D28785F9B307EE
:10780000804093F7F70FB3D7FA020DB79700000047
:10781000E780409FA285668597000000E780809EF4
:10782000B9BB9305610017E5FF1F0345450617E443
:10783000FF1F0344D40597000000E78040AD930587
:107840007100228597000000E78060AC3C0017E7DC
:10785000FF1F2323F73A834761002304F100834786
:107860007100A304F100894717E7FF1F2306F726DD
:107870008357810017E7FF1F231AF700094409B354
:10788000154793F64700B336D00093F78703850674
:1078900085C32146638BC7066146638AC706130604
:1078A00080026388C706130680036393C70091476D
:1078B00017E6FF1F230AD62297E6FF1FA386F622AC
:1078C00097E7FF1F2383E72217E7FF1F034747FCC4
:1078D0009376070497E7FF1F83C797FB8DEE137717
:1078E000770C93067008630CD7021377F7078D4661
:1078F0006312D70CB307F040B7955B0093F7F70F0F
:10790000938505D849A81947ADBF854755B789471D
:1079100045B78D4771BF930670086311D7021307EF
:10792000300FB7150E006389E7021307900DB7B546
:1079300004006383E7021307700845BF9306800CB9
:107940006311D702B307F040B775460013F7F70F7E
:10795000938785CDB3D5E70297E7FF1F23A4B71818
:10796000D9BB9306900C631CD700B307F04093F586
:10797000F70F91679387C766B3D5B702F1BF930638
:10798000A00C631DD700B307F040B7153D0093F777
:10799000F70F93850590B3D5F5027DBF9306B00C24
:1079A000E315D7F4B307F04093F5F70F916793878A
:1079B00097D0D9B78946631BD700B307F040B77596
:1079C0000B0093F7F70F9385051BF1B78546631AF4
:1079D000D700B307F040DD6593F7F70F938565E3B4
:1079E0005DBFD28535FBB305F04093F5F50FB3D5F8
:1079F000BA029DB783C72400C18B99C7854717E793
:107A0000FF1F230EF70CA5BE97E7FF1F2389070C66
:107A1000BDB6854717E7FF1FA309F70C8DB63C00DD
:107A200017E7FF1F232AF71C0947930700032314B6
:107A3000F10097E6FF1F2381E60A2DBD63940756E8
:107A4000A94763E5B742179701001307A7568A05B0
:107A5000BA959C41BA97828717E4FF1F034434E329
:107A6000894C6306940D63E68C0685476303F4082E
:107A70009307F00F17E7FF1F0347070663F6E700BA
:107A800017E7FF1F230AF70497ECFF1F83CCCC04F2
:107A90009307000413F4FC0F63F49701130400042C
:107AA00097E7FF1F9387471503AD070022862685BA
:107AB000EA85B38C8C40229D97700100E780C0F569
:107AC00097E7FF1F238A970197E7FF1F23A6A713B6
:107AD00045BC8D47630CF40A9947E31BF4F897976C
:107AE00001009387A75317E7FF1F2327F710A94724
:107AF00051B717E7FF1F0347871397E7FF1F9387C8
:107B0000A7FF4946979501009385455A630687006C
:107B100097950100938585553E8597700100E78014
:107B2000A0EF17E7FF1F2329A70CC947A1B797E6C6
:107B3000FF1F83C6C60F054797E7FF1F9387C7FB45
:107B40006394E6023E8513067002979501009385C3
:107B5000655397700100E78020EC17E7FF1F232D86
:107B6000A7089307700239B73E851306300497952E
:107B700001009385654B97700100E780E0E917E706
:107B8000FF1F232BA70693073004EDB597E5FF1FD2
:107B900083C5E5CF179501001305C55A97700100FD
:107BA000E780E0F2054D97EDFF1F83CD4D0897E587
:107BB000FF1F83C5C5CD179501001305A558639810
:107BC000AD0B97700100E78080F097E7FF1F83C738
:107BD00007CCB5CBE36EF4E81794010013044451CD
:107BE000638CB70117940100130404516386970155
:107BF000179401001304C451228597700100E78097
:107C000020061375F50F93071500860717E7FF1F6A
:107C10002304F7EE8D4717E7FF1FA30FF7EC97E755
:107C2000FF1F938767ED0147BE861376F70F89071D
:107C30006365A60297E7FF1F23A0D7FC97E7FF1F06
:107C400083C787EB05BD979701009387674317E7C5
:107C5000FF1F2323F7FA914731BD3306E4000346A3
:107C60000600A380070005072380C7007DBF97702B
:107C70000100E780C0E597E7FF1F83C747C1E1D751
:107C8000E368F4DE1794010013048443638CA701B6
:107C9000179401001304444363869701179401006D
:107CA00013040444228597700100E78060FB13757C
:107CB000F50F93071500860717E7FF1F230EF7E25E
:107CC0008D4717E7FF1FA309F7E297E7FF1F938789
:107CD000A7E20147BE861376F70F8907E37CA6F477
:107CE0003306E40003460600A3800700050723804F
:107CF000C700D5B797E5FF1F83C565B91795010084
:107D00001305054597700100E78060DC97E7FF1FCA
:107D100083C757DE93E7470017E7FF1FA30CF7DC85
:107D200083C7240017E7FF1FA304F7DC89B8179562
:107D300001001305254397700100E78020F197E7C4
:107D4000FF1F9387E7DA83C7070017E7FF1F230F9B
:107D5000F7B217E4FF1F034424D8333480000DB07A
:107D6000179501001305454197700100E78000EE6B
:107D700097E7FF1F83C717D893E7070117E7FF1F90
:107D8000A30AF7D683C7240017E7FF1F2302F7D6FD
:107D90006FF0EFFE179501001305453F9770010046
:107DA000E780C0EA03C704007D8B51EFB78700402E
:107DB00003C767021377C70B136727002383E70204
:107DC00003C7A7021377C70B136727002385E702B2
:107DD00003C7E7021377C70B136727002387E70260
:107DE00003C727031377C70B136727002389E7020D
:107DF000854717E7FF1F230BF7B417E7FF1F23097A
:107E0000F7C017E7FF1F2307F7CC17E7FF1F23046F
:107E1000F7CC97E7FF1FA38B07B297E7FF1FA38954
:107E200007BE97E7FF1FA38707CA97E7FF1FA38433
:107E300007CA97E7FF1FA38B07CA97E7FF1FA3880F
:107E400007DE6FF0CFF389476312F70297E7FF1F52
:107E500083C707A49146638CD70863E0F604638E5A
:107E6000E70C6369F70A05476380E70EFD5717E7DC
:107E7000FF1FA303F7C637074000B7E700E023A0C2
:107E8000E71801000100B78600401306F0FC2381CB
:107E9000C60223A0E7106FF00FE2130720086382E9
:107EA000E7086362F70213071008E391E7FC3787DE
:107EB00000408347670293F7C70B93E7270023032C
:107EC000F7026FF0CFEB130730086389E70213075F
:107ED0004008E39DE7F8378700408347270393F77F
:107EE000C70B93E727002309F7026FF04FE93787A5
:107EF00000408347270393F73707F5B737870040DC
:107F00008347E70293F7C70B93E727002307F7029E
:107F10006FF0EFE6378700408347E70293F73707B4
:107F2000F5B7378700408347A70293F7C70B93E75E
:107F300027002305F7026FF08FE43787004083475F
:107F4000A70293F73707F5B73787004083476702E3
:107F500093F73707ADB717950100130525249770E0
:107F60000100E780A0CE97E7FF1F23810792D5B3DA
:107F7000179501001305852397700100E78000CD58
:107F800097E7FF1F2394079097E7FF1F9387C7B4D6
:107F900003C40700894763F3870009441374F40F8F
:107FA0006FF00FDE13070002E392E7EC631B0B0A8E
:107FB000638FF500930720026383F508179501008E
:107FC0001305452297700100E78060B045B517950D
:107FD00001001305651E97700100E78020C701446A
:107FE000179D0100130D8D1EA14CB387840083C51E
:107FF00007006A85050497700100E78040ADE3162D
:1080000094FF178501001305A56E97700100E780A6
:10801000E0C317E4FF1F0344A48701E897E7FF1FAD
:1080200023880784014B6FF0AFD58947E310F4E450
:10803000854717E7FF1F230DF7826FF04FD417E630
:10804000FF1F0346D68497E5FF1F83C54584179518
:1080500001001305251897700100E78040A76FF015
:108060000FD26380F50693071002E399F5F497E5C4
:10807000FF1F83C5E581179501001305A5179770AC
:108080000100E780C0A497E7FF1F23A797B697E7F3
:10809000FF1F938727A5944383D7470017E7FF1F48
:1080A0000347A7A417D6FF1F2322D67E1D4497D6C9
:1080B000FF1F239FF67C97D7FF1F238CE77C6FF071
:1080C0002FCC97D5FF1F83C5A57C179501001305FD
:1080D000E51397700100E780809F97D7FF1F2389E2
:1080E000077897D7FF1F2393077A6FF02FF925475B
:1080F000638FE7C89946378700406394D70223000F
:108100008702B7E700E0B706400023A0D7180100B8
:108110000100130600FC2301C70223A0D7106FF053
:108120008FB99306100A639FD70023008702B7E731
:1081300000E0B706400023A0D71801000100130695
:1081400080FCD1BF9306A009E381D7FE9306400AC5
:10815000E38DD7FC93062002639DD700B7E700E0CC
:10816000B706400023A0D7180100010023008702B2
:10817000F9B78546E384D7FE93070008E300FBFECA
:10818000B7E700E0B706400023A0D71801000100C0
:10819000130620FC23008702BDBF17E7FF1F03471C
:1081A000B7936302F71E63E7E70295476300F71092
:1081B0009947630AF704B786004023800602B7E7B1
:1081C00000E03707400023A0E71801000100130674
:1081D000A0FC75B99307F005630AF70093075009EF
:1081E0006306F70093071002E317F7FCB7E700E018
:1081F0003707400023A0E71801000100B7860040C0
:10820000130620FC69B117EBFF1F034BEB8C9307A0
:1082100000045A8D63F46701130D000497E7FF1FF4
:108220009387879D83AC07001374FD0F2286E68534
:10823000268597600100E780207EB3078B40669417
:1082400017E7FF1F230AF78897E7FF1F23A6879AE0
:10825000B7870040630C0B022380A703B7E600E05A
:108260003706400023A0C6180100010003C72702FB
:10827000134707042381E70203C727021377C70FB9
:108280002381E70223A0C6106FF0EFA2238007022C
:1082900037E700E0B70640002320D71801000100AF
:1082A000130620FC2381C7026FF0AFB93787004067
:1082B0008347370097E6FF1F83C6968393F7070827
:1082C000D58FA301F700B7064000B7E700E023A071
:1082D000D718010001001306A0FC35BD97E7FF1F6A
:1082E0009387C792CA9783C7070093F7F70FC1CF49
:1082F00097E7FF1F83C7A793D9E717D7FF1F034748
:10830000B77D930700026310F70883AD040017DD03
:10831000FF1F034DED5797DCFF1F83CC7C5717DB06
:10832000FF1F034B0B57E6876A87DA866E8697D561
:10833000FF1F83C5E553179501001305A5EE976050
:108340000100E780C07897D7FF1F23ADB77997D793
:10835000FF1F238BA77997D7FF1FA387977997D7FD
:10836000FF1F2384677997D7FF1FA3828750B7E742
:1083700000E03707400023A0E71801000100B7869E
:1083800000406FF04FA2B7E700E03707400023A09E
:10839000E71801000100B786004015BD97E6FF1FF2
:1083A00083C6E6880547639CE60429472381E702E4
:1083B00009472383E7022385E70297D7FF1FA38797
:1083C000077297E7FF1FA3840786B7870040A38142
:1083D000070017D7FF1FA30D077005472383E7008A
:1083E000B640264496440649F259625AD25A425B34
:1083F000B25B225C925C025DF24D61618280294732
:108400002381E70209472383E7022385E7022387C5
:10841000E7022389E70255B717D7FF1FA309F744DF
:108420006FE01FFF854717D7FF1F2301F75217D7AC
:10843000FF1F230FF75C17D7FF1F230DF76817D710
:10844000FF1F230AF7686FE0BFFE854717D7FF1F9E
:10845000230EF74E17D7FF1F230CF75A17D7FF1F0E
:10846000230AF76617D7FF1F2307F76617D7FF1FE3
:10847000A30E074C17D7FF1FA30C075817D7FF1FD2
:10848000A30A076497D7FF1FA3870764828041115F
:1084900006C697000000E78080FBB7870040238076
:1084A0000700130740FC2386E7001307C004A386D8
:1084B000E70017D7FF1F1307673D2398E70017D77B
:1084C000FF1F1307A740239AE70017D7FF1F1307C3
:1084D000274C239CE70017D7FF1F1307A757239E9E
:1084E000E70029472381E70209472383E702238521
:1084F000E7022387E7022389E702A38107009306A7
:1085000000F8A380D700930690022380D700FD5681
:108510002383D7002381E7009306000537E700E0B7
:10852000230BD740B70640002320D71003C71700FE
:1085300013671700A380E700B24097D7FF1F239966
:10854000075A41018280411106C697000000E7806A
:1085500000F0B787004023800700130700FC238644
:10856000E7003147A386E70017D7FF1F130707323D
:108570002398E70017D7FF1F13074735239AE70013
:1085800017D7FF1F1307C740239CE7002947238104
:10859000E70209472383E7022385E702A381070057
:1085A000930600F8A380D700930690022380D7009B
:1085B000FD562383D7002381E7009306000537E7A4
:1085C00000E0230BD740B70640002320D71003C795
:1085D000170013671700A380E700B24097D7FF1F6B
:1085E0002398075041018280F1679387072017D7AE
:1085F000FF1F2329F74E854717D7FF1F2316F74E76
:10860000A14717D7FF1F2302F74E97D7FF1FA38E4F
:10861000074C97D7FF1F238B074C97D7FF1F238942
:10862000072497D7FF1FA3840724814717D5FF1F6F
:1086300013054524FD5517D6FF1F13066624294749
:10864000B306F5002380B600B306F60023800600CB
:108650008507E397E7FE97D7FF1FA380074897D7C3
:10866000FF1FA38E074697D7FF1F2389074697D77B
:10867000FF1F2384074697D7FF1F2383074697D7FB
:10868000FF1FA38D074497D7FF1F238A0744814705
:1086900017D6FF1F130686564147B306F600238000
:1086A00006008507E39BE7FE828017D7FF1F03477D
:1086B000075885476316F700170300006700E3E8D3
:1086C000170300006700E3DC411122C406C617D778
:1086D000FF1F0347C75585472E8613F4F50FAA855C
:1086E0006317F70417D5FF1F1305852E9760010048
:1086F000E780803297D7FF1F238C0730B787004071
:1087000023848702B7E600E03706400023A0C6189E
:108710000100010003C7A7021377C70F2385E702F3
:10872000B240224423A0C61001454101828017D5E2
:10873000FF1F1305A51D97600100E780E02D97D767
:10874000FF1F23850720B787004023828702B7E6F3
:1087500000E03706400023A0C6180100010003C74F
:1087600067021377C70F2383E7025DBF411106C677
:1087700097000000E78080E7B24041011703000046
:108780006700E3F2411106C697F0FFFFE78080BF64
:1087900097D7FF1F83C7971BA1CB97D5FF1F83C513
:1087A000051B89C917D5FF1F1305851A97E0FFFF21
:1087B000E780C05397D7FF1FA38A071897D7FF1FDB
:1087C0002386073237E700E0B70640002320D7189A
:1087D00001000100378600408347660293F7370F98
:1087E0002303F6022320D710B2404101828041C901
:1087F000D9C597D7FF1F83C7A72FD1C3011122CC9B
:108800004AC84EC656C25AC006CE26CA52C42E897F
:10881000AA890144930A0004371B030063772403E9
:10882000B3078940C207C183BE8463F4FA0093048E
:108830000004C204C180130A1BD497D7FF1F83C74B
:10884000E7109DE37D1A631C0A00F2406244D244A3
:108850004249B249224A924A024B0561828097F00E
:10886000FFFFE78020B2D1BF338589002694A6851B
:10887000420497000000E78060E5418045B78280B0
:1088800097D7FF1F9387473E18429C4383D64500E6
:108890000345070083C5C700035646006396A5003D
:1088A00083D5E700638DD502011106CE2386A7008C
:1088B0002397D700B705CF00DC4B9385757D05075F
:1088C0007D162EC2230001003AC42316C1002317CF
:1088D000D10099C30A858297F24005618280828027
:1088E000DC4DDC4B81CFB7E70400904503A387053F
:1088F000914517D5FF1F03456537028382806D714F
:108900003C083EC6B707E500232291103EC8AA8462
:108910003C083285232611103ECA232481102320CF
:1089200021112E8997300000E780C0642A84979532
:1089300001009385A592177501001305A57897602E
:108940000100E780C018A28517950100130585A1D5
:1089500097600100E780A017294597600100E78034
:10896000E01BB705CB009385757D6800971000006C
:10897000E780406AA285680097300000E780E051F8
:10898000014781467000CA85268597200000E78050
:10899000C08D05CD2A84979501009385258C177588
:1089A00001001305257297600100E7804012A2853F
:1089B000179501001305C59B97600100E780201102
:1089C000294597600100E78060158320C1100324CA
:1089D000811083244110032901105161828097D7AF
:1089E000FF1F9387672818429C43797122D406D6CB
:1089F0000348070083C807012A8483D6450003552E
:108A000046006396080183D82701638DD802238826
:108A1000070105072399D7003708CC00DC4B130862
:108A2000787D3ACC1307F5FF42CA23080100231EC4
:108A3000E100231FD10099C7080832C62EC48297CF
:108A40003246A245228597000000E78080EBB250B5
:108A50002254456182806D713C083EC0B707E50035
:108A60003EC23C083EC42326111023248110232239
:108A70009110231701002318010023190100231A64
:108A80000100231B010097B7FF1F83D7679799E366
:108A9000C167FD172316F10097B7FF1F83D76796AD
:108AA00091EB97D7FF1F9387271C9C439C43DC4780
:108AB00083D7070017B4FF1F13048494584C23175F
:108AC000F10083574400484B2318F10031E19785AA
:108AD00001009385A57F177501001305A55E9760BA
:108AE0000100E780C0FE178501001305657F9760D0
:108AF0000100E780C0FD294597600100E780000282
:108B00008320C1100324811083244110516182808D
:108B100097B7FF1F83C7378F89EBB7E70400BC57B0
:108B200082975C4C23AA0700E1BFFD1797B6FF1F91
:108B3000A38BF68C03560701834704014C470A8533
:108B4000230BF10097300000E780403297D7FF1FDA
:108B5000938787119C430147814688430A866C00AE
:108B600097100000E7806070AA8429C197850100F2
:108B70009385C575177501001305C55497600100ED
:108B8000E780E0F4A6851785010013052576976038
:108B90000100E780C0F3294597600100E78000F8F5
:108BA000584CB7E70400BC57484B9DBF97B7FF1F11
:108BB00083C77785F5D7B7E70400BC4F10448545D8
:108BC00017D5FF1F0345850A82971DBF5C4EDC4BFE
:108BD000B9CFB1CD411122C4177501001305854EDF
:108BE0002E84978501009385A56C06C697600100C9
:108BF000E780E0EDA285178501001305E571976018
:108C00000100E780C0EC294597600100E78000F192
:108C1000B7E704002244B24003A3870517D5FF1F1E
:108C20000345C50413064006914541010283828035
:108C3000411122C417A4FF1F1304447A1C4C06C61A
:108C400089C7DC4399C34C488297584CB7E7040066
:108C5000BC57484B82975C4CB240224423AA070081
:108C60004101828017A7FF1F130747798347070039
:108C70009306F00B850793F7F70F63E9F60097A6C5
:108C8000FF1F238DF676034507008280930700F8C7
:108C9000FDB7835745006386071001114AC817A91D
:108CA000FF1F1309E97552C4032AC90106CE22CC5D
:108CB00003274A0126CA4EC656C2F15735E31307A9
:108CC000D00DFD57636EC704B7E9040083A70907F9
:108CD0002A841305860042054181B284AE8A8297B8
:108CE000232AAA000325C9015C49A9E79785010049
:108CF0009385055A177501001305C53C976001005F
:108D0000E780E0DC178501001305456997600100E5
:108D1000E780E0DB294597600100E78020E0DD5730
:108D2000F2406244D2444249B249224A924A3E85C4
:108D30000561828093874400B705CF002319F500B1
:108D40009385757D310597100000E780A02C0325E1
:108D5000C90183456400310597300000E780E013C6
:108D60000325C9012686D685310597300000E780A6
:108D7000E00F7146A2854A8597600100E780C0C96F
:108D8000504419CA83A78905854517D5FF1F034598
:108D9000E5ED8297814769B797000000E780E0CB57
:108DA000D5BFFD573E858280411126C297A4FF1F83
:108DB00093840465D84C22C437E404003C54484BE7
:108DC00006C68297DC4C0323C4052244B240924479
:108DD00023AA070017D5FF1F034545E98545410133
:108DE0000283411126C297D4FF1F9384E4E79C407D
:108DF00006C622C44AC0D5C3DC43C5C35CC1230038
:108E0000B5002A84978501009385C5431775010035
:108E10001305452B97600100E78060CB29459760DB
:108E20000100E780A0CF9C4023A4070023A20700F5
:108E300097A7FF1F9387875ADC4FDC4B91C72955B3
:108E400097000000E78000DF97A7FF1F9387475B2D
:108E5000DC4FDC4B89C797000000E78020F537E93D
:108E600004008327C905894517D5FF1F034505E081
:108E700082978327C905914517D5FF1F034505DF55
:108E800082979C4003A34701630903002285224483
:108E9000B2409244024941010283B24022449244CA
:108EA0000249410182800111328506CE22CC26CAB8
:108EB0002E8497300000E780E00BAA84978501009C
:108EC0009385853B177501001305C51F9760010049
:108ED000E780E0BF03078400035664008355440025
:108EE000A686178501001305254597600100E780D8
:108EF00000BE294597600100E78040C297A7FF1F89
:108F000083C7274E639D9700014597000000E780C7
:108F100060D281450A8597000000E780C0ECF240EE
:108F20006244D244056182806D712324811023261E
:108F300011102322911093F745002E8463870714A4
:108F40003C083EC0B707E5003EC23C083EC42317BC
:108F500001002318010023190100231A0100231B1B
:108F6000010097A7FF1F83D7674799E3C167FD17E4
:108F70002316F10097A7FF1F83D7674691EB97D77A
:108F8000FF1F938767CE9C439C43DC4783D7070032
:108F900017A7FF1F130787442317F100544F835768
:108FA00047002318F100DC4AA1E79785010093856B
:108FB000E530177501001305E51097600100E780A3
:108FC00000B1178501001305A53197600100E78006
:108FD00000B0294597600100E78040B41345440084
:108FE0008320C110032481108324411051618280A9
:108FF00097A7FF1F83C7F73E2555D9C3FD1717A6AF
:10900000FF1FA300F63E03D6060183470701CC46A7
:109010000A85230BF10097300000E78020E597D701
:10902000FF1F938767C49C4317A7FF1F1307073BC6
:10903000978601009386C62D88430A866C00971098
:109040000000E7808022AA8451D99785010093858A
:10905000E526177501001305E50697600100E78016
:1090600000A7A68517850100130545289760010014
:10907000E780E0A5294597600100E78020AA2685C2
:1090800097000000E78000BB91BF93F725009DC7C4
:10909000B7E70400BC47414681452808829725551B
:1090A00097000000E78000B928089305F00F9700AB
:1090B0000000E78040D3134524001DB793F7150047
:1090C000014599DF97000000E780209913451400BF
:1090D00001BF5C4D411106C688C317D7FF1F23256A
:1090E000F7B8B7E7040083A70708170500001305C2
:1090F000E5E38297B24097D7FF1F2389A7B60145C2
:109100004101828001113335A000A307A100B7E718
:10911000040083A7471706CE1306F1008545130503
:1091200050308297F240056182808280411122C4D2
:1091300006C617D4FF1F0344E4B431E497B7FF1FFA
:1091400083C7970EB9E397C7FF1F83C7274E99E7D9
:1091500017B4FF1F0344440D1344140022859700E5
:109160000000E78060FA178501001305252E09E449
:10917000178501001305852E2244B2404101176373
:1091800001006700C3940144D1BF0544C1BF797198
:1091900022D4A30F010037E404008327841726D2CA
:1091A0004AD006D6AA842E89130550309305F101C2
:1091B00032C6829732468347F10193150601C18179
:1091C00085CB01452EC697000000E780E0F383279A
:1091D0004417B2454A8626858297054597000000C8
:1091E000E78080F2B2502254925402594561828045
:1091F000832744174A8626858297EDB741119397B6
:10920000050122C406C626C2C1872E8463D4070284
:10921000B7E40400FC5417A5FF1F0345652182979E
:1092200019C1BC5482972165218DB24022449244D9
:109230004101828093F715008DC7B7E7040083A72B
:10924000471A17A6FF1F1306A61D97D5FF1F938564
:10925000A5A217A5FF1F0345A51D8297134514005E
:10926000E9B793F7250099CFB7E70400BC4F130681
:109270000064894517A5FF1F0345851B8297134589
:10928000240065B793F7850085CF97D7FF1F83C765
:1092900027A085E7B7E7040003A8871A1307401F34
:1092A00097A7FF1F83C7C718814613064006994535
:1092B00017D5FF1F0355459D029813458400B5B788
:1092C00093F745000145B5D3B7E4040083A704181C
:1092D00017D5FF1F0355459B8297BC4C13060064AE
:1092E000914517A5FF1F0345A51482971345440018
:1092F0002DBF97D7FF1F83D727996398A70217D74A
:10930000FF1F2314B79817D7FF1F2311C79817D72C
:10931000FF1F231ED7962E86178501001305851A79
:10932000BE85175301006700837A17850100130576
:10933000E51A17630100670063910357450097D74B
:10934000FF1F83D76794631EF704C1674111F917A4
:1093500022C417D7FF1F2329F79237E4040097D7B9
:10936000FF1F23A5079297D7FF1FA38D079097D7BD
:10937000FF1F238F07907C4C06C6894517A5FF1F4A
:109380000345050B82977C4C914517A5FF1F0345AC
:10939000250A82972244B24041011703000067006A
:1093A00023D91785010013056513176301006700B2
:1093B000E3897D15954763E2A71C17870100130712
:1093C00067070A053A951C41011122CC06CEBA97CF
:1093D0002E848287178501001305C5109760010050
:1093E000E780C086A1A203C7250099476311F70251
:1093F0002E8597000000E78080F483456400178580
:1094000001001305250F97500100E780406C97B7C6
:10941000FF1F238B07E0178501001305650F7DBF34
:1094200003C7250095476319F702C16717D7FF1FC8
:1094300003578785F91703D5A5006309F702B7E736
:10944000040083A7C7178297178501001305450DF0
:1094500097500100E780807F854717B7FF1F2305DE
:10946000F7DC178501001305250E8DBF97D7FF1F69
:10947000239CA78083D7E50097D6FF1F2397F6800C
:1094800083D7050197D6FF1F2392F68083D7250146
:1094900097C6FF1F239DF67E97C7FF1FA384077EF5
:1094A000631BE502B7E70400BC4F0966130606908C
:1094B000A14517A5FF1F0345A5F782970356E400B2
:1094C0008355A400178501001305C50697500100B8
:1094D000E780E05F51B79307700F2316F100B7E7FD
:1094E000040083A7870D17A6FF1F034666F46C00D0
:1094F00082974DF9854717C7FF1FA305F7785DB71A
:109500001785010013050505D1BD83C525009147C9
:109510006392F50217850100130545059750010078
:10952000E780C07297000000E78080C0F24062448C
:109530000561828099476392F502228597000000B9
:10954000E780E0DF8345640017850100130585FA95
:1095500097500100E780A057D1BF9547639AF50067
:1095600083471400E1F31785010013056502BDB5BB
:109570001785010013054502E1BF82803757315F2F
:1095800097A7FF1F938707EC130777D598C39356C8
:10959000C500178701001307A7EFBA9683C5060019
:1095A00093568500BD8ABA9603C6060093564500B9
:1095B000BD8A3D89BA962A9783C6060003470700ED
:1095C000238407002383D700A383E7002382B70007
:1095D000A382C70097A7FF1F9387C7E72383B7001E
:1095E000A383C7002384D700A384E70082804111AE
:1095F00006C697000000E780A0F8B7E7040083A73D
:10960000871417A6FF1F1306E6E3D5450145829789
:10961000B2404D4697A5FF1F9385C5E313057030F3
:109620004101170300006700C3B661712324811A4A
:1096300037E40400832704082326111A2322911AF1
:109640002320211B232E311917050000130545BBCC
:10965000829717A9FF1F1309A9DD994785442300A5
:10966000A900231CF10097850100938565E193070C
:109670004006177501001305E5A4231CF108230813
:10968000910097C9FF1F9389C90A97500100E7808D
:10969000004483D5090017850100130565DD975047
:1096A0000100E780C042294597500100E78000474C
:1096B00003D5090097000000E78080EC832744175A
:1096C000100885451305503082978327441717A645
:1096D000FF1F130626D8CD451305703082978327C8
:1096E000441717A6FF1F1306E6D4B54513056030CF
:1096F00082978327441730088945130510318297D4
:109700008327441730098945130520318297832721
:1097100044159305000A0D45829783274415930548
:10972000000A11458297A30591002306910002CDFE
:1097300023080100230C010083278416300991457A
:10974000130570408297832784161306B100854560
:109750001305004082978327841670008545130502
:1097600010408297832784163008854513052040D2
:1097700082978327841610088545130550408297E9
:10978000832704157D558297832744137D5582973F
:109790007D5597A0FFFFE78040EF8327440C829719
:1097A00097A0FFFFE780A0CA8327841417A6FF1F96
:1097B000130646C9D5450145829789471306700FA0
:1097C000814528092306F1009790FFFFE780209448
:1097D0008D471306000881452808230CF10897904F
:1097E000FFFFE780C0929147230CF10097670100CB
:1097F0009387C77E984383C747003AC8230AF1007E
:1098000097D0FFFFE78080AF70008545054597A0A2
:10981000FFFFE780A0EE30099305700F094597A080
:10982000FFFFE780A0ED3008930500080D4597A0E5
:10983000FFFFE780A0EC10089545114597A0FFFFBA
:10984000E780C0EBC16717C7FF1F1307E743F9178E
:109850001CC32322070017A5FF1F130525BD97A0D2
:10986000FFFFE78080E88327C41D17C5FF1F13058E
:10987000254082973C48034509008545829783200F
:10988000C11A0324811A8324411A0329011A832946
:10989000C1195D618280C16717C8FF1F0358C83EA8
:1098A000F9176301F8083DCDB5CD011126CAB7E41B
:1098B000040083A7841222CC2E862315B10006CE85
:1098C0002A8401478146ED45428582972AC611EDDB
:1098D00017850100130505BD97500100E78000378B
:1098E000F2406244D24405618280FC440356A100E8
:1098F000A28582972C0017C5FF1F0355E53897A056
:10990000FFFFE78040EB69DD178501001305C5BA4D
:1099100097500100E780803383A7C412ED452800EB
:1099200082977DBF82800DC5854717A7FF1FA308BB
:10993000F7B097A7FF1F238507B0354697A5FF1FF0
:10994000938545AF130560301703000067006384FB
:1099500097A7FF1FA38507AEE9BF97C7FF1F83C760
:109960002733A9EFC16717C7FF1F0357E731F9175F
:109970006306F7044111854722C417C7FF1F230957
:10998000F73037E404007C4C06C6A14517A5FF1F3D
:10999000034505AA82970323841A2244B24097A75D
:1099A000FF1F83C7E7A817C5FF1F0355E52D130742
:1099B000401F8146314699454101028382806D7185
:1099C000232481102326111023229110328401CDEB
:1099D0008947630AF5028320C11003248110832480
:1099E000411051618280178501001305A5BBAE842B
:1099F00097500100E7808025A285268597C0FFFF4C
:109A0000E78000B2C9BFB7E70400FC47280082978F
:109A1000178501001305C5B997500100E7800023A1
:109A20008347810039C41307000B6380E702138763
:109A3000A7051377F70F8D4663EDE602A285280090
:109A400097C0FFFFE780C02179B78547E3F587F826
:109A5000834591001775010013050598B335B000D3
:109A600097A7FF1F2382B76497500100E780200665
:109A70009DB703479100A207D98F35671307D755C4
:109A80006385E7086368F7022D671307B755638797
:109A9000E70631671307C755638AE7042967130789
:109AA000A7556394E702A285280097C0FFFFE780CF
:109AB000205A15B739679306E7656381D70863E9CC
:109AC000F6001307E7556384E706A28528003DB733
:109AD0003D679306F755638AD7061307F766E39643
:109AE000E7FE97C0FFFFE7800070F5B50146A2854D
:109AF000280097C0FFFFE7804042F1BDA285280003
:109B000097C0FFFFE7800053F9B58947E3F587EC7D
:109B100097000000E780A0E49305E4FFC205C1813F
:109B20001305A1009790FFFFE780806B6DB5A285BC
:109B3000280097C0FFFFE780A05271BDA2852800D2
:109B400097C0FFFFE780C05A79B597C0FFFFE78055
:109B5000406351B5C16717C5FF1F0355E512F917DB
:109B60006307F500B7E7040003A3C71702838280E9
:109B7000854717C7FF1F2307F710014517F3FFFF9E
:109B80006700835817F3FFFF6700835A1783FFFFAF
:109B9000E70243532A8408452E89B28919C900C1B6
:109BA000971500009385A586610597300100E78031
:109BB000200581447D5A97100000E780E03963C793
:109BC000A404814497100000E780003A63C8A4040D
:109BD00097C7FF1F9387070C9C43DC47B307F940E7
:109BE00091872302F400638309048327C900B30724
:109BF000F4409587A302F4001C4C89C79C4799C385
:109C0000228582971783FFFF6700034F5C441397F9
:109C100014008504BA972390470171BF1C4813971D
:109C200014008504BA972390070069BF8327890031
:109C30000547B307F4409587A302F4008357040057
:109C4000638EE7028DC309476384E7040D47E395FC
:109C5000E7FA97870100938767E81CCC9787010094
:109C60009387C7E811A8978701009387A7AE1CCCFC
:109C700097870100938707AF5CC8BDBF9787010036
:109C80009387479A1CCC978701009387A79AEDB7D3
:109C900097870100938747E91CCC9787010093873A
:109CA000A7E9D9BF95E51783FFFFE70243430046C5
:109CB00018448347940075839D8B6317F7009710B2
:109CC0000000E78060B448C41783FFFF6700634368
:109CD00082801783FFFFE702E33E13893500C164EA
:109CE00042094111AA890144F11413590901054A95
:109CF0002EC697100000E7802026B2456348A400D6
:109D0000014541011783FFFF6700033F83A7090057
:109D100013171400BA9783D707006388B7006394BA
:109D2000970063742A010504E1B70545D9BF17837D
:109D3000FFFFE7024338AA892E89328BB6843A8A1C
:109D4000BE8A97A00000E780C0FE71C926859720D3
:109D50000000E780C00C8D4763E7A7007D5517839F
:109D6000FFFF6700C33883DB440097100000E780E3
:109D7000A0242A8497100000E780402593077400F0
:109D800031443305850263CDA70297100000E780B8
:109D9000A02297100000E78020222A84971000005C
:109DA000E780C0229307740031443305850263C302
:109DB000A70497100000E78020209307450029A8FA
:109DC00097100000E7808020330585021307F01705
:109DD0009307C017E35FA7FA2D55E3C277F9630431
:109DE0000B02D6865286A6854A8597200100E78019
:109DF000C0BDB5B797100000E780401D3305850250
:109E00009307C5FFD1BF832749001385C90083D5B8
:109E1000270097000000E78000EC61F581B76955E5
:109E20003DBF97C7FF1F2399A7E697C7FF1F9387DB
:109E300067E6904381470C463307F50042074183AC
:109E40006393B70082805446139847008507C296F3
:109E50002390E600D5B797C7FF1F9387A7E39C43DE
:109E600003C58700828017C5FF1F0355E5E2828086
:109E70001783FFFFE702A326C1671387D7FF630B92
:109E8000E502636AA700F1176300F5020145178335
:109E9000FFFF670003271387E7FF6302E502FD1753
:109EA0001D8D13351500E5B797500000E780602A37
:109EB0007D15C5BF97500000E780E0FED5BF9750E5
:109EC0000000E78000FDEDB71783FFFFE7022321C5
:109ED0004111AA8401442EC697100000E780C008F3
:109EE000B2456348A400014541011783FFFF6700A5
:109EF00043219C48131514003E9583570500E385C4
:109F0000B7FE0504C9BF03485500814693F7F60F15
:109F100063E5070181473E85828058459397560047
:109F2000BA9703D727006316B70003D70700E304E7
:109F3000C7FE8506E1BF8346450001479377F70FCB
:109F400063E4D700814711A81C4513165700050785
:109F5000B29703D60700E313B6FE3E8582801783CF
:109F6000FFFFE702231693170501C18797CAFF1F5A
:109F7000938A4AD2635BF00883A70A00C0479C47D4
:109F800003570400198D420541816368F5000144BF
:109F900022851783FFFF6700231612052A94CDBF81
:109FA000DC4713944900014A3E94834744006341CF
:109FB000FA02014A834754006349FA028509C2093B
:109FC00093D9090183A70A009847E3EBE9FCC1B7DD
:109FD0001C4413195A00A6853E994A859700000033
:109FE000E780C0EE05E1050AC9B75C4413195A00C1
:109FF000A6853E994A8597000000E78020ED19E18B
:10A00000050A4DBFE30C09FA61B7AA8481495DBF17
:10A010001783FFFFE702A30C1C452A8481E79307FF
:10A02000C5001CC51C44231204001CC09307F00F7C
:10A0300063EDB70093F5F50F228597200000E780C8
:10A04000C0E51783FFFF6700C30B93940501C16749
:10A05000C18063F9F500A685228597200000E7807E
:10A06000E0E8C5B7C18193F5F50F22859720000080
:10A07000E780A0E2A685228597200000E780E0E344
:10A08000C9B797C7FF1F9387E7C0884382801C45E5
:10A0900099C797C7FF1F23AFA7BE014582807D5593
:10A0A000828097C7FF1F9387E7BE98438347450089
:10A0B000484792073E9582801783FFFFE7022302FD
:10A0C000617100451C183EC6B70780013EC81C18C8
:10A0D0003ECA8357440002CE02D002CC231EF100B8
:10A0E000834784002A8902D22301F1023C083ED42E
:10A0F00002D697000000E78000FB83570500231677
:10A10000F10297500000E78000C82307A1025C40DD
:10A1100003556400F18313F717008347F1025205DA
:10A120005181F99BD98FA307F10297100100E780B5
:10A13000207939CDAA840355050097A00000E78057
:10A1400020C083D704002AD26800231CF10083D7E3
:10A150002400231DF1001C4803D647008C439720A0
:10A160000000E780A0D08347B400CA8617760100BC
:10A170001306C6448117A305F4006C00481097200D
:10A180000100E78080845D611783FFFF670063F74C
:10A190002155D5BF1C45B1CF03C5A700894613572C
:10A1A0006500630BD7028D46630ED70285466300B8
:10A1B000D702130740063305E50203C7B700418BFA
:10A1C00015CB83C7B700BD8B3355F540828013751F
:10A1D000F5031307803EC5B709671375F503130729
:10A1E0000771D1BF372709001375F5031307077CE3
:10A1F000D9B7014582801783FFFFE70243EE03A929
:10A200008500630C09048347B900AE8493F7070EF9
:10A2100085C303459900930520030D810505B3050A
:10A22000B5028844610597300100E78080AD35A014
:10A230002E8597000000E78020F62A8419CD97002C
:10A240000000E780605C8325C900B307B54063FA6E
:10A2500087002E94B305A440E9F51783FFFF67003C
:10A2600043EA85457DBF1783FFFFE70243E72A8462
:10A2700003D50500011132C636C43AC22EC002CA47
:10A2800002CC02CE97A00000E78080AB82452ACAAC
:10A2900022852ECC97000000E780E0E00357050000
:10A2A000231EE10097500000E780E0ADA246324651
:10A2B0009247230FA10036874C08B28622850146BB
:10A2C00097000000E780E0A605611783FFFF6700A5
:10A2D00043E31783FFFFE70283E061711C183EC66A
:10A2E000B70780013EC81C183ECA3C0800453ED452
:10A2F000AA8402CC02CE02D002D202D6970000007D
:10A30000E78060DA8357050035592316F10297502C
:10A310000000E78040A72307A10209C48357440037
:10A3200081EB21594A855D611783FFFF670063DD7B
:10A33000035564005205518197100100E780405891
:10A340002A8965D18347B40093F7070E99C713058F
:10A35000840197300100E780009D83574400231E4D
:10A36000F100834784002301F1025C40035509009A
:10A37000D98313F7070883471102231CA10093F721
:10A38000F707D98FA300F10283572900231DF1009D
:10A390005C40F18313F717008347F102F99BD98FD3
:10A3A000A307F10297A00000E78080992AD235D94F
:10A3B000834794006800139757008347B400FD8BD0
:10A3C000D98FA305F4001C4803D647008C4397207F
:10A3D0000000E780A0A9A687177701001307071ED2
:10A3E000740005464C10268597000000E7806094B5
:10A3F0002A890DD98347B400A685FD8BA305F400F7
:10A4000097000000E78060DF31BF1783FFFFE7029E
:10A4100003CD832485FE2A84411126859700000000
:10A42000E78080D7834734FF93F7070E8DCB2AC68A
:10A43000268597000000E78060C809CD834734FF78
:10A44000B245FD8BA309F4FE91C52285973001002A
:10A45000E780208B41011783FFFF670083CA7DD906
:10A460008327C4FF2685829775F5834734FF93F7CA
:10A47000070E91C7228597300100E780C08A032527
:10A4800084FE97000000E78000E5E9B71783FFFF2F
:10A49000E702E3C19C4141112A8903C707008947AC
:10A4A0002E84935667006380F6040D466388C604C5
:10A4B0009307F0076304F7022E8597200000E780DA
:10A4C00060ABAA848149C16B130C490097B7FF1F89
:10A4D0009387477C9C43984763E4E90441011783D1
:10A4E000FFFF670083C003D745008547E3F8E7FE19
:10A4F0002E8597200000E78040ADE1B703D74500E7
:10A50000E3FEE7FC2E8597200000E780A0A6AA8442
:10A51000228597200000E78000A8C204C98C5DB79F
:10A52000DC470355A900139A49003E9A9317050189
:10A53000C187635DF00083570A006397A70263E752
:10A5400074038327CA00034D5A002DA0A167216719
:10A55000A98F1307F7EFE374F7FE639709009700DD
:10A560000000E780209161FD85098DB783278A006F
:10A57000034D4A00835DA90003576900216A138BCC
:10A58000C7003AC6814A33CA4D01631E5D0197B7C1
:10A59000FF1F9387A7709C43E1DBA28662868145FB
:10A5A00026858297D1B7A1679387F7EF930C4BFF6E
:10A5B00063F24703B2455A8597F0FFFFE780A07129
:10A5C0000DC103278B00104709CE10436382C402DC
:10A5D0003107D5BFEE85668597000000E780008FC4
:10A5E00071F993861A0093FAF60F130B0B0271BFE1
:10A5F000835644005C43E3E9F6F622853AC6972089
:10A600000000E7802081A1679387D7042A8A035D31
:10A610004400324763E897008347D90093E707F87F
:10A62000A306F9001C4766852286E2858297C167EA
:10A630000844FD17337AFA00529508C02312A4018A
:10A6400025B797B7FF1F9387E7649843814715C3E2
:10A650001447814763FFD500939745004C47BE954B
:10A6600019C903C7550081476375E600DC45160626
:10A67000B2973E85828003C745008147E37BE6FEB3
:10A6800016069C45F5B71783FFFFE702A3A3AA8927
:10A690002E8A814497BAFF1F938ACA5F83A70A0054
:10A6A000984763E6E4001783FFFF6700E3A4DC47F5
:10A6B0001394440001493E9413BB140083474400A3
:10A6C000634BF900014913BB140083475400634FE7
:10A6D000F9008504E1B70844931759005287DA86D8
:10A6E0000146A2853E9582990509C9BF4844931742
:10A6F00059005287DA860546A2853E95829905095A
:10A70000E9B71783FFFFE702839D814517F5FFFF38
:10A710001305054897B7FF1F2390075897000000BF
:10A72000E780A0F61783FFFF6700A39D97B7FF1F81
:10A73000938747569C4395C31783FFFFE702239AED
:10A74000814517F5FFFF1305A54497000000E7803A
:10A75000C0F31783FFFF6700C39A82801783FFFF50
:10A76000E702439637E4040083278412411123153E
:10A77000E100AE893289368A3A8681460147ED4545
:10A78000AA8482972AC621C90356A100D285974080
:10A790000100E78060288327C413CE852685829731
:10A7A000058905C98327440D2314210101462C0086
:10A7B000268582972A8401C9B7E7040083A7C712B8
:10A7C000ED4528008297228541011783FFFF67002E
:10A7D000A3924944D5B76554FDB75C41FD175CC1F0
:10A7E00082801783FFFFE702838FB7E70400FC5FD7
:10A7F000829795473305F50281450D811783FFFF49
:10A80000670023901783FFFFE702638DB7E704001B
:10A81000FC5F829795473305F5020D811783FFFF93
:10A820006700238E1783FFFFE702638BB7E70400FF
:10A8300083A7870B0355050082971783FFFF6700E7
:10A84000438C1783FFFFE702838903550500328796
:10A85000AE861796FF1F035606C697B5FF1F938552
:10A86000254497000000E780A0EF1783FFFF6700F3
:10A8700043891783FFFFE7028386B7E7040083A7B6
:10A88000C71782971783FFFF6700A3871783FFFF10
:10A89000E702E384B7E7040083A7871397B5FF1F98
:10A8A00093850540829701451783FFFF6700638505
:10A8B0001783FFFFE702A382B7E7040083A7C71F40
:10A8C00081451795FF1F035505BB82971783FFFF2F
:10A8D000670023831783FFFFE7026380B7E7040065
:10A8E00083A7871397B5FF1F9385853C8297014502
:10A8F0001783FFFF6700E3801773FFFFE702237EE4
:10A90000B7E7040083A7C71F81451795FF1F0355AD
:10A9100085BC82971773FFFF6700A37E1773FFFF45
:10A92000E702E37B2E8597800000E78080B3978065
:10A930000000E78080F01773FFFF6700837C1773C8
:10A94000FFFFE702C37997800000E78080FA177362
:10A95000FFFF6700037B5C49E1175CC95CC5835757
:10A960002501A1072319F50083570501A107231825
:10A97000F5008280F1473305F50297B7FF1F9387F3
:10A9800027359C433E9582808D476315F60803D793
:10A990004600854763F0E7081773FFFFE70223745B
:10A9A000368536842E8997100000E780A05C29C97F
:10A9B0008357440093140501C18063E39704228503
:10A9C00097100000E780005BFD14231294009307AA
:10A9D000A0026300F5029307B0026307F502930734
:10A9E0009002631FF500228597000100E7806089CF
:10A9F00001A80146CA85228597A00000E78000B41F
:10AA00001773FFFF6700E36F228597100000E78050
:10AA10006007FDB7828097B6FF1F9386A62B9C42E6
:10AA2000014599CF9843D44217B6FF1F2324E62A45
:10AA30006396D70097B6FF1F23A0E62A1385C7FEAB
:10AA400082801773FFFFE702836997000000E780A9
:10AA5000A04B714433058502914597900000E78033
:10AA6000C0EC11E565551773FFFF6700836997B761
:10AA7000FF1F23ADA72497000000E780E0483305BF
:10AA80008502914597900000E78020EA61DD97B745
:10AA9000FF1F23AFA72297000000E780E04697B78B
:10AAA000FF1F239FA72097000000E780E04597B78E
:10AAB000FF1F2398A72097770100938767B517B7E3
:10AAC000FF1F2323F72097070000938707E917B795
:10AAD000FF1F2329F71E014579B71773FFFFE70210
:10AAE0000360AA8517B5FF1F1305851D9710000089
:10AAF000E780605F1773FFFF6700A3601773FFFFB6
:10AB0000E702E35D97000000E78060FD971000001A
:10AB1000E780E05E97B7FF1F9387C71B9C4391CFE9
:10AB20001387C7FE19CB83D5C7FF17B5FF1F1305C2
:10AB3000E51A97200100E780C01C1773FFFF67002C
:10AB4000435C1773FFFFE702835997000000E7801B
:10AB5000C0EC09CD834785002A8493F7070499EB5D
:10AB60000355E50097000000E78080F91773FFFFA9
:10AB7000670023598347C5009304450117B9FF1F98
:10AB80001309491585E3832709005CC997B7FF1F9F
:10AB900023A2971483274900F1FB97B7FF1F23AD2A
:10ABA0009712E9B7FD172306F500610597800000AD
:10ABB000E78060DA8307840063CB0704834784005F
:10ABC00093E707F82304F400B7E704009C5F82973B
:10ABD0004205A94741813375F5028347840093F705
:10ABE00007FCC98F2304F4008347D4003E951C4022
:10ABF0002318A40089CF984319CB8347C400504041
:10AC0000814585073305F502420541810297832777
:10AC100009005CC897B7FF1F23AE970A8327490036
:10AC200089E797B7FF1F23A9970A8347C4009DDFD1
:10AC30008355040117B5FF1F1305450A972001002E
:10AC4000E780200C25B71773FFFFE702434997B74A
:10AC5000FF1F9387E72D9C4701448583858B85E300
:10AC6000AE84B2853A8697100000E780204F2A8490
:10AC700019C597100000E7806045829408CC2285B2
:10AC80001773FFFF6700E3471773FFFFE702834374
:10AC900041112E8932C6AA8997000000E780C03191
:10ACA000324713060502CA86970500009385C5CC76
:10ACB00017B5FF1F1305C50097000000E780E0F8F7
:10ACC0002A8425C99304C50097000000E780E0416D
:10ACD0001946AA85268597100000E780201985452A
:10ACE000268597100000E7800015177501001305F1
:10ACF000E58F4E9583450500268597100000E78077
:10AD0000C0195C4831468145A1075CC85CC48357C3
:10AD10002401E1172319F40083570401E1172318D4
:10AD2000F4001C4C3E859770FFFFE780403EA30473
:10AD30002501228541011773FFFF6700E33B17736D
:10AD4000FFFFE702C3394111AA842EC632C497100F
:10AD50000000E780003A004DB24522468347840058
:10AD60000CC050C093F7F70393E707042304F400E3
:10AD700023180400268597100000E78020358347BC
:10AD80009400A9462317A40013D7370005073307FB
:10AD9000D7029D8B85072306F400A306E40083C732
:10ADA0000401D8488507230FF7FE17B7FF1F1307C5
:10ADB00067F25843232A04009307440129E317B795
:10ADC000FF1F232BF7F017B7FF1F2325F7F017B44A
:10ADD000FF1F1304A4F0228597200100E780A0E460
:10ADE0001C44858B5D8D19E58145228597200100E6
:10ADF000E78020F141011773FFFF670083301CC318
:10AE000017B7FF1F232AF7ECD9B71773FFFFE70225
:10AE1000032D97050000938565B701459700000055
:10AE2000E78000B001451773FFFF6700832D17739C
:10AE3000FFFFE702C32A97000000E78080B0177386
:10AE4000FFFF6700032C8347C500A5E31773FFFFCF
:10AE5000E702E3282A840355E50097000000E78015
:10AE600000C821C18347840093F7F7FB2304F40053
:10AE70001C4091C7DC4381C74C4001458297970035
:10AE80000000E78080B917B5FF1F130525E597205F
:10AE90000100E78040E90355E40097000000E780E7
:10AEA00020C61773FFFF6700C32582801773FFFF5B
:10AEB000E702E32297B7FF1F9387C7E197050000DA
:10AEC000938565C817B5FF1F130545E123A007004B
:10AED00023A2070097200100E78080D21773FFFFAD
:10AEE000670023221C4D91CFDC4381CF1773FFFFF6
:10AEF000E702E31E8345070082971773FFFF670091
:10AF00004320828097B7FF1F938787DF9C4303C549
:10AF10000700828097B7FF1F938787DE9C4303C596
:10AF20001700828097B7FF1F938787DD9C4303C577
:10AF30002700828097B7FF1F938787DC9C4303C558
:10AF40004700828097B7FF1F938787DB9C4303C529
:10AF50003700828097B7FF1F938787DA9C4303C52A
:10AF60005700828097B7FF1F938787D99C4303C5FB
:10AF70006700828097B7FF1F938787D89C4303C5DC
:10AF80007700828097B7FF1F938787D79C4303C5BD
:10AF90008700828097B7FF1F938787D69C4303C59E
:10AFA0009700828097B7FF1F938787D59C4303C57F
:10AFB000A700828097B7FF1F938787D49C4303C560
:10AFC000B70011E11D45828097B7FF1F938747D3D4
:10AFD0009C4303C5C700828097B7FF1F938747D262
:10AFE0009C4303C5D700828097B7FF1F938747D143
:10AFF0009C4303C5E700828097B7FF1F938747D024
:10B000009C4303D50701828097B7FF1F938747CFE3
:10B010009C4303C52701828097B7FF1F938747CEC4
:10B020009C4303D54701828097B7FF1F938747CD85
:10B030009C4303D56701828097B7FF1F938747CC56
:10B040009C4303D58701828097B7FF1F938747CB27
:10B050009C4303C5A701828097B7FF1F938747CA08
:10B060009C4303C5B701828097B7FF1F938747C9E9
:10B070009C4303C5C701828097B7FF1F938747C8CA
:10B080009C4303C5D701828097B7FF1F938747C7AB
:10B090009C438857828097B7FF1F938767C69C435E
:10B0A00003D5C702828097B7FF1F938767C59C436C
:10B0B00003D5E70219E11305800C828097B7FF1FC3
:10B0C000938707C49C4303C50703828097B7FF1F7C
:10B0D000938707C39C43C85B828097B7FF1F938702
:10B0E000A7C18843828097B7FF1F938727C18843F2
:10B0F000828019E17D558280F5DE984265DFFDD9B9
:10B1000017B7FF1F1307C7E21847AA877155058BAA
:10B11000631D072403C507001547E37DA7FC03C78C
:10B1200037001305F0057D171377F70FE364E5FC8F
:10B1300003C35700E30003FC83C86700E38C08FAED
:10B1400003C77700494579171377F70FE364E5FAEA
:10B1500003C7A70011481305F7FF1375F50FE36B3D
:10B16000A8F803CE97000D481305FEFF1375F50FE1
:10B17000E362A8F803C8B7006309080065181378EC
:10B18000F80F1305600DE36705F703C5C70079489D
:10B1900079151375F50FE36FA8F403C8D7000D45B3
:10B1A0007D181378F80FE36705F503D80701930EB0
:10B1B00040175118420813580801E3ED0EF303C875
:10B1C000E7007D181378F80FE36605F303C827013D
:10B1D0007D181378F80FE36F05F103C88700C54E9B
:10B1E00075181378F80FE3E70EF103D86701856E41
:10B1F000938EBEE06D18420813580801E3EC0EEF81
:10B2000003D847016D18420813580801E3E40EEF14
:10B2100003D887017918420813580801E36C05ED3B
:10B2200003C8A7017D181378F80FE36505ED03C582
:10B23000B7011D487D151375F50FE36DA8EA03C529
:10B24000D701714879151375F50FE365A8EA03D5A1
:10B25000E7011308E00F7D1542054181E36CA8E882
:10B2600003C50702494879151375F50FE364A8E88B
:10B27000C85301C937C834005915130858BFE36BC8
:10B28000A8E603A8870237C53400130555BF59182F
:10B29000E36205E717B5FF1F2322C5A603C6050114
:10B2A00017B5FF1F232EF5A40545E375C5E403D8A4
:10B2B0002501D04933760603E31E06E203C61501D5
:10B2C000E30A06E217B6FF1F2328B6A283C52700AC
:10B2D00001466387A50003C61700F1453306B60291
:10B2E00083C707039305C00272971A071307C705A0
:10B2F00016031A9796084697B387B70241553E97AB
:10B300003297420741836362E8061773FFFFE70243
:10B3100003DD368597800000E780406C97000100D0
:10B32000E780C04B2A8497A00000E780205E2A9423
:10B3300097F00000E780002A2A9497900000E780A9
:10B3400040852A9497F0FFFFE780E06F2A949740AA
:10B350000000E78000972A9497700000E78040A0E3
:10B3600022951773FFFF6700C3D982801773FFFF11
:10B37000E702E3D64111A307A10097A00000E780F0
:10B3800040C99305F100170500001305E5B597F0D6
:10B39000FFFFE780802F014541011773FFFF670022
:10B3A00043D61773FFFFE70203D117B4FF1F13043F
:10B3B00024B80328840079599368180097B4FF1FB4
:10B3C00023AC14B71378180063100802BA84BE893E
:10B3D000368B328A2E89AA8A97F0FFFFE780E0A792
:10B3E0007D15269519E531594A851773FFFF6700CA
:10B3F00003D097F0FFFFE78040A67D152695A16753
:10B40000E353F5FE97B7FF1F938747E998433E8CB8
:10B41000814B01CB014597F00000E780C047933B8B
:10B4200015004A85DA865686D28597900000E78017
:10B4300060512A8911CD1C44F99B17B7FF1F232D9A
:10B44000F7AE83270C00CDD3E3800BFA829769BF58
:10B45000268597B7FF1F23AF07AC97F0FFFFE78064
:10B46000809C4146CE8517B5FF1F1305E5B5973083
:10B470000100E780605A97D00000E780E09C032538
:10B48000040B97D00000E780A0A0054597D00000EE
:10B49000E780A0A7054597000000E78060EDA9B709
:10B4A00097B7FF1F9387C7A89C47858BEDC7177376
:10B4B000FFFFE702C3C217B5FF1F130525AF97B7FC
:10B4C000FF1F23A707A697B7FF1F23A507A697B7B8
:10B4D000FF1F23A307A697200100E780C084975091
:10B4E0000000E78080F997100100E7804050971036
:10B4F0000100E780405697B7FF1F9387E7A19C4361
:10B5000091C7054597800000E780E02397B7FF1FAC
:10B510009387478A9C4399C741657D1597700000C2
:10B52000E780E0A597F00000E780804197D0000019
:10B53000E780209397B7FF1F938747B49C431397E7
:10B5400017016356070097F00000E780A0B097B797
:10B55000FF1F23AB07A697B7FF1F23A907A697B71F
:10B56000FF1F23A707A697B7FF1F23A507A69700CE
:10B570000000E780008C97000000E780A07597F03E
:10B58000FFFFE780401897F00000E780E0D91773CD
:10B59000FFFF670003B7828097B7FF1F9387479924
:10B5A0008843828097B7FF1F93878798C84382801C
:10B5B000B7E7B0009387075063E1A70297B7FF1F73
:10B5C00093870797D843FD576367E50097B7FF1F39
:10B5D00023A2A79681473E858280B957EDBF177396
:10B5E000FFFFE702C3AF97800000E7806075978098
:10B5F0000000E780C0771773FFFF670083B0177301
:10B60000FFFFE70223AC2A849304140201112E8564
:10B61000B289A685214636C63A8997300100E7806F
:10B62000403D0DE9B24638082686CE8513059404C0
:10B6300097500000E780604121462C084A859730EA
:10B640000100E780003B1335150005611773FFFF0C
:10B65000670083AA0145D5BF1773FFFFE70223A840
:10B660009305450617A5FF1F1305C569971001002F
:10B67000E78020691773FFFF6700A3A81773FFFF18
:10B68000E702E3A541112EC697F0FFFFE780C01740
:10B69000B24588C141011773FFFF670083A6177386
:10B6A000FFFFE70223A2AA842E8497800000E78090
:10B6B000006CAA898545228597000000E780E07D1F
:10B6C00083C7E4011389940899E313890403CE85A1
:10B6D000228597000000E780407C214693051902EF
:10B6E000228597000000E780607897B7FF1F938757
:10B6F00027848C43228597100000E780C082214672
:10B7000093858402228597000000E78020761773D6
:10B71000FFFF6700639E1773FFFFE702C39939714C
:10B7200097F00000E780E0B49305400661E9978058
:10B730000000E78000606302051497A7FF1F83C71E
:10B74000275E13B7170097A6FF1F238BE65C014403
:10B7500099CFC16417A9FF1F1309897D9309400E72
:10B76000FD1497000000E78020836342A40A97F04D
:10B77000FFFFE78060094169B7290900096AFD7A7E
:10B780002A8B81447D199389F97B130A0A71938A64
:10B790008AC797000000E780208063D7A4041304C1
:10B7A000400EB387840217A7FF1F1307677803248F
:10B7B000070B3E948357C4016382270B184033075D
:10B7C000EB4063EAE900834744008507B3874703FA
:10B7D000D6976365F70801468145094597F0FFFF55
:10B7E000E780C04AAA8B29E597400000E780808364
:10B7F00085476317F50689659385057117A5FF1FB2
:10B800001305455097100100E780A04F95A0B3079E
:10B8100034030327090BBA9703D7C70163089700BE
:10B8200003C75700A38207002382E700050415BF62
:10B830009305C500228597000000E78080E65E85BD
:10B840002286976501009385A5DB97F0FFFFE780CF
:10B85000404F5E8597100000E780608A850415BF21
:10B8600097A7FF1F9387C76C9C478D83858BC1F774
:10B8700021611773FFFF67008387014685450945EE
:10B8800002D002D202D402D697F0FFFFE780004038
:10B89000AA8479DD97F00000E780E09C1389C4005A
:10B8A0002A8481454A8597000000E780005F0C40AC
:10B8B00041464A8597000000E780405B83294400A9
:10B8C0006385090C4E8502D802DA02DC02DE97306D
:10B8D0000100E780E0382ACE141005462C0808182D
:10B8E0004ECC97500000E780E00A1375F50F51ED3C
:10B8F0008355840093E525004A8597000000E78082
:10B90000E05E11460C104A8597000000E780005663
:10B91000014697650100938525CF268597F0FFFFA7
:10B92000E7802042268597000000E780407D5C404C
:10B93000A1D3014685450D4597F0FFFFE78000350F
:10B94000AA841DD548401389C40097300100E780C0
:10B9500020312AC64A8597000000E780404C3246D5
:10B96000636FC5004C404A8597000000E780005097
:10B9700001468145268597F0FFFFE780803C2685BC
:10B9800097000000E780A077E5B583558400ADB748
:10B990001763FFFFE702A37497A7FF1F9387475919
:10B9A0009C471DC193E7870017A5FF1F1305853529
:10B9B00017A7FF1F2322F75897100100E780403296
:10B9C0001763FFFF6700E373DD9B17A7FF1F2325A6
:10B9D000F75697300000E780E0647DF117A5FF1F60
:10B9E0001305453297100100E780E033D1BF17639C
:10B9F000FFFFE702436C4169AA892E8AB28A368B1F
:10BA0000BA8B814417ACFF1F130C8C52930C400E61
:10BA10007D1997F0FFFFE780205863C4A40001441C
:10BA20003DA03384940383270C0B3E948357C401B9
:10BA3000638627055A87D6865286CE85130504036A
:10BA400097000000E780E0BB01C923800B0022853E
:10BA50001763FFFF6700A3698347F40185C35A8713
:10BA6000D6865286CE851305940897000000E7809D
:10BA700040B909C585472380FB00D1BF850451BF6C
:10BA8000835745006380071E1763FFFFE702836348
:10BA900001112A8497000000E780C04D09C985473D
:10BAA0006309F50605611763FFFF6700E36497E02C
:10BAB0000000E780007C7DF5835744004947ED9BFB
:10BAC000E392E7FEC145228597000000E7804033FE
:10BAD000AA84228597000000E780204F0357440086
:10BAE00002CE91472A89631AF70022859700000049
:10BAF000E780A0513C082ACC3ECE97E00000E780CA
:10BB000080765C55C5D374084A86A685054582971C
:10BB100051BF03574400D147E3F6E7F8032A040076
:10BB2000C169014997AAFF1F938A8A40130B400EEF
:10BB3000FD1997F0FFFFE7802046634FA90E22858D
:10BB4000032A040097000000E780C042A1452A892B
:10BB5000228597000000E780A02AAA84228597000A
:10BB60000000E780804A14402A86AA897808268542
:10BB7000CA8597000000E780C0E7AA8405D503C7FF
:10BB8000F40189476315F7008347C10181DF5546FA
:10BB9000D2851385640097300100E780E0E7014516
:10BBA00097800000E780C01901C583D7C401A5E7CD
:10BBB00097A7FF1F9387C7379C479355190085891F
:10BBC00013D73700058B01CF8983858B6399B70025
:10BBD00001452EC697000000E780C0DBB2454E85C8
:10BBE00097800000E780601F0346C1012A84937597
:10BBF0001900268597900000E780E03935C1268539
:10BC000097800000E780E018268511C001459780E5
:10BC10000000E780004C97300000E780A040854797
:10BC2000E312F5E883C754001307F00FE38CE7E64F
:10BC30008507A382F400BDB5B304690383A70A0B8B
:10BC4000BE9483D7C401638B37015546D2851385D3
:10BC5000640097300100E780C0D955DD0509D1BDEA
:10BC60005DD86DB782801763FFFFE702A345978019
:10BC70000000E780000C05C1C164014417A9FF1F43
:10BC80001309092B9309400EFD1497F0FFFFE7807D
:10BC9000A030634EA40017A5FF1F1305A50697103B
:10BCA0000100E780E0031763FFFF6700E34433050B
:10BCB00034038327090B3E958357C501638897009A
:10BCC0002312050097800000E780A00C050475BFD3
:10BCD00097A7FF1F9387C7259C478D83858B8DE38F
:10BCE0001763FFFFE702A33F17A5FF1F1305850199
:10BCF00097100100E78020031763FFFF6700634090
:10BD000082801763FFFFE702833D9705000093855C
:10BD1000C5A017A5FF1F1305E5FE97100100E780DA
:10BD200020EE1763FFFF6700C33D1763FFFFE702C5
:10BD3000033B8841B7E70400BC5B05054205418130
:10BD4000829709C585472300F50005051763FFFFA6
:10BD50006700233B83C7F5FF2E858507A38FF5FE7C
:10BD6000828083C7F5FFFD1793F7F70FA38FF5FECA
:10BD700099EF1763FFFFE7028336B7E70400BC576C
:10BD80001385F5FF82971763FFFF67008337828073
:10BD90001C41035745008D8FBA951CC12312B50075
:10BDA0003E85828093D78500A2051441DD8D83579F
:10BDB00045001387E6FF18C189072312F50013D643
:10BDC00085004111238FB6FEA38FC6FE41018280FC
:10BDD00018419307F7FF1CC18357450085072312BD
:10BDE000F500A30FB7FE8280835745008D8F231285
:10BDF000F5001C41BE950CC12E858280AA8703D711
:10BE0000470008410D8FAA952392E7008CC38280DA
:10BE1000184108453305A7408280835745000357E2
:10BE200065001D8F1C4108453385A7403305A74099
:10BE300082801763FFFFE702832A41112EC62A84FE
:10BE400097000000E780A0FDB2456373B50001A034
:10BE5000835744000840BE952312B4003E9541012B
:10BE60001763FFFF6700E3291763FFFFE70223273C
:10BE700041112E84B28532C697000000E780A0FBF6
:10BE80003246A28597300100E78000B9410117636F
:10BE9000FFFF670003271763FFFFE70243242E8499
:10BEA000854597000000E78000F9230085001763AF
:10BEB000FFFF670003251763FFFFE70243224111DD
:10BEC0002317B100894597000000E780C0F683473B
:10BED000E1002300F5008347F100A300F5004101D4
:10BEE0001763FFFF6700E3211763FFFFE702231FCC
:10BEF00093D78500A2054111DD8D2317B100894537
:10BF000097000000E78020F38347E1002300F5005D
:10BF10008347F100A300F50041011763FFFF6700AD
:10BF2000431E1763FFFFE702831B1397850193D717
:10BF30008501C166938606F0D98F13D78500758F6A
:10BF4000D98FA2053707FF00F98D4111DD8D2EC66F
:10BF5000914597000000E78000EE6C001146973095
:10BF60000100E78060AB41011763FFFF67006319C1
:10BF70001763FFFFE702A3161C41854503C40700B2
:10BF800097000000E78080E622851763FFFF6700C7
:10BF900043171763FFFFE70283141C4141118945D2
:10BFA00003C7070083C717002307E100A307F100B9
:10BFB00097000000E78080E30355E100410117632B
:10BFC000FFFF670003141763FFFFE70243111C41E3
:10BFD0004111894503C7070083C717002307E10004
:10BFE000A307F10097000000E78040E08357E100DD
:10BFF000410113D58700A2075D8D4205418117637A
:10C00000FFFF670003101763FFFFE702430D0C41BA
:10C0100041112A841146680097300100E780C09FD3
:10C020009145228597000000E78040DCB247C16659
:10C03000938606F01397870113D58701598D13D77F
:10C040008700758F598DA2073707FF00F98F5D8D27
:10C0500041011763FFFF6700C30A1C45BE950CC171
:10C060008280AE87944391E6584101EF0CC15CC1D8
:10C07000828003C7570013671700A382E700B687C3
:10C08000D5B70CC3EDB7AA87084119CD1841D443E1
:10C0900098C36313D500D8C32A8703465700937605
:10C0A000160081E6232007008280944381CA8C42D7
:10C0B00003A847008CC363930601CCC3799A14C3C9
:10C0C000A302C7003687D1BF1C45DC471D8DB7775B
:10C0D000DBB6938777DB09853305F502420541819D
:10C0E0008280F147B385F50248452E9582808347CB
:10C0F000450085072302F50082801763FFFFE702F2
:10C1000003FE2A8409E41763FFFF670083FF834768
:10C110004400F5DBFD1793F7F70F2302F400E5F772
:10C120001C4403D7270005072391E700DC4399C38C
:10C13000228582974C4889CD83475400898B99E7A3
:10C140001C4422859C479C439C478297232A0400D9
:10C150000040232004007DB71763FFFFE70223F8A8
:10C160008357250041112EC681EB014422854101F0
:10C170001763FFFF6700E3F8035705008147F146A7
:10C18000E305F7FEB385D702404585072E94834526
:10C19000440008C4F5F5B247AA8481E7232A0400C5
:10C1A00009A81C456C0022859C439C43829748C883
:10C1B0004DDD85472312F400B247232004002318E5
:10C1C00004002319F4005C485CC483D72400FD17E5
:10C1D0002391F40061BF1763FFFFE70243F097A7C5
:10C1E000FF1F938727B488432326050023240500D7
:10C1F000410597100100E78000B31763FFFF670058
:10C2000043F01763FFFFE70283ED17A4FF1F13043A
:10C2100064B11C40411199CF9C472300B5002AC648
:10C220005CC197000000E78040FB1C40DC4399C3E1
:10C230003245829741011763FFFF670083EC034794
:10C24000450029E3584DAA877D551DCF1763FFFF91
:10C25000E702E3E81CC3DC4797A6FF1F23A4E6AC74
:10C26000F156130507012390D70097050000938529
:10C27000050297100100E780A09801451763FFFFB2
:10C28000670023E87D55828082801763FFFFE70205
:10C2900003E501116146814528009760FFFFE780B3
:10C2A00000E797A7FF1F9387E7A79C432800930504
:10C2B000F00FDC473EC697000000E780C0F4056140
:10C2C0001763FFFF6700E3E397A7FF1F938787A527
:10C2D0009C43D847A1679387C702631EF70A397149
:10C2E00006DE22DC26DA80004AD84ED652D456D258
:10C2F0003285B28497000000E780C0C7AA892685EE
:10C3000097000000E78020C92318A4FC2685970029
:10C310000000E78040C82319A4FC26859700000090
:10C32000E78060C783D744000A8A231AA4FC858368
:10C3300093F7F70F230EF4FC8607BD0793F7073F2B
:10C340003301F1408A8A01498347C4FD6367F902DA
:10C35000CE85130584FC232C54FD97000000E78054
:10C3600080EA5281130104FCF2506254D2544259C3
:10C37000B259225A925A2161828026859700000084
:10C38000E78060C193171900D69705092390A7008D
:10C390001379F90F55BF828097A7FF1F938787985E
:10C3A0009C43D847A1679387A702631AF70A39719C
:10C3B00006DE22DC26DA80004AD84ED652D456D287
:10C3C0003285B28497000000E780C0BAAA8926852A
:10C3D00097000000E78020BCFD572318A4FC2685A9
:10C3E0002319F4FC97000000E780E0BA83D74400EB
:10C3F0000A8A231AA4FC858393F7F70F230EF4FC13
:10C400008607BD0793F7073F3301F1408A8A014948
:10C410008347C4FD6367F902CE85130584FC232C92
:10C4200054FD97000000E78000DE5281130104FCF8
:10C43000F2506254D2544259B259225A925A21614E
:10C440008280268597000000E780E0B493171900EA
:10C45000D69705092390A7001379F90F55BF82805D
:10C4600097A7FF1F9387078C9C43D847A16789072D
:10C470006310F70A397106DE22DC26DA80004AD81A
:10C480004ED652D456D23285328997000000E780CA
:10C4900060AEAA894A8597000000E780C0AF835745
:10C4A00049000A8A2318A4FC858393F7F70F230C0D
:10C4B000F4FC8607BD0793F7073F3301F1408A8AF2
:10C4C0008144834784FD63E7F402CE85130584FC31
:10C4D000232A54FD97000000E780E0D25281130127
:10C4E00004FCF2506254D2544259B259225A925A20
:10C4F000216182804A8597000000E780C0A9939758
:10C500001400D69785042390A70093F4F40F55BF29
:10C51000828097A7FF1F9387E7809C43D847A16736
:10C520009387E704631EF70A397106DE22DC26DAF8
:10C5300080004AD84ED652D456D23285B284970063
:10C540000000E78020A3AA89268597000000E780E5
:10C5500080A42318A4FC268597000000E780A0A3F0
:10C56000231AA4FC268597000000E780C0A283D789
:10C5700044000A8A2319A4FC858393F7F70F230E3E
:10C58000F4FC8607BD0793F7073F3301F1408A8A21
:10C5900001498347C4FD6367F902CE85130584FC16
:10C5A000232C54FD97000000E780E0C55281130161
:10C5B00004FCF2506254D2544259B259225A925A4F
:10C5C00021618280268597000000E780C09C931738
:10C5D0001900D69705092390A7001379F90F55BFC5
:10C5E00082809797FF1F9387E7739C43D847A16783
:10C5F0009387C704631AF70A397106DE22DC26DA4C
:10C6000080004AD84ED652D456D23285B284970092
:10C610000000E7802096AA89268597000000E78021
:10C620008097FD572318A4FC2685231AF4FC970055
:10C630000000E780409683D744000A8A2319A4FCAF
:10C64000858393F7F70F230EF4FC8607BD0793F756
:10C65000073F3301F1408A8A01498347C4FD63677C
:10C66000F902CE85130584FC232C54FD97000000AD
:10C67000E78060B95281130104FCF2506254D25435
:10C680004259B259225A925A2161828026859700D6
:10C690000000E780409093171900D6970509239072
:10C6A000A7001379F90F55BF82809797FF1F9387D3
:10C6B00067679C43D847A167DD076317F7041763D3
:10C6C000FFFFE702C3A17971328532849700000031
:10C6D000E780408A2AC6228597000000E780A08B69
:10C6E0002311A102228597000000E780A088B245AF
:10C6F0002300A102280897000000E780C0B0456130
:10C700001763FFFF6700E39F82809797FF1F938760
:10C7100067619C43D847A167938787046317F70431
:10C720001763FFFFE702A39B79713285328497007C
:10C730000000E78020842AC6228597000000E78059
:10C7400080852311A102228597000000E780808266
:10C75000B2452300A102280897000000E780A0AAA4
:10C7600045611763FFFF6700C39982809797FF1F9A
:10C770009387475B9C43D847A1679387A7046312BD
:10C78000F7021763FFFFE702839501112800814537
:10C7900097000000E78020A705611763FFFF67008F
:10C7A000439682809797FF1F9387C7579C43D8472C
:10C7B000A167938757026319F7021763FFFFE70228
:10C7C00003920111328597F0FFFFE780A07A2308DA
:10C7D000A1008145280097000000E780C0A2056104
:10C7E0001763FFFF6700E39182809797FF1F93878E
:10C7F00067539C43D847A1679387E702631BF704FD
:10C800001763FFFFE702A38D01113285328497F091
:10C81000FFFFE7804078AA84228597F0FFFFE7803A
:10C820008077854709E9228597F0FFFFE7808074CC
:10C830004205B337A00028008145231891003ECA65
:10C8400097000000E780209C05611763FFFF6700E9
:10C85000438B82809797FF1F9387C74C9C43D84791
:10C8600099476313F7081763FFFFE702438779715E
:10C870003285328497F0FFFFE780C06F2AC6228599
:10C8800097F0FFFFE78020712310A102228597F027
:10C89000FFFFE780206E2301A102228597F0FFFFB2
:10C8A000E780406DA301A102228597F0FFFFE7809A
:10C8B000606C2302A102228597F0FFFFE780806B66
:10C8C0002313A102228597F0FFFFE780A06AB245FB
:10C8D0002314A102280897000000E780C092456158
:10C8E0001763FFFF6700E38182809797FF1F93879D
:10C8F00067439C43D847A1679387C7036313F7082F
:10C900001753FFFFE702A37D79713285328497F0D8
:10C91000FFFFE78020662AC6228597F0FFFFE780A9
:10C9200080672310A102228597F0FFFFE780A066B1
:10C930002311A102228597F0FFFFE780A063230265
:10C94000A102228597F0FFFFE780C062A302A10247
:10C95000228597F0FFFFE780E0612303A102228593
:10C9600097F0FFFFE7800061B245A303A10228080A
:10C9700097000000E780208945611753FFFF67009B
:10C98000437882801753FFFFE702637501112A8401
:10C9900097F0FFFFE780005EAA84228597F0FFFFF3
:10C9A000E780605F228597F0FFFFE780C05E035756
:10C9B00044008D4763F7E700228597F0FFFFE7808B
:10C9C000805D228597F0FFFFE780E05C2800A68568
:10C9D00097000000E780208305611753FFFF670081
:10C9E00043729797FF1F9387E7339C43D847A1670C
:10C9F000FD07631FF7001753FFFFE702436E328501
:10CA000097000000E78040F81753FFFF6700636F4F
:10CA100082809797FF1F9387E7309C43D847A16791
:10CA2000E5076315F7081753FFFFE702436B7971BA
:10CA30003285328497F0FFFFE780C0532AC62285F3
:10CA400097F0FFFFE7802055228597F0FFFFE780F2
:10CA500080542310A102228597F0FFFFE780A053A6
:10CA6000520551812311A10222852302010297F070
:10CA7000FFFFE7802050A302A102228597F0FFFF6D
:10CA8000E780404F2303A102228597F0FFFFE78054
:10CA9000604EB245A303A102280897F0FFFFE7808C
:10CAA000807645611753FFFF6700A36582809797E3
:10CAB000FF1F938727279C43D847A1679387E703E6
:10CAC000631FF7001753FFFFE7026361328597008A
:10CAD0000000E78060EB1753FFFF670083628280EE
:10CAE0009797FF1F938707249C43D847A167938795
:10CAF0004704631EF7021753FFFFE702435E797195
:10CB00003285328497F0FFFFE780C0462AC622852F
:10CB100097F0FFFFE7802048B245280897F0FFFF15
:10CB2000E780606E45611753FFFF6700835D828079
:10CB30009797FF1F9387071F9C43D847A167938749
:10CB400087026310F7041753FFFFE7024359797117
:10CB50003285328497F0FFFFE780C0412AC62285E4
:10CB600097F0FFFFE7800041B2452300A1022808AB
:10CB700097F0FFFFE780206945611753FFFF6700CB
:10CB8000435882801753FFFFE7026355011197F066
:10CB9000FFFFE780203EAA85280097F0FFFFE7808F
:10CBA000806605611753FFFF6700A3559797FF1F26
:10CBB000938747179C43D847A167D107631FF700A6
:10CBC0001753FFFFE702A351328597000000E7806B
:10CBD000A0FB1753FFFF6700C35282809797FF1F88
:10CBE000938747149C43D847A167C507631FF70085
:10CBF0001753FFFFE702A34E328597000000E7803E
:10CC0000A0F81753FFFF6700C34F82809797FF1F5D
:10CC1000938747119C43D847A167B907631FF70063
:10CC20001753FFFFE702A34B328597000000E78010
:10CC3000A0F51753FFFF6700C34C82809797FF1F33
:10CC40009387470E9C43D847A167AD07631FF70042
:10CC50001753FFFFE702A348328597000000E780E3
:10CC6000A0F21753FFFF6700C34982809797FF1F09
:10CC70009387470B9C43D84789476318F70217539C
:10CC8000FFFFE702C3450111328532C897F0FFFF6D
:10CC9000E780402EAA85280097F0FFFFE780A05686
:10CCA00005611753FFFF6700C34582809797FF1FF9
:10CCB000938747079C43D847A1678D076311F70403
:10CCC0001753FFFFE702A34101113285328497F029
:10CCD000FFFFE780202A13066100AA844C0022850A
:10CCE00097300000E780C0232800A68597F0FFFF5B
:10CCF000E780605105611753FFFF67008340828022
:10CD00009797FF1F938747029C4381CFDC4391CBCA
:10CD10001753FFFFE702A33C82971753FFFF6700FB
:10CD2000433E82801753FFFFE702633B79713C0863
:10CD3000AE843ED2A165B7070A002A843ED44810CB
:10CD40003C08DD053ED636C432C63AC297D0FFFF56
:10CD5000E780402C12474810BA8597F0FFFFE78024
:10CD6000C01332464810B28597F0FFFFE780E01409
:10CD7000A2464810B68597F0FFFFE78000125010DA
:10CD800001478146A685228597D0FFFFE780E04DC9
:10CD900045611753FFFF6700C3361753FFFFE702D4
:10CDA000033401117C000329C501AE843ECAA1658C
:10CDB000B70707002A843ECC48087C00C5053ECE54
:10CDC00097D0FFFFE78000258345D900480897F0FA
:10CDD000FFFFE780800C500801478146A685228529
:10CDE00097D0FFFFE780604805611753FFFF67009A
:10CDF00043311753FFFFE702832E83C7950093F754
:10CE0000F707A384F50097000000E78040F9175367
:10CE1000FFFF6700032F1753FFFFE702432C7971D1
:10CE20003C08AE843ED2A165B70709002A843ED4EF
:10CE300048103C08938545043ED632C636C497D088
:10CE4000FFFFE780201DA2464810B68597F0FFFF40
:10CE5000E780A00432464810B28597F0FFFFE780D4
:10CE6000C005501001478146A685228597D0FFFF57
:10CE7000E780A03F45611753FFFF670083281753E2
:10CE8000FFFFE702C32583C7950041112A8493F76A
:10CE9000F707A384F50032852EC697F0FFFFE780E1
:10CEA000800F85672AC46370F50297700000E780E1
:10CEB00020E92246B24509ED1147814622859700B7
:10CEC0000000E78060E641011753FFFF670063231E
:10CED00001478346F501DDB71753FFFFE702831EC5
:10CEE00001113C003ECAB7070A003ECC3C003ECED2
:10CEF00083C79500AA89328593F7F707A384F500C5
:10CF00002E8497F0FFFFE78000098567637DF504B5
:10CF1000A165AA8493858504480897D0FFFFE78020
:10CF2000600F268597700000E78080E12A8929E15B
:10CF30009145480897F0FFFFE78020F6A68548084E
:10CF400097F0FFFFE78060F7CA85480897F0FFFF7A
:10CF5000E780A0F4014781465008A2854E8597D00E
:10CF6000FFFFE780803005611753FFFF6700C3189C
:10CF70008145480897F0FFFFE78020F20349090246
:10CF800075BF1753FFFFE702E31379711C103ECA08
:10CF9000B7070F003ECC404D1C10AA84AE8948084C
:10CFA000994532C636893ECE97D0FFFFE78080068E
:10CFB00032464808B28597F0FFFFE78000EE630C29
:10CFC0000902A545480897F0FFFFE780C0E625461F
:10CFD000CA8597200100E78020A4500801478146B8
:10CFE000CE85268597D0FFFFE7802028456117531F
:10CFF000FFFF670063108355C402480897F0FFFFE6
:10D00000E780A0EB0355E402814505C585478545CA
:10D010006301F502C167FD179305F00F630BF5007F
:10D020007D1597700000E780208E9305150093F51D
:10D03000F50F480897F0FFFFE78020E683450403DB
:10D04000480897F0FFFFE78040E583451403480850
:10D0500097F0FFFFE78060E483552403480897F0CA
:10D06000FFFFE78080E583554403480897F0FFFF02
:10D07000E780A0E49DB71753FFFFE702430683C78D
:10D0800095008146014693F7F707A384F5009700C2
:10D090000000E78040EF1753FFFF67008306175338
:10D0A000FFFFE702C30379713E841C103ECA2E893C
:10D0B000B7070F00A1653ECCFD051C10AA844808E7
:10D0C00042C03AC23ECE36C432C697D0FFFFE78098
:10D0D00060F432464808B28597F0FFFFE780E0DB56
:10D0E000A2464808B68597F0FFFFE78000DD1247AB
:10D0F0004808BA8597F0FFFFE78020DC0248630C00
:10D1000008029145480897F0FFFFE780C0D211461A
:10D11000A28597200100E7802090500801478146B2
:10D12000CA85268597D0FFFFE780201445611753F5
:10D13000FFFF670003FD8945480897F0FFFFE78080
:10D1400080CF834704002300F50083471400A30029
:10D15000F500E1B71753FFFFE702C3F683C7950059
:10D1600001112A8A93F7F707A384F5003285AE846C
:10D1700032C697F0FFFFE78000E232462A89328507
:10D1800097F0FFFFE78000DF85676373F902AA89E4
:10D190004A8597700000E780A0BA2A8419ED1147EC
:10D1A00081464A86A685528597000000E780C0B771
:10D1B00005611753FFFF670023F49387E9FF93F797
:10D1C000F70F0547E366F7FE8347F50195EB8947BF
:10D1D000E380F9FE8346F401528501474A86A6851D
:10D1E00097000000E78040B4A167D90748083ECC0B
:10D1F000230A010002CE97000000E780A0B04DBFD7
:10D20000639EE7008947639EF90093071020231F60
:10D21000F50097700000E780C0B76DBF0947E39B3A
:10D22000E7FA8D47E398F9FA228597700000E780C6
:10D2300080DF9797FF1F938727CE9C4399E79797A7
:10D24000FF1F938727B79C4399C703D50400978096
:10D250000000E780A0CE231F040022855DBF175386
:10D26000FFFFE702C3E701113C003ECAB7070B000E
:10D270003ECC3C003ECE83C795002A89328593F789
:10D28000F707A384F500AE8497F0FFFFE780A0D0F6
:10D2900093170501C187635AF006A1652A84938517
:10D2A000E502480897D0FFFFE780C0D6A28548086E
:10D2B00097F0FFFFE78060C09797FF1F938787AFC6
:10D2C0009C43A9EB01449375F40F480897F0FFFFC6
:10D2D000E780A0BC9355844093F5F50F480897F07C
:10D2E000FFFFE78080BB9355044193F5F50F480895
:10D2F00097F0FFFFE78060BA014781465008A68596
:10D300004A8597D0FFFFE78040F605611753FFFF7E
:10D31000670023DF416585460546A2857D15975048
:10D320000000E78060BD59DD510597000100E780EE
:10D33000808F130440063344850271B71753FFFFF3
:10D34000E702E3D90111B70706003EC683C795007F
:10D3500021642A8993F7F707A384F500AE84280097
:10D360009305A4040AC40AC897D0FFFFE78080CAC7
:10D37000300001478146A6854A8597D0FFFFE780A8
:10D38000C0EE97E0FFFFE780E01113049404480823
:10D3900022CC230A010002CE97000000E78080968D
:10D3A00005611753FFFF6700C3D51753FFFFE7025F
:10D3B00063D1C1642A8901449799FF1F938949B7B2
:10D3C000130A8002FD1497E0FFFFE780E0BD63478A
:10D3D000A40001451753FFFF670003D2B3074403BE
:10D3E00003A7C90ABA9703D707006306970083D734
:10D3F0002700638427010504F9B70545E1BF1753EA
:10D40000FFFFE70223CC2A8A2E8999C123A00500B9
:10D4100081498144979AFF1F938A4A91614B97E013
:10D42000FFFFE780A0BE63C7A4004E851753FFFF30
:10D43000670083CC3384640383A70A003E94835738
:10D44000040099E763040900232089008504C1BF13
:10D450004146D2851305440097100100E7806059CA
:10D4600075F5A289E5B71753FFFFE702A3C5397128
:10D470007C083ED4B7070A003ED67C083ED883C756
:10D4800095002A8A328593F7F707A384F5002E8941
:10D4900032C697F0FFFFE78000B085676373F50839
:10D4A0003246AA84328597F0FFFFE780A0AC85471B
:10D4B000AA8963E8A706A16593858504281097D0FB
:10D4C000FFFFE78020B5268597700000E780408742
:10D4D0002A8429ED9145281097F0FFFFE780E09B13
:10D4E000A685281097F0FFFFE780209DCE852810A5
:10D4F00097F0FFFFE780609A014781463010CA85A8
:10D50000528597D0FFFFE78040D6A16793877704C5
:10D5100048183EDC230A010202DE97F0FFFFE78095
:10D52000607E21611753FFFF670003BD814528100E
:10D5300097F0FFFFE7806096A685281097F0FFFF21
:10D54000E780A0979797FF1F938707D59C4381CBD0
:10D5500022856389090097D00000E7804024834535
:10D56000040271B797D00000E780C022CDBF1753E7
:10D57000FFFFE70223B583C795004111AA8993F7FE
:10D58000F707A384F5003285AE84328A97F0FFFF57
:10D59000E78060A08567637FF5022A8997600000B5
:10D5A000E780007A2A84914631C58347F501054713
:10D5B0006387E70291C70D476366F704AD461DA870
:10D5C0009305050303250A00414697100100E780F3
:10D5D00040420DE941011753FFFF6700E3B1930596
:10D5E000950803250A00414697100100E780604036
:10D5F000814669F54A86A6854E8597000000E7803A
:10D60000C081C9BF83250A001305940897700000E4
:10D61000E780A02919C1C146F1BF9797FF1F9387E3
:10D62000A78F9C4399E79787FF1F9387A7789C4311
:10D6300099C7228597800000E780208A69FD854789
:10D64000A30FF400228597B00000E7806084228554
:10D6500097600000E780E0734E8581464A86A68584
:10D6600097F0FFFFE780607BA1679387570448002E
:10D670003EC42302010002C697F0FFFFE7808068E6
:10D6800091BF1753FFFFE70203A383C79500411122
:10D69000AA8993F7F707A384F50032852E89B28A09
:10D6A00097F0FFFFE780208F85676374F50EAA84EB
:10D6B00097600000E780C0682A840DED416B014A45
:10D6C000979BFF1F938BCB86130C400E7D1B19A8D5
:10D6D00033048A0383A70B0B3E948357C4016383EF
:10D6E0006705050A97E0FFFFE780008BE342AAFE8B
:10D6F00095460DA08357C5016396970293050503D0
:10D7000003A50A00414697100100E780802E994644
:10D7100011E181462686CA854E8597F0FFFFE78096
:10D72000C06F85A883A50A00130504039770000045
:10D73000E780A017C14679FD2285231E940097A09B
:10D740000000E780E074228597600000E780606455
:10D750009797FF1F938747B49C43A9C323000402F4
:10D76000228597D00000E78040F04E8581462686CE
:10D77000CA8597F0FFFFE780406AA1679387070497
:10D7800048003EC42302010002C697F0FFFFE78075
:10D79000605741011753FFFF6700639589472300D6
:10D7A000F402E1B7397106DE22DC4AD8800052D497
:10D7B00056D25AD026DA4ED65ECE2E8A32892A8B9F
:10D7C00097D0FFFFE780407A0605710541998A8A64
:10D7D0003301A140232224FC231404FC97D0FFFF33
:10D7E000E780807883479A000605350593F7F707A9
:10D7F0002315A4FCA304FA004A85232624FC97E001
:10D80000FFFFE780407993170501C1876340F0026D
:10D810005681130104FCF2506254D2544259B25959
:10D82000225A925A025BF24B21618280AA844A8575
:10D8300097E0FFFFE7802076AA894A8597E0FFFFFF
:10D84000E7806075A1659385C5022A89130544FCAC
:10D8500097C0FFFFE780007C268597C0FFFFE78029
:10D860004070854511C94A86CE8597C0FFFFE78085
:10D87000C069AA8B21E98945130544FC97E0FFFFA5
:10D88000E780A061A685130544FC97E0FFFFE780D1
:10D89000C062CE85130544FC97E0FFFFE780E0619E
:10D8A000CA85130544FC97E0FFFFE780006101474C
:10D8B0008146130644FCD2855A8597D0FFFFE78046
:10D8C000C09AB9B78145130544FC97E0FFFFE78094
:10D8D000C05CA685130544FC97E0FFFFE780E05D90
:10D8E000CE85130544FC97E0FFFFE780005DCA8505
:10D8F000130544FC97E0FFFFE780205C814497D04C
:10D90000FFFFE7806066E3D4A4FA83A70B011397B7
:10D910001400BA9783D5070099C5130544FC97E016
:10D92000FFFFE78080598504D9BF797106D622D4DC
:10D930004AD000184ECE52CC56CA26D25AC8AE890A
:10D940003289AA8A97D0FFFFE78000620605690541
:10D9500041990A8A3301A140232A24FC231C04FC98
:10D9600097D0FFFFE780406083C7990006052D052B
:10D9700093F7F707231DA4FCA384F9004A85232EFF
:10D9800024FC97E0FFFFE780006193170501C18742
:10D99000634FF0005281130104FDB250225492549F
:10D9A0000259F249624AD24A424B45618280AA84B6
:10D9B0004A8597E0FFFFE780005EA1659385A50299
:10D9C0002A89130544FD97C0FFFFE780A0642685E0
:10D9D00097C0FFFFE780E058854509C9CA8597C011
:10D9E000FFFFE78080552A8B29E18945130544FD17
:10D9F00097E0FFFFE780604AA685130544FD97E0A6
:10DA0000FFFFE780804BCA85130544FD97E0FFFFC9
:10DA1000E780A04A01478146130644FDCE8556851E
:10DA200097D0FFFFE7806084B5B78145130544FDBB
:10DA300097E0FFFFE7806046A685130544FD97E069
:10DA4000FFFFE7808047CA85130544FD97E0FFFF8D
:10DA5000E780A046814497D0FFFFE780E050E3DBFA
:10DA6000A4FA83270B0113971400BA9783D50700F4
:10DA700099C5130544FD97E0FFFFE7800044850446
:10DA8000D9BF1743FFFFE702836583474500404D39
:10DA9000D5EFFD575DC48346940009476363D70AF9
:10DAA0000346B400854663EEC6088306E40063CAF5
:10DAB00006085C45F9562390D7009787FF1F83C758
:10DAC000272799E3A304E4009787FF1F9387872EF6
:10DAD0009C4381E78947A306F4009787FF1F93873C
:10DAE000A77B9C4381E789472306F4009705000044
:10DAF00093854506AA841305040197F00000E7808A
:10DB00002010FD57231AF40281471CDC0148978737
:10DB1000FF1F23AB87209787FF1F93872721232E83
:10DB2000040304C0804397D0FFFFE780204E614686
:10DB30003306C502814522859740FFFFE780205DBF
:10DB400081473E851743FFFF6700A35BFD57D5BFA5
:10DB50001743FFFFE702A3582A8403554502976045
:10DB60000000E780E01D19E5231E04001743FFFFB6
:10DB7000670023598357E401F5DB930504FF17453C
:10DB80000100130525E297E00000E780E014F9BFEB
:10DB90001743FFFFE702A3542E89A1654111938526
:10DBA000E5032A8436C432C6BE843AC297C0FFFF5A
:10DBB000E780404612472285BA8597E0FFFFE7805D
:10DBC000C02D32462285B28597E0FFFFE780E02E28
:10DBD000A2462285B68597E0FFFFE780002E63030B
:10DBE00009029145228597E0FFFFE780C024114696
:10DBF000A68597100100E78020E241011743FFFF4F
:10DC0000670023508945228597E0FFFFE780A02227
:10DC100083C704002300F50083C71400A300F500A8
:10DC2000E9BF1743FFFFE702834B83C79500444DCD
:10DC3000054793F7F707A384F5001C42411183C7FA
:10DC400007006367F7062E842A89B1C003C7D40092
:10DC5000630FF7021787FF1F1307C715184305C384
:10DC6000A386F40097A00000E780404A83C7D40051
:10DC700099E741657D1597400000E780403083D7E4
:10DC80002403918B89C797E00000E780C0134A8581
:10DC9000A28597F0FFFFE7808010A167C1074800C9
:10DCA0003EC42302010002C697F0FFFFE780800513
:10DCB00041011743FFFF6700C3441743FFFFE7021B
:10DCC000034203D745008D47AA8441112E8432892F
:10DCD0002E8563E3E70297E0FFFFE780C02BAA856C
:10DCE00023000900268597C0FFFFE780002541013A
:10DCF0001743FFFF6700E34097E0FFFFE780A0299D
:10DD00002AC6228597E0FFFFE780E028B2458547D5
:10DD10002A862300F900268597C0FFFFE780E01ED2
:10DD2000F9B7397106DE22DC26DA80004ED652D4ED
:10DD300056D24AD85AD05ECEAE89B284AA8A97D03B
:10DD4000FFFFE780602106051305250241990A8A35
:10DD50003301A140232224FC231404FC97D0FFFFAD
:10DD6000E780801F83C7990006054D0593F7F707E5
:10DD70002315A4FCA384F9002685232624FC97E020
:10DD8000FFFFE780402193170501C1876340F00240
:10DD90005281130104FCF2506254D2544259B259D8
:10DDA000225A925A025BF24B21618280AA8B03AB0A
:10DDB000040097C0FFFFE780C01A51E583D74400F5
:10DDC00001498544F11793B71700A301F4FC834779
:10DDD00034FCA165C9C79385E504130544FC97C0CD
:10DDE000FFFFE7802023A685130544FC97E0FFFF93
:10DDF000E780A00ADE85130544FC97E0FFFFE7807B
:10DE0000C00B834734FC114691E30946DA851305BC
:10DE100044FC97E0FFFFE78060058144630A090046
:10DE2000416B7D1B97D0FFFFE780001363CCA402FA
:10DE300001478146130644FCCE85568597C0FFFFF7
:10DE4000E780A042B1B7A685130634FC9700000016
:10DE5000E780E0E6933415002A8986048DBF938518
:10DE6000C504A5BF8327C90013971400BA9783D5AB
:10DE7000070063886501130544FC97E0FFFFE78016
:10DE8000C003850445B71743FFFFE702C32279713A
:10DE90001C103EC4B7070F003EC61C103EC883C707
:10DEA0009500AA8A328593F7F707A384F500AE8917
:10DEB000328497E0FFFFE780000E93170501C187CA
:10DEC000635AF0062A8A228597E0FFFFE780A00CBC
:10DED0002A895285032B040097C0FFFFE780600862
:10DEE00039ED8357440081440544F11793B7170077
:10DEF000A303F10083457100DA872287CA86528620
:10DF0000280097000000E780E0C801478146300004
:10DF1000CE85568597C0FFFFE7802035A1679387A0
:10DF2000D70348083ECC230A810026CE97F0FFFF96
:10DF3000E78040DD45611743FFFF6700431BA28573
:10DF40001306710097000000E78060D7AA84094497
:10DF500055D13544E30055FB4A8597F0FFFFE78034
:10DF600000450D4441D9014497D0FFFFE780C0FE32
:10DF7000634DA400C16B0144FD1B97D0FFFFE780F8
:10DF8000A0FD634EA4001544B5B7DC44131714007C
:10DF9000BA9783D70700638327030504F1B7D844F2
:10DFA00093171400BA9703D70700631B77012390D8
:10DFB0002701268597A00000E78080DB01441DBF74
:10DFC000050465BF1743FFFFE702C30F83C7950032
:10DFD00041112A8A93F7F707A384F50032852E8929
:10DFE000328497E0FFFFE78000FB93170501C187AC
:10DFF0006353F006AA89228597E0FFFFE780A0F926
:10E000002311A1004E85832A040097C0FFFFE780FB
:10E0100040F539E58357440085440144F11793B72F
:10E020001700A300F1000348110003572100D68711
:10E030005285CE862686CA8597F0FFFFE780600668
:10E04000A167F10748003EC42302910022C697F061
:10E05000FFFFE78020CB41011743FFFF6700C309A3
:10E06000A2851306110097000000E78040C52A84AE
:10E07000894455D98357210011678544BA97C2074F
:10E080001167C1831307F7EFE36FF7F89787FF1F57
:10E09000938787E89C4381CB8545130521009750E2
:10E0A0000000E7802075835521002285814497C0B8
:10E0B000FFFFE780A0E125D923100500228597A066
:10E0C0000000E78040CD85B71743FFFFE702A3FEBE
:10E0D00083C7950041112A8B93F7F707A384F500B6
:10E0E00032852E8A328497E0FFFFE780C0EA9317DB
:10E0F0000501C1876351F006AA8A228597E0FFFFD8
:10E10000E78060E92A895685832B040097C0FFFFCA
:10E11000E78020E531E58357440081440544F11749
:10E1200093B71700A301F10003483100DE875A8539
:10E130004A87D6862286D28597F0FFFFE78060F671
:10E14000A167ED0748003EC42302810026C697F070
:10E15000FFFFE78020BB41011743FFFF670023F962
:10E16000A2851306310097000000E78040B5AA841D
:10E1700009445DD99167CA97C2071167C183130724
:10E18000F7EF0544E362F7FACA8597C0FFFFE7801F
:10E19000E0D3014451F9814997D0FFFFE780C0DC0B
:10E1A00063DBA900984893971900BA9703D7070033
:10E1B00005EF2390270197D0FFFFE780E0DA1544B1
:10E1C000E384A9F6268597A00000E780C0BC978766
:10E1D000FF1F938767D49C430144B9D74A85975062
:10E1E0000000E780C05889B785097DB71743FFFF56
:10E1F000E70243ED79713E847C083EC82E8AB7075A
:10E200001400A1653ECAE5057C08AA89080836C441
:10E21000428932C6BA8AC6843ECC97C0FFFFE780E7
:10E2200060DFCA85080897E0FFFFE78000C7324635
:10E230000808B28597E0FFFFE78020C8A246630A7E
:10E2400009049D45080897E0FFFFE780C0BE1D4612
:10E2500081459740FFFFE78080EB63890A0891457D
:10E26000080897E0FFFFE78000BD1146A6859700EC
:10E270000100E780607A100801478146D2854E850B
:10E2800097C0FFFFE78060FE45611743FFFF67000F
:10E29000A3E6B685080897E0FFFFE78000C21C40B0
:10E2A0000808D8439355C701858912075183B205E1
:10E2B000D98D97E0FFFFE78040C01C40080883C568
:10E2C000870097E0FFFFE78040BD1C40080883C53A
:10E2D000A70097E0FFFFE78040BC1C40080883C50B
:10E2E000970097E0FFFFE78040BB85BF894508089E
:10E2F00097E0FFFFE78020B483C704002300F50008
:10E3000083C71400A300F500BDB71743FFFFE70262
:10E3100063DB83C795004111AA8993F7F707A384AC
:10E32000F5003285AE84328497E0FFFFE780A0C617
:10E3300093170501C187635DF0042A89032A04004D
:10E3400097C0FFFFE780E0C119E983574400054803
:10E35000F11793B71700A307F100814631A8130600
:10E36000F100A28597000000E78060951DC51C455F
:10E370009DC783D6470001480347F10093078500F6
:10E38000D2884A86A6854E8597000000E78040E641
:10E3900041011743FFFF670023D609487DBF1D4891
:10E3A0006DBF1743FFFFE702E3D165715C083EC410
:10E3B000B7077B013EC65C083EC883C795002A8A22
:10E3C000328593F7F707A384F500AE8997E0FFFF46
:10E3D000E78040BA8357E100E1C78945280097C02C
:10E3E000FFFFE78020C38145280097E0FFFFE7801B
:10E3F000C0AA97C0FFFFE78000C99787FF1F9387D8
:10E40000A7E99C431784FF1F03448492AA843334F2
:10E41000800099C3136424009787FF1F938787990F
:10E420009C4399C3136444009787FF1F9387C7AE2B
:10E430009C4399C31364840083D5040028000149D8
:10E4400097E0FFFFE78060A783D52400280097E0CE
:10E45000FFFFE78080A683D54400280097E0FFFFF8
:10E46000E780A0A597D0FFFFE78000AB93150501DB
:10E47000C181280097E0FFFFE78020A4A285280043
:10E4800097E0FFFFE78060A39C446360F9020147C7
:10E4900081463000CE85528597C0FFFFE780E0DCE3
:10E4A00059611743FFFF670023C5DC44131449007B
:10E4B00028003E9497E0FFFFE78060968347440082
:10E4C0000347540089070607BA978607E36AF5FCF5
:10E4D000835524002800814A97E0FFFFE780E09DF4
:10E4E00083454400280097E0FFFFE780009B8345B9
:10E4F0005400280097E0FFFFE780209A83474400FC
:10E5000063C9FA00814A8347540063C1FA020509CE
:10E51000A5BF1C4413975A002800BA9783D507005B
:10E52000850A97E0FFFFE7804099C9BF032BC4002D
:10E5300093975A0028003E9B83552B00850A97E04D
:10E54000FFFFE780809783550B00280097E0FFFFCF
:10E55000E780A0964DBF1743FFFFE70243B85C4931
:10E5600093E717005CC997A00000E78020B6174327
:10E57000FFFF670003B91743FFFFE70243B62E848E
:10E58000814597F0FFFFE780C0E705C58357050089
:10E59000FD172310F50009C4835725002310F4004C
:10E5A00097000000E78060FB01451743FFFF67000D
:10E5B00043B531457DD823100400C5BF1743FFFF85
:10E5C000E70243B083C7950041112A8A93F7F70702
:10E5D000A384F50032852E89328497E0FFFFE7801F
:10E5E000809B93170501C1876356F006AA89C14530
:10E5F000228597E0FFFFE780A0802A8B4E85832A43
:10E60000040097C0FFFFE780C09531E983574400BD
:10E61000231101000544F11793B71700A300F1007F
:10E6200081440348110003572100D6875285CE86C6
:10E630002286CA8597F0FFFFE780A0A6A16793878F
:10E64000170248003EC42302810026C697E0FFFF60
:10E65000E780406B41011743FFFF6700E3A9130602
:10E660001100A28597F0FFFFE7806065AA8409E5A5
:10E6700023110100094475B7930521005A859700BD
:10E680000000E78080EF835721002A84D9DB978739
:10E69000FF1F938767889C4381CB85451305210025
:10E6A00097500000E78000158355210026853144EE
:10E6B00097C0FFFFE78080812DD5231005002685B8
:10E6C00097900000E780206D0144A1BF1743FFFF32
:10E6D000E702E3A041112E896C00AA8402C697F0DC
:10E6E000FFFFE78000D20DC1035705000507231087
:10E6F000E50097000000E78040E681473E85410144
:10E700001743FFFF6700E39F3247954765DBCA85E4
:10E71000268597300000E780400DC147E34005FEA5
:10E720003244854741462310F40083570900A685EB
:10E73000130544002311F40097000100E780C02D69
:10E74000228545BF1743FFFFE702C39783C79500A4
:10E750004111AA8A93F7F707A384F5003285AE89A1
:10E76000328497E0FFFFE780008393170501C1879C
:10E770006356F0062A8AC145228597D0FFFFE780BD
:10E780002068AA845285032B040097B0FFFFE7801E
:10E79000407D31E983574400231101008544F1177E
:10E7A00093B71700A300F100014403481100035779
:10E7B0002100DA875685D2862686CE8597F0FFFF20
:10E7C000E780208EA1679387070248003EC423029A
:10E7D000910022C697E0FFFFE780C0524101174336
:10E7E000FFFF67006391A2851306110097F0FFFFFA
:10E7F000E780E04C2A8409E523110100894475B7BC
:10E8000026859305210097000000E78060ECAA842C
:10E8100049FD83552100228597B0FFFFE780006BFB
:10E8200049F5014997C0FFFFE7800074635DA900C7
:10E83000184893171900BA9703D707000DEF03572D
:10E8400021002390E70097C0FFFFE780E071630697
:10E8500025039777FF1F9387276C9C4399C7035520
:10E86000210097500000E78080F0228597900000FB
:10E87000E78060521DBF050975B795443DB705C1D6
:10E880009307F00F630FF500C547630CF50093077E
:10E89000F5FF05453315F5004205418182800145AC
:10E8A000828041657D158280B9E91743FFFFE70249
:10E8B000038303450603328497000000E78060FC71
:10E8C0009305803EB305B502C205C18181CD0357D2
:10E8D000E402854763F8E7001305040197E00000B0
:10E8E000E78020428357E40241677D176385E70094
:10E8F000FD172317F4021743FFFF67008380828010
:10E900001733FFFFE702237B004283C79500444D86
:10E910000349140093F7F707A384F5008347040025
:10E92000220911673369F900A167B347F900411162
:10E930002A8BAE8A63ECE70E834724001307C00ED0
:10E94000B91793F7F70F6373F71003473400C14704
:10E9500063EEE70E834744001307E00793C70708F9
:10E960006371F70C8349840083477400A209B3E9FB
:10E97000F900856763F7F90A034A64008347540086
:10E980004E85220A336AFA0097500000E780403B28
:10E9900061C123962403834B3400137AFA00239A2F
:10E9A0003403238874032399440393890401631C6B
:10E9B000090023A60402239804024E8597E0000074
:10E9C000E78060363DA0034924004A859700000097
:10E9D000E78020EB2397A402834744004E85A38859
:10E9E000F402E38D0BFCE30B09FC97E00000E780E9
:10E9F000202F97900000E780007381460146D6855E
:10EA00005A8597E0FFFFE7800058A1679387970337
:10EA10003EC423020100480002C697E0FFFFE780E2
:10EA2000602E41011733FFFF6700636C8544A286A7
:10EA30002686D6855A8597E0FFFFE780C054A167F8
:10EA4000938797033EC423029100F1B7BD44C5B735
:10EA50009144F1BF1733FFFFE702C36601111C08A1
:10EA6000404D3EC2B7070F003EC41C083EC62A896F
:10EA7000AE8997C0FFFFE78000D7585C1C5C6346F7
:10EA8000B70E6394E50063E2A70E3385A740B3B7E2
:10EA9000A700B305B7401306803E81469D8D9700C1
:10EAA0000100E78080B793140501C180A1659385BB
:10EAB000C503480097B0FFFFE780C0558145480077
:10EAC00097D0FFFFE780603D83550404480097D04E
:10EAD000FFFFE780803E83552404480097D0FFFF66
:10EAE000E780A03D814589CCC167FD179305F00FF4
:10EAF0006388F400268597500000E780E0E0AA854F
:10EB0000480097D0FFFFE780403903554404814512
:10EB100001CDC167FD179305F00F6307F50097500E
:10EB20000000E78060DEAA85480097D0FFFFE780FD
:10EB3000C03683456404480097D0FFFFE780E03586
:10EB400083457404480097D0FFFFE78000355000EC
:10EB500001478146CE854A8597B0FFFFE780E07088
:10EB600005611733FFFF67002359814481B71733CD
:10EB7000FFFFE702C35683C7950093F7F707A38407
:10EB8000F50097000000E78020ED1733FFFF6700D6
:10EB900043571733FFFFE702E35283C79500411144
:10EBA000404D93F7F707A384F5002A8A3285B28493
:10EBB000AE8997D0FFFFE780003E2A8B268597D04D
:10EBC000FFFFE780403D2A89268597D0FFFFE78039
:10EBD000603A93170B0163CA0702E177CA97C2072D
:10EBE000C183116763E3E70293070910C207C1837A
:10EBF0001307B00F637BF70093170901C187AA8A37
:10EC0000634AF000C54763FE570141011733FFFF18
:10EC10006700834E97B0FFFFE7802025E31725FFAD
:10EC2000D5B763080B0263060902814463890A02AF
:10EC3000B7077F0023106405231124057CC0568587
:10EC400097000000E780E0C39304803EB304950280
:10EC500039A0B7077F00232004047CC081440355FA
:10EC6000240497E00000E780A0A3A1C497C0FFFFA1
:10EC7000E78060B7269593D7F44133379500AE9778
:10EC8000BA9708DC5CDCCE85528597000000E780EF
:10EC9000A0DC99E023220404A1679387B70348000E
:10ECA0003EC42302010002C697E0FFFFE780800513
:10ECB000A9BF814701481CDC232E0403E9B71733A1
:10ECC000FFFFE702C34197C0FFFFE7802034E14721
:10ECD0003305F502914597500000E78000C5E557E0
:10ECE00011C59777FF1F23A3A70481473E851733DC
:10ECF000FFFF6700034185471777FF1F230AF702CD
:10ED000082801733FFFFE702833D9777FF1F9387CA
:10ED1000A70180433DC0835704046390A70683572F
:10ED20002404639CB7043689B28497C0FFFFE78050
:10ED300080AB5C5C63C3B7046395B7001C5C63EE97
:10ED4000A7028347640463F3F400A6872303F40453
:10ED50008347740463F39700A687A303F4048357DF
:10ED6000440441677D176385E70085072312F40497
:10ED70003C4481C7CA85268582971733FFFF670009
:10ED800043389777FF1F938727FA9C43014599C320
:10ED900003C5870082801733FFFFE7024334011168
:10EDA000B70707003EC683C79500584D0AC493F7BE
:10EDB000F7070AC8A384F5002A89AE8411CB1C4248
:10EDC00083C707002304F70097900000E780003412
:10EDD000216493055402280097B0FFFFE780802349
:10EDE00097000000E78020FAAA85280097D0FFFF4F
:10EDF000E780A00A300001478146A6854A8597B082
:10EE0000FFFFE780804613044402480822CC230A0F
:10EE1000010002CE97E0FFFFE780C0EE05611733E7
:10EE2000FFFF6700032E1733FFFFE702432B01119B
:10EE30007C003ECAB70707003ECC7C003ECE83C7AD
:10EE400095002E84AA8493F7F707A384F500A165A3
:10EE500093855502480897B0FFFFE780A01B9700F5
:10EE60000000E78040F2AA85480897D0FFFFE780BE
:10EE7000C002500801478146A285268597B0FFFF52
:10EE8000E780A03E05611733FFFF67008327977770
:10EE9000FF1F938767E99C43094599C303C5970002
:10EEA00082809777FF1F938727E89C43094599C382
:10EEB00003C5D70082809777FF1F9387E7E69C43BF
:10EEC000014599C303C5A70082801733FFFFE702FE
:10EED000631F0111B70708003EC683C79500404D68
:10EEE0000AC493F7F7070AC8A384F5002A89AE84F9
:10EEF00029C41442854703C7060063E0E70A834735
:10EF00009400094681496380C702B307F740A30410
:10EF1000E400B339F00083C716002305F40097908E
:10EF20000000E780A01E03572403058B19C76386E2
:10EF3000090097D00000E78000E92164930584026E
:10EF4000280097B0FFFFE780E00C97000000E78003
:10EF500040F4AA85280097D0FFFFE78000F49700CF
:10EF60000000E78080F5AA85280097D0FFFFE780A2
:10EF7000C0F2014781463000A6854A8597B0FFFF61
:10EF8000E780A02E13047402480822CC230A010053
:10EF900002CE97E0FFFFE780E0D605611733FFFF61
:10EFA000670083151733FFFFE702631301117C002D
:10EFB0003ECAB70708003ECC7C003ECE83C7950012
:10EFC0002E84AA8493F7F707A384F500A16593859F
:10EFD0008502480897B0FFFFE780C0039700000054
:10EFE000E78020EBAA85480897D0FFFFE780E0EA9A
:10EFF00097000000E78060ECAA85480897D0FFFFE3
:10F00000E780A0E9500801478146A285268597B090
:10F01000FFFFE780802505611733FFFF6700630E60
:10F020009777FF1F938747D09C43014599C303C53A
:10F03000B70082801733FFFFE702630A0111B707A9
:10F0400007003EC683C79500404D0AC493F7F707F3
:10F050000AC8A384F5002A89AE8405C81C42054766
:10F0600083C707006368F7060347B400630FF70020
:10F07000A305F40097900000E78040098347B4009F
:10F08000B9CF97D0FFFFE78040BE21649305B4005D
:10F09000280097B0FFFFE780E0F797000000E780C7
:10F0A00060F8AA85280097D0FFFFE78000DF0147BE
:10F0B00081463000A6854A8597B0FFFFE780E01AB9
:10F0C0002904480822CC230A010002CE97E0FFFF62
:10F0D000E78040C305611733FFFF6700830297D0C5
:10F0E000FFFFE78020BF55B71733FFFFE70223FF7D
:10F0F00001117C003ECAB70707003ECC7C003ECE23
:10F1000083C795002E84AA8493F7F707A384F5009C
:10F11000A165AD05480897B0FFFFE780A0EF970015
:10F120000000E78020F0AA85480897D0FFFFE7801D
:10F13000C0D6500801478146A285268597B0FFFFBB
:10F14000E780A01205611733FFFF670083FB977705
:10F15000FF1F938767BD9C43094599C303C5C7003B
:10F1600082801733FFFFE70283F701117C00AE8432
:10F170003ECAA165B70707002A843ECCD1057C00B2
:10F1800048083ECE97B0FFFFE780C0E89700000038
:10F19000E78020FCAA85480897D0FFFFE780E0CFF2
:10F1A000500801478146A685228597B0FFFFE7807A
:10F1B000C00B05611733FFFF6700A3F41733FFFF90
:10F1C000E702E3F183C7950093F7F707A384F500FF
:10F1D00097000000E78020F91733FFFF670063F214
:10F1E0001733FFFFE70203EE83C795000329C5012C
:10F1F000411193F7F707A384F5001C4283C9070068
:10F20000854763E637079777FF1F9387E7089C4397
:10F210002E84AA8485CF97000000E78080F3894779
:10F220006306F502630409028347C900638037035C
:10F230002306390197900000E78040ED83572903AA
:10F24000898B89C797D00000E780E0B72685A28523
:10F2500097000000E78020F1A167CD0748003EC479
:10F260002302010002C697E0FFFFE780A0A9410149
:10F270001733FFFF670043E89777FF1F9387C7AAFD
:10F280009C431D4599C303C5E70082801733FFFFE8
:10F29000E702E3E40111B70707003EC683C7950004
:10F2A000584D0AC493F7F7070AC8A384F5002A89C2
:10F2B000AE8415C71C4283C7070093968701E18679
:10F2C00063C4060685466381D7068346E7006388E4
:10F2D000F6002307F70097900000E78020E3216401
:10F2E0009305E400280097B0FFFFE780A0D29700C5
:10F2F0000000E780A0F8AA85280097D0FFFFE780EC
:10F30000C0B9014781463000A6854A8597B0FFFF06
:10F31000E780A0F53504480822CC230A010002CE7C
:10F3200097E0FFFFE780009E05611733FFFF67004E
:10F3300043DD1733FFFFE70283DA01117C003ECA89
:10F34000B70707003ECC7C003ECE83C795002E84D5
:10F35000AA8493F7F707A384F500A165B9054808C7
:10F3600097B0FFFFE78000CB97000000E78000F137
:10F37000AA85480897D0FFFFE78020B250080147D0
:10F380008146A285268597B0FFFFE78000EE0561E4
:10F390001733FFFF6700E3D61733FFFFE70283D27F
:10F3A000AA8401441779FF1F13094998E14997C0BE
:10F3B000FFFFE780A0C56344A400014519A83305F9
:10F3C0003403832709003E958357250063979700F0
:10F3D00011051733FFFF670023D20504C9BF032EB1
:10F3E0008500630A0E121773FF1F1303E3B2032392
:10F3F00003006315030029436390061203234E01A3
:10F40000631503001D43639907101733FFFFE702DD
:10F4100083CAC689428A3E89BA8AB684328BAE8B49
:10F420002A84B5E103554E0019E501431A851733C7
:10F43000FFFF6700C3CBA167A98F116763FBE700DC
:10F4400097000000E78080F5814597F0FFFFE78097
:10F45000C0120844B70700E05841F98F18455CC155
:10F46000B707001FF98F1CC55C4991C7610597E07C
:10F470000000E780408BE38A09FA2285979000001C
:10F48000E78060C65DB7328597C00000E7804043E3
:10F490000D4349DD1C44116703D54700A167A98FBF
:10F4A00063FBE70097000000E78040EF814597F09D
:10F4B000FFFFE780800C0323840093164B01D18269
:10F4C0008347B300035663008588FD8BA305F300D3
:10F4D000FD777D8E558EFD76FD16B204F18E832765
:10F4E0004301C58E231273012313D3002304530158
:10F4F00023052301A3044301BDDF228597B0FFFF4D
:10F50000E78080C9AA850844B5D1610597D000007D
:10F51000E780207F8DB71D431A8582801733FFFF58
:10F52000E70243BA0569AA84AE89328A0144FD5ACA
:10F530007D1997C0FFFFE78020A26347A400014523
:10F540001733FFFF670043BBD84493171400BA97E3
:10F5500003D70700631F37032390570163070A008F
:10F56000268597900000E780A0809C449DC383D7A8
:10F570006700B3F72701639E3701D28801488147AE
:10F580000147814601468145268597000000E780B6
:10F5900040E5050479BF1733FFFFE702A3B2797195
:10F5A0001C103EC4B7070F003EC61C103EC883C7E0
:10F5B0009500AA8A328593F7F707A384F5002E8970
:10F5C000328497D0FFFFE780009D93170501C18724
:10F5D000635AF006AA89228597D0FFFFE780A09B97
:10F5E0002A8A4E85032B040097B0FFFFE7806097BF
:10F5F00039ED8357440081440544F11793B7170050
:10F60000A303F10083457100DA872287D2864E86F4
:10F61000280097E0FFFFE780E05701478146300070
:10F62000CA85568597B0FFFFE78020C4A1679387FE
:10F63000F70348083ECC230A810026CE97D0FFFF6F
:10F64000E780406C45611733FFFF6700E3AAA2859E
:10F650001306710097E0FFFFE7806066AA84094403
:10F6600055D1528597E0FFFFE78060D40D4459D90A
:10F670000546D285268597000000E78060EA2A8447
:10F6800051B71733FFFFE70283A5835507000346F1
:10F69000270041112A842E8532C62EC497E0FFFF31
:10F6A000E780E0D001C93246A245228597000000DC
:10F6B000E78000E741011733FFFF670083A417339A
:10F6C000FFFFE702439F83C795004111AA8A93F782
:10F6D000F707A384F5003285AE89328497D0FFFF07
:10F6E000E780608B93170501C1876357F00AC14516
:10F6F0002A8A228597C0FFFFE78080702A8D2285A5
:10F7000097D0FFFFE78020892A89228597D0FFFFC5
:10F71000E7804086930705F893F7F70F1307E00794
:10F72000AA8B637BF706228597D0FFFFE780808452
:10F730002A8C228597D0FFFFE780C083AA8C528550
:10F74000032B040097B0FFFFE780A08139E98357BE
:10F750004400231101008144F11793B71700A3005F
:10F76000F10005440347110083562100938784006C
:10F770005685DA8822885286CE8597F0FFFFE7808B
:10F7800020A7A167E90748003EC42302810026C6DE
:10F7900097D0FFFFE780005741011733FFFF670055
:10F7A000039513061100A28597E0FFFFE780205123
:10F7B000AA8409E52311010009446DB793052100CE
:10F7C0006A8597F0FFFFE780A0F02A8441FD83550A
:10F7D00021009356C9001316490185486688E287BF
:10F7E0005E87858A5182268597000000E78060BF8A
:10F7F0002A848DBF1733FFFFE702E38B83C7950091
:10F8000041112A8B93F7F707A384F5003285AE895F
:10F81000328497C0FFFFE780007893170501C18706
:10F820006352F00A2A8A228597C0FFFFE780A076FC
:10F83000AA8A228597C0FFFFE780E0752A89228582
:10F8400097C0FFFFE7800073930705F893F7F70F62
:10F850001307E0072A8C6377F706228597C0FFFF1E
:10F86000E7804071AA8C228597C0FFFFE7808070F7
:10F870002A8D5285832B040097A0FFFFE780606EDE
:10F8800039E58357440085440144F11793B71700C5
:10F89000A301F10003473100930784005A85DE88F5
:10F8A0002688D6865286CE8597F0FFFFE780409463
:10F8B0008D4748003EC42302910022C697D0FFFF27
:10F8C000E780404441011733FFFF67004382A28570
:10F8D0001306310097E0FFFFE780603E2A848944E9
:10F8E00055D99356C9001316490185486A88E68799
:10F8F0006287858A5182D68597000000E78060AED6
:10F90000AA8449BF1723FFFFE702C37B2A898144EA
:10F910000144617A916A176BFF1F130BEB5F97B07D
:10F92000FFFFE780606463C7A40022851723FFFF01
:10F930006700837C8327090093991400CE9703D531
:10F94000070033074501420741836364570305C13C
:10F9500003270B0019C785453E8597400000E780C7
:10F9600060E9832709000504CE97239007008504EA
:10F970007DB797000000E78060A283270900050497
:10F98000CE972390070065D5814597F0FFFFE7806C
:10F99000C0BEF1BF1723FFFFE702C37283C7950004
:10F9A00041112A8A93F7F707A384F50032852E893F
:10F9B000328497C0FFFFE780005E93170501C1877F
:10F9C000635AF004AA89832A040097A0FFFFE78006
:10F9D000405931E58357440085440144F11793B7FA
:10F9E0001700A301F10003483100D6875285014773
:10F9F000CE862686CA8597D0FFFFE780806AA167FA
:10FA0000F50748003EC42302910022C697D0FFFFAD
:10FA1000E780402F41011723FFFF6700E36DA285B8
:10FA20001306310097E0FFFFE78060292A848944AC
:10FA30005DD99767FF1F9387274E9C4381CF044969
:10FA400097B0FFFFE7804052AA85268597400000C7
:10FA5000E78040DA1305040197000000E780C0EA60
:10FA6000228597800000E78000338144ADBF1723D3
:10FA7000FFFFE702436483C795004111AA8A93F709
:10FA8000F707A384F5003285AE8932842311010083
:10FA900097C0FFFFE780205093170501C18763548B
:10FAA000F0062A8AC145228597C0FFFFE7804035CE
:10FAB000AA8B5285032B040097A0FFFFE780604AC2
:10FAC00021E98357440085440144F11793B7170097
:10FAD000A300F1000348110003572100DA8756857F
:10FAE000D2862686CE8597D0FFFFE780805BA16710
:10FAF0009387270248003EC42302910022C697D074
:10FB0000FFFFE780202041011723FFFF6700235EEE
:10FB1000A2851306110097E0FFFFE780401A2A84B0
:10FB200089444DD99767FF1F9387073F98433E89C4
:10FB300001CF044997B0FFFFE7800043AA852685DF
:10FB400097400000E78000CB1305040197000000F8
:10FB5000E78080DB97B0FFFFE780004195443DD907
:10FB6000930521005E8597F0FFFFE78060B6AA84C9
:10FB700035F11C480357210022852390E700978028
:10FB80000000E780402183270900A9D70355210001
:10FB900097400000E780A0BD35BF1723FFFFE702B5
:10FBA000835183C795004111AA8A93F7F707A3846D
:10FBB000F5003285AE89328497C0FFFFE780A03D13
:10FBC00093170501C1876351F0062A8A228597C0E1
:10FBD000FFFFE780403C2A895285032B040097A051
:10FBE000FFFFE780003831E5835744008544014436
:10FBF000F11793B71700A301F10003483100DA872A
:10FC000056854A87D2862686CE8597D0FFFFE78025
:10FC10004049A167F90748003EC42302910022C66B
:10FC200097D0FFFFE780000E41011723FFFF670019
:10FC3000034CA2851306310097E0FFFFE780200800
:10FC40002A8489445DD99167CA97C2071167C18325
:10FC50001307F7EF8544E362F7FA9767FF1F93876F
:10FC6000A72B9843BE8B01CF044997B0FFFFE780D5
:10FC7000A02FAA85268597400000E780A0B713052E
:10FC8000040197000000E78020C897B0FFFFE780DD
:10FC9000A02D95443DD11C48228581442390270105
:10FCA00097800000E780200F83A70B00B9D74A8513
:10FCB00097400000E780A0AB89B71723FFFFE7025A
:10FCC00003422A844105B28497000000E780C0C344
:10FCD00011C5228597800000E780E00B8146014630
:10FCE000A685228597800000E780C04E1C4C89C7FE
:10FCF000DC4799C3228582971723FFFF6700634083
:10FD00009767FF1F938747029C43014599C313855B
:10FD1000070182809767FF1F9387070188438280CE
:10FD20001723FFFFE702A33B9317C600DD8DC20533
:10FD30004111C1812A8432C697C0FFFFE780E017D6
:10FD40003246228511829375F60F97C0FFFFE78038
:10FD5000C01441011723FFFF6700A33A1723FFFFD9
:10FD6000E702433679713C083ED2B7070C003ED417
:10FD70003C083ED683C79500AE842A8993F7F707DF
:10FD8000A384F500A16593853504481097A0FFFF73
:10FD9000E7804028C165FD150144176AFF1F130A5B
:10FDA0002A19930A400EAE892E8B2EC697B0FFFFFC
:10FDB000E780801E4205931704014181C183B2454B
:10FDC00063E9A702C167FD176387F500481097C074
:10FDD000FFFFE780800E501001478146A6854A85C7
:10FDE00097A0FFFFE780604845611723FFFF67008A
:10FDF000A3303307540383270A0BBA9703D6C701EE
:10FE0000630A3601638A3501481097000000E780D5
:10FE100060F1DA85050451BFB285EDBF1723FFFFFE
:10FE2000E702632979717C083EC8B70711003ECA12
:10FE30007C083ECC83C79500AA89328593F7F707E3
:10FE4000A384F5002E8997C0FFFFE780C014856763
:10FE50006378F504A165AA848905080897A0FFFFC7
:10FE6000E780401B268597400000E78060ED133453
:10FE700015000A04A285080897C0FFFFE780E0018B
:10FE8000A685080897C0FFFFE780200325CC01471F
:10FE900081461008CA854E8597A0FFFFE780E03CA9
:10FEA00045611723FFFF67008324B307540303272B
:10FEB000CA0ABA9703D70700631C970003D6270026
:10FEC00063806505080897000000E780A0E5DE85EF
:10FED00005042EC697B0FFFFE780000D420593177B
:10FEE00004014181C183B245E3E1A7FCC167FD176D
:10FEF000E38FF5F8080897C0FFFFE78000FC41BFDB
:10FF0000B285F9B7C165FD150144176AFF1F130AD1
:10FF10002A02930A80022E8BAE8B65BF1723FFFF48
:10FF2000E702E31B18418347170083460700A20737
:10FF3000D58FD207D1832390F5008347270003474D
:10FF400017008D45A207D98F91832310F60097C023
:10FF5000FFFFE780A0E91723FFFF6700831A17233D
:10FF6000FFFFE7022316C16401441769FF1F13094D
:10FF700029FC93098002FD1497B0FFFFE780C002BF
:10FF80006347A40001451723FFFF6700E31633050D
:10FF900034038327C90A3E9583570500E38597FEFE
:10FFA0000504D9BF1723FFFFE702C3112A8AAE89D0
:10FFB000B284B68A97400000E78080D819E591475F
:10FFC0003E851723FFFF670023132A894E8597C0BC
:10FFD0000000E780E08E2A84638E0A048D476DD18D
:10FFE00003570500C547E31D47FD0347F901854653
:10FFF000AD47E317D7FC8347450081CF4146A6852F
:020000040001F9
:100000005D0597F00000E780C09E814755D9AD4758
:1000100045BF130965012302E500CA8526859710AF
:100020000000E780606231C1A547E38B0AF8230234
:10003000040079B705C183570500E39247F94146AB
:10004000A685190597F00000E780A09A81472DD971
:100050009947BDB74E8597000000E78080F02A845D
:10006000954739DD130955004DBF4146A68523103C
:100070004401231134011305190097F00000E780B3
:10008000A099228597800000E780A0EA81470DBFF4
:100090001723FFFFE702A30479717C003ECCB7076A
:1000A0000A003ECE7C003ED083C79500B2842E84E9
:1000B00093F7F707A384F5001306A1002A892C0003
:1000C000268597000000E780A0E5A16528088D053A
:1000D00097A0FFFFE78000F490408355A1000355EF
:1000E0008100854697000000E78000ECAA84AA857D
:1000F000280897C0FFFFE78040DA0356A100835528
:100100008100280897000000E780C0C1300801473F
:100110008146A2854A8597A0FFFFE78000158547A5
:1001200048103ED42302910202D697D0FFFFE78009
:1001300060BD45611723FFFF6700A3FC1723FFFF86
:10014000E702E3F979717C003ECCB7070A003ECEA6
:100150007C003ED083C79500B2842E8493F7F707C6
:10016000A384F5001306A1002A892C002685970098
:100170000000E780E0DAA16528088D0597A0FFFF61
:10018000E78040E990408355A100035581008146F6
:1001900097000000E78040E1AA84AA85280897C05C
:1001A000FFFFE78080CF0356A10083558100280818
:1001B00097000000E78000B7300801478146A2851C
:1001C0004A8597A0FFFFE780400A4810230291026A
:1001D00002D402D697D0FFFFE780C0B24561172353
:1001E000FFFF670003F21723FFFFE70243EF9700CB
:1001F0000000E78060DB1723FFFF670083F097674D
:10020000FF1F9387A7B2884382801723FFFFE7026F
:1002100003ED835725004111AE842A842307B100E2
:1002200017F5FFFF130525466C002316F10097A074
:10023000FFFFE780804591C4228597800000E7801A
:10024000E0D6FD572310F400130620028145130564
:1002500054009720FFFFE78080EB41011723FFFF49
:10026000670023EA1723FFFFE702C3E579717C00EB
:100270003ECCB7070A003ECE7C003ED083C7950037
:10028000AA89AE8493F7F7073285A384F500130695
:10029000A1002C0097000000E78080C80355810072
:1002A000114497400000E780A0A915C50355A1009F
:1002B000014497B00000E780A06011CD035705000E
:1002C0008357810045446318F70085459700000077
:1002D000E780E0F30144216993053900280897A0DD
:1002E000FFFFE78020D3A285280897C0FFFFE780A3
:1002F000C0BA0356A100835581002808970000006A
:10030000E78040A2300801478146A6854E8597A028
:10031000FFFFE78080F548104AD42302810202D60D
:1003200097D0FFFFE780009E45611723FFFF67001E
:10033000A3DC1723FFFFE702E3D89767FF1F93872C
:10034000A79E2A8488432E8915C5035745038357E2
:10035000C4016311F7022326050223180502410593
:1003600097D00000E780209C63060900978000007A
:10037000E78060DB81449769FF1F938969BB130A9B
:10038000800297B0FFFFE78020C263C4A404976790
:10039000FF1F938727A29C4399C70355C401972049
:1003A0000000E780C0BD6307090022859780000038
:1003B000E780C0A01306400E814522859720FFFFED
:1003C000E780E0D4FD57231EF4001723FFFF6700EA
:1003D000A3D23385440383A7C90A3E95035705007A
:1003E0008357C4016317F700CA8597000000E780B0
:1003F00000E2850479B71723FFFFE702A3CC83C788
:1004000095004111AA8993F7F707A384F500328577
:10041000AE8497C0FFFFE78000B885676378F50476
:100420002A8997400000E780A091014401CD83D73D
:100430000400314463882701854597000000E78068
:1004400080EF01444E85A2864A86A68597D0FFFF9D
:10045000E780A09CA1679387170448003EC423024D
:10046000810002C697D0FFFFE780C08941011723B2
:10047000FFFF670063C81723FFFFE702A3C4976766
:10048000FF1F9387678A804329C4014597C00000F6
:10049000E780002181470148C1641CDC232E04034E
:1004A000232004041769FF1F130989A80144930935
:1004B000400EFD1497B0FFFFE78000AE634FA4002D
:1004C000814517F5FFFF1305857F97A0FFFFE780A4
:1004D000C01B1723FFFF670023C2330534038327A4
:1004E000090B3E958357C5016387970085459700A3
:1004F0000000E78040E4050475BF9357050113D75A
:100500008700A380F50093170501C183A183238091
:10051000E5002381F500A381A50082801723FFFF5A
:10052000E702E3BB2300050083C71500A300F50025
:1005300083C725002301F50083C73500A301F5001B
:1005400083C745002302F50083C75500A302F500C9
:1005500083C7650093059500A30305002303F500F9
:1005600023040500328597000000E78040F9172337
:10057000FFFF670003B91723FFFFE702A3B4411190
:10058000E9540DCD85CD93F9C5FF2E842A89AA841F
:10059000338AA900B7EA040063189A020D888544DB
:1005A00011CCB7E704009C5F82972AC622866C00B4
:1005B0003305390197E00000E780004626854101B8
:1005C0001723FFFF670043B383A78A039104829731
:1005D00093170501C183A183A38EF4FE93570501F0
:1005E000238FF4FEA183238EA4FEA38FF4FE6DB7A8
:1005F00063E6D5021723FFFFE70263AEB28741111E
:100600003686BE8536C697E00000E780E040B246F9
:10061000410136851723FFFF6700A3AE814636856B
:100620008280838705001387F5003D05FD8793F7DA
:100630007708834607007D158606B58FA300F50071
:100640006307B7007D17834717009D83DDB782805E
:100650001723FFFFE702A3A8B7E7040083A7070952
:1006600032872A863A858297133515001723FFFFB4
:10067000670023A915C181478DC11723FFFFE7023A
:1006800003A6414697E00000E780003985473E8594
:100690001723FFFF6700E3A681473E8582801DCDBB
:1006A0001723FFFFE702A3A3414681452A84972031
:1006B000FFFFE780C0A5414681451305040397204D
:1006C000FFFFE780C0A40147C1672322040438C8A4
:1006D0007CC805451723FFFF6700A3A20145828060
:1006E00081473DCDB5CD1723FFFFE702439FB2847D
:1006F0002E891306800581452A849720FFFFE78015
:1007000000A1CA8524C4268597000000E780C0F6B2
:100710004146814522859720FFFFE780409F304476
:10072000A285228597000000E780C0F293040401AF
:10073000A285268597000000E780E0EEA6851305D8
:10074000040297000000E78000EE22859700000079
:10075000E78020F585473E851723FFFF6700639AF2
:100760003E8582801723FFFFE702C3954111E954BC
:100770000DCD85CD93F9C5FF2E842A89AA84338AAD
:10078000A900B7EA0400639844030D88814411CCA2
:10079000B7E704009C5F82972AC622866C00330567
:1007A000390197E00000E7802027268541011723C3
:1007B000FFFF6700639483A78A03910482979317CE
:1007C0000501C183A183A38EF4FE93570501238FF6
:1007D000F4FEA183238EA4FEA38FF4FE6DB765CD36
:1007E0001723FFFFE702038EB28411E605451723A6
:1007F000FFFF670063902A842E890145EDD93C48AC
:100800007848B3E6E700E5D69386F7FFB3B7F6007E
:100810007D17032A4404BA9734C87CC863050A06C6
:10082000C14913050A03B38949412295637D360105
:10083000B2862E86A68597000000E780A0DB7C406C
:10084000BE9464C065B7CE862E86CE859700000024
:10085000E78040DAC114D2944E9923220404A2877F
:100860009306040103C7070003C607038507318FFA
:10087000A38FE7FEE398F6FE3044A2852285970019
:100880000000E78020DD2699C1493306994063ECDA
:100890009900A9DCA686A68513050403970000002D
:1008A000E78040D579BF8147B306F4003307F600EF
:1008B0000347070083C5060085072D8F2380E600C8
:1008C000E39437FF3044A285228597000000E7803B
:1008D00060D8C1145DBF014582800DC11713FFFFB1
:1008E000E702E37F1306800581459720FFFFE7803D
:1008F000008205451723FFFF6700A3800145828022
:10090000814749C5C1C51713FFFFE702437DFC417D
:1009100041462E84AA846399C70413860501A287E1
:100920008146C14503C7070003C507038507298F13
:100930003305D600034505008506298FA38FE7FE02
:10094000E392B6FE3044A285268597000000E7803A
:1009500060D0228597000000E78060F885473E85DB
:100960001713FFFF6700E379138507031D8E814589
:1009700022959710FFFFE78080797C40130700F8ED
:1009800013060402A2972388E70251BF3E858280A6
:100990001713FFFFE702A3746D712E84B284AA853A
:1009A00090102800368997000000E780A0D309ED59
:1009B000D55725A050400C40280097000000E78044
:1009C00040E27DD5FD142104F5F42C004A85970002
:1009D0000000E78020F3814761DD3E8551611713F8
:1009E000FFFF670003721713FFFFE702436F411118
:1009F0002EC432C62C00054697000000E78080F91F
:100A000041011713FFFF6700C36F1713FFFFE702D2
:100A1000036D01112A842EC602C802CA02CC02CE7E
:100A200097E00000E780C023B2462A86A285080826
:100A300097000000E78060FB1375F50F0561171341
:100A4000FFFF6700036C1713FFFFE702436979712B
:100A5000B2872A8421462308B10013051101BE85FF
:100A60003AC436C697E00000E78000FBB246930523
:100A70009101368597000000E78060A82285141058
:100A800035460C0897000000E78020F62A842247AC
:100A900001E921460C103A8597E00000E780C0F795
:100AA000228545611713FFFF6700A3651713FFFF3A
:100AB000E702E3627171AE84AA850A8532849700E9
:100AC0000000E78060BB11C90A86A68522859700D1
:100AD0000000E78020B8814711E1C5473E854D61A0
:100AE0001713FFFF6700E3611713FFFFE702235CA3
:100AF0001D712A8AB289BE843546854713051101C6
:100B00002E8CB68A3A8BC28C468D2308F10097E072
:100B10000000E78060F010100C085285231F0100D0
:100B200097000000E780C0F82A843DEDA1476313D9
:100B3000FD089307900591E0E5473546E2851305EA
:100B4000110113990A012308F1001359090197E0D3
:100B50000000E78060EC1357890093978A00D98FD3
:100B600090080C085285231FF10097000000E780D1
:100B700020F42A8415E9A1E49387FA00918313797C
:100B8000F9003EC6631309004149668B8144C14B9D
:100B9000854DB247639F970C6A868C0033855C0154
:100BA00097E00000E78040E7228525611713FFFFEB
:100BB0006700A35393079004C9F0A547BDBF8347BF
:100BC00001050947C14B2308F10083471105A58F93
:100BD000A308F10093872400814463E1FB040147EB
:100BE00014083386E6008C08B386E400BA95DA96DA
:100BF00083C6060083C505000507AD8E2300D60019
:100C0000E390E7FE4147639CE70490080C08528597
:100C100097000000E780C0E925D181A0B3069B00C2
:100C2000BA871008B305F60090083E9603C5060083
:100C30000346060085078506298E2380C500E392BA
:100C400077FF998F90080C085285BE94970000009A
:100C5000E78000E68947014749D12A84B1B7900867
:100C60003E96034606001408BE962380C6008507FC
:100C700059BFB24785046387971481471808B306A4
:100C8000F70098083E973386F900034707000346AC
:100C900006008507318F2380E600E39177FF9008F7
:100CA0000C08528597000000E78080E05DF535462E
:100CB000E285130511012308B10197E00000E780E8
:100CC000A0D5139704014183939784002183D98F82
:100CD00010180C085285231FF10097000000E780D0
:100CE00020DD25FD814710183387F9003E96034724
:100CF000070003460600B306FB008507318F2380FB
:100D0000E600E39277FF65A81808B306F700980895
:100D10003E973386F9000347070003460600850720
:100D2000318F2380E600E3E127FFCA87639E7709BE
:100D300090080C08528597000000E78060D711FDED
:100D400081479800B306F700900818103E973E962A
:100D500003470700034606008507318F2380E6001E
:100D6000E39177FF3546E285130511012308B101B0
:100D700097E00000E78040CA1397040141839397EE
:100D800084002183D98F10180C085285231FF1008D
:100D900097000000E780C0D1E31105EC81471018EF
:100DA0003387F9003E960347070003460600B30663
:100DB000FB008507318F2380E600E3E227FFC109AE
:100DC000410BC1BB814785B79408BE9683C6060018
:100DD00018083E972300D700850789BF6380063235
:100DE0001713FFFFE702A32C59712A84BE89B28B27
:100DF00085473546130511022E8B468C4289BA8AE7
:100E0000368A2300F10297E00000E780E0C0101866
:100E10000C1022852317010297000000E78040C9CB
:100E200063180512A147631FFC069307900563939F
:100E30000900E5473546DA851305110293140A01C6
:100E40002300F102C18097E00000E780E0BC931727
:100E50008A0013D78400D98F90080C10228523179D
:100E6000F10297000000E780A0C47DE163920904CD
:100E70009307FA00BD88918391E0C144C207C18302
:100E8000DE8C814A3EC6414DB24763E2FA0E62866D
:100E9000B3854B01881097E00000E78080B54DC90D
:100EA0003D557DA093079004E39609F8A54759B7EF
:100EB000834701050947C14C2300F102834711050F
:100EC000B3C7F900A300F10293872900814963E1C8
:100ED000FC04814618103306D7008C083387D900EC
:100EE000B69556970347070083C5050085062D8FE5
:100EF0002300E600E390D7FE41476390E7069008A1
:100F00000C10228597000000E78080BA35D189A0B7
:100F1000B3863A01BA871010B305F60090083E96E2
:100F200003C506000346060085078506298E238033
:100F3000C500E39297FF3387EC4090080C102285A0
:100F4000BA9997000000E780A0B68947014741D1D0
:100F500065611713FFFF6700431990083E9603462B
:100F600006001410BE962380C600850779B7B247E5
:100F7000850A93990A01939D8A0093D90901639187
:100F8000570F85473546DA85130511022300F10214
:100F900093D9890097E00000E78000A8B3ED3D01F8
:100FA00090000C1022852317B10397000000E78002
:100FB00020B059FD8147A68963EA970626860C086A
:100FC0004A8597E00000E78020A581471810B30606
:100FD000F700100898083E973E960347070003461F
:100FE00006008507318F2380E600E3E197FE639FCB
:100FF000A90590080C10228597000000E78040ABFF
:1010000021F981479810B306F700900818183E9709
:101010003E9603470700034606008507318F23806D
:10102000E600E391A7FF4109C10CB9BD1808900083
:10103000B306F7003E963387FC00034707000346DC
:1010400006008507318F2380E600B5B798084E97D4
:10105000034707001C10CE972380E700850941BF96
:1010600085473546DA85130511022300F10293D92D
:10107000890097E00000E780209AB3ED3D019000E1
:101080000C1022852317B10397000000E78040A2CF
:10109000E31005EC814718089000B306F7003E9670
:1010A0003387FC0003470700034606008507318F9E
:1010B0002380E600E391A7FF41460C084A8597E0AC
:1010C0000000E780609581471810B306F70010080C
:1010D00098083E973E96034707000346060085079B
:1010E000318F2380E600E391A7FF90080C10228542
:1010F00097000000E780C09B1DD599BD7D5582807B
:101100001713FFFFE702A3FD01112A842E85930523
:101110005100328902C002C202C402C693047400A4
:1011200097F0FFFFE780A03D1D46A68513059100BF
:1011300097E00000E780408E10088A854A85970076
:101140000000E780E09619ED93071400180883C6A5
:1011500007000346070085070507B18EA38FD7FE5A
:10116000E397F4FE05611713FFFF670083F9171378
:10117000FFFFE70223F52E848C414111AA89838762
:1011800015003289914463D30700A1449757FF1F8C
:10119000938787109C43A1C7C1CA8D472310F100D4
:1011A00083C725004A852301F10083C73500A301C9
:1011B000F10083C745002302F10083C75500A30255
:1011C000F10083C7650093059100A3030100230389
:1011D000F1002304010097F0FFFFE78040320C404C
:1011E0004A860A8597F0FFFFE780803303280400D2
:1011F00083564400A6881D0881470147E5164286AC
:101200008A854E8597000000E780408E2A8919E57F
:10121000A685228597B0FFFFE780E0C14A8541019E
:101220001713FFFF670043ED4A860A8597F0FFFF1B
:10123000E780002F6DB71713FFFFE702A3E82E84A6
:101240008C414111AA89838715003289914463D367
:101250000700A1449757FF1F938707049C43A1C72A
:10126000C1C68D472310F10083C725004A8523019D
:10127000F10083C73500A301F10083C745002302B5
:10128000F10083C75500A302F10083C765009305F1
:101290009100A30301002303F1002304010097F050
:1012A000FFFFE780C0250C404A860A8597F0FFFFC4
:1012B000E780002783564400032804008A85858E32
:1012C000C2061D08C1822312D400A68881470147A7
:1012D000E51642864E8597000000E78060B0410128
:1012E0001713FFFF670043E14A860A8597F0FFFF67
:1012F000E78000234DBF1713FFFFE70243DEB3353E
:10130000B000011185052A891315F6013365150111
:101310002308B1009305110136843AC632C03EC499
:1013200042C297F0FFFFE780801DA2471248425556
:1013300093D68700230BF100930591019357880002
:10134000A30AD100A30BF100230C010197F0FFFFCA
:10135000E780E01A3247024603280400B337E00072
:10136000835644009207914411C2A1444A85A6883D
:1013700042860C0897F0FFFFE78040772A8919E53D
:10138000A685228597B0FFFFE780E0AA4A85056120
:101390001713FFFF6700E3D61713FFFFE70283D29F
:1013A00001113EC68647B335B0008505AA891315DD
:1013B000F6015D8D2308B1009305110136843A8949
:1013C000B28442C446C297F0FFFFE7804013224830
:1013D0009248164593578800A30AF100930591019E
:1013E00093D78800230B0101A30BF100230C1101FB
:1013F00097F0FFFFE780A01032471040835644006B
:10140000B337E000920703280900914891C0A14832
:101410000C084E8597000000E780809CAA8401E9B3
:10142000835544004A8597B0FFFFE780C0A026851A
:1014300005611713FFFF670023CCAA959307F00FF0
:1014400017070100130787596317B50013C5F7FF86
:101450001375F50F828005058346F5FFB58FBA97A2
:1014600083C70700D5B70357450014419307F00F12
:1014700017060100130686563697420741831395D7
:1014800006014181631BE500AD8FB29703C50700DC
:10149000130515F3133515008280850603C5F6FF85
:1014A000A98FB29783C70700D9BF1713FFFFE702C1
:1014B00003C3B28736842E86BA86AA853E85BA844F
:1014C00097F0FFFFE7806052634F0500228597D0B9
:1014D0000000E780E0782A86A686A285268597F018
:1014E000FFFFE78080501713FFFF670083C11713CA
:1014F000FFFFE70223BD5D712A8BAE8A170501004D
:101500001305454B2C00B284368ABA893E8997F080
:10151000FFFFE780C04F2A845DE134104146DA8541
:10152000280097F0FFFFE780404C2A8449E985476F
:10153000A303F100A6C2930771002408BEC4A686C7
:1015400085470D462C18281002DC02DED6C0BEC628
:1015500097F0FFFFE78000442A8435E1834771025A
:10156000A6860D4693F7F7072300FA00C1473EDE33
:101570002C188947281026DCA303F10097F0FFFF01
:10158000E78040412A8405ED4146A6854E8597D0E7
:101590000000E78060488D47A6860D462C1828106D
:1015A000A303F10097F0FFFFE780C03E2A8401E922
:1015B0004146A6854A8597D00000E780E045228510
:1015C00061611713FFFF670023B31713FFFFE702E3
:1015D00003B197F700009387E7A0984383C74700BC
:1015E00079712A89AE84170501001305253D0C0881
:1015F0003AC42306F10097F0FFFFE78040412A84B8
:1016000005ED14104146CA85080897F0FFFFE780F2
:10161000C03D2A8415E1140815462C00081097F0E7
:10162000FFFFE780803C2A8401E921462C082685BB
:1016300097D00000E780403E228545611713FFFFE9
:10164000670023AC1713FFFFE70263A997F70000B9
:10165000938747999C477971AA842E8417050100C6
:10166000130545360C083EC697F0FFFFE780203A89
:101670000DE914104146A685080897F0FFFFE780A2
:10168000C03605E1140811466C00081097F0FFFF02
:10169000E780A03519E58347F10193F7F7032300AD
:1016A000F40045611713FFFF6700A3A51713FFFFA1
:1016B000E702E3A23688A14881470147E54697F053
:1016C000FFFFE780A0421713FFFF670083A31713F4
:1016D000FFFFE702C3A03688A14881470147E546DE
:1016E00097F0FFFFE780C06F1713FFFF670063A14C
:1016F0001713FFFFE702A39E01112A842E850C0811
:1017000032C697F0FFFFE780803009ED3247970639
:1017100001009386A6291008C14522859700000084
:10172000E780E0D805611713FFFF6700839D17135B
:10173000FFFFE702C39A4111C1472EC032C48A8518
:1017400009463EC23EC697F0FFFFE780A024410154
:101750001713FFFF6700E39A1713FFFFE7022398B1
:101760004111AE8613061009AA850A8502C002C27D
:1017700002C402C697F0FFFFE7802027410117133C
:10178000FFFF670003981713FFFFE70243953287B7
:1017900097060100938686232E8693050002970004
:1017A0000000E780C0D01713FFFF67008395171371
:1017B000FFFFE702C3927971C1472ACC2ED032D401
:1017C0002C080D4628003ECE3ED23ED602C402C6AC
:1017D00002C802CA97F0FFFFE780C01B45611713DC
:1017E000FFFF670003921713FFFFE702438F01110A
:1017F000AA842E84170501001305C51D8A8597F05C
:10180000FFFFE780C02015E514084146A6850A853C
:1018100097F0FFFFE780601D09ED8347E101034773
:10182000F101A207D98FCA07C9836177D98F231025
:10183000F40005611713FFFF6700A38C15CD171384
:10184000FFFFE702C3899747FF1F9387A752904383
:101850009745FF1F938545521745FF1F1305854D7B
:1018600097D00000E78000C51745FF1F1305854C82
:101870001713FFFF6700E3881745FF1F1305854B0C
:1018800082808DCD1713FFFFE70263859747FF1F07
:101890009387474E944301112E840A869745FF1F74
:1018A0009385854D97D00000E78040C60A85029455
:1018B000014505611713FFFF6700A3847D558280F2
:1018C0001713FFFFE702A38197D00000E78080D1C4
:1018D0009747FF1F23A0A74A17F5FFFF1305E5C988
:1018E00097B00000E780C0741713FFFF67006381A3
:1018F0001747FF1F1307474A9317150008433E95E4
:10190000FD572310F50082801703FFFFE702237DB8
:101910002A84084009E51703FFFF6700837E1C4106
:1019200058401CC06313E5005CC08347550023206A
:101930000500F99BA302F50097A0FFFFE780207C3C
:10194000C9BF1703FFFFE702E3779747FF1F93879E
:10195000A74698432A8411CB8347350093F70702A3
:1019600089C703550500894502971305440197B0BF
:101970000000E780403B835504000355E4009730A6
:101980000000E780A00C485819C597A0FFFFE7802A
:101990000077232A04021305840397000000E780E0
:1019A000E0F68144B1499790FFFFE780206A63CB5E
:1019B000A402834734002320040493F727FCA301E7
:1019C000F40000489790FFFFE78040691316150068
:1019D000814522859700FFFFE78060731703FFFFB3
:1019E00067008371B38734030329040385043E9998
:1019F0004A8597000000E78060F12304090065B77D
:101A00008347350093F7070299E3014582808357A6
:101A1000E500E39CB7FEC167FD176316F6000545B8
:101A20008280054599A81703FFFFE702436B9317D0
:101A30000601C187B2842A8401496359F0028357A1
:101A400005009DCB01456367F600034584003E9584
:101A50003325A6001375F50F0DA01C4813171900A8
:101A6000BA9783D70700E38E97FA05099790FFFF8F
:101A7000E780C05EE343A9FE01451703FFFF67004F
:101A800043681703FFFFE702E363AE89AA849790D8
:101A9000FFFFE78060522A8497D0FFFFE780A02EE7
:101AA000AA8601471306840197050000938585E403
:101AB0001745FF1F1305852E9790FFFFE780E0185D
:101AC0002A8925C98C441304C50022859E0593F5F7
:101AD000050897A0FFFFE780403CCC408387740057
:101AE000E18163DD070493E50508228597A0FFFFE8
:101AF000E780A03A0D4693854400228597A0FFFF1A
:101B0000E780C03683D50400228597A0FFFFE780D9
:101B1000E03D83D52400228597A0FFFFE780003DAC
:101B200003D6490083A50900228597A0FFFFE7801F
:101B3000E0334A851703FFFF6700035C93F5F50761
:101B40006DB71703FFFFE702835901112A8432851D
:101B500032C697A0FFFFE780E0279780FFFFE7806E
:101B6000C030835704001747FF1F1307673C3246F6
:101B7000231BF100930700F8A30DF1001C47184345
:101B8000231AA1008983858BB307F740B2854808E3
:101B90003ECE231C0100230D010097000000E780CA
:101BA00080EE05611703FFFF6700A3551703FFFFD2
:101BB000E7024351004101453DC49304C40026851A
:101BC0003289AE8997A0FFFFE780C02495452A8A15
:101BD0002685035B040197A0FFFFE780202126856F
:101BE00097A0FFFFE780603E8D45AA8A268597A0D3
:101BF000FFFFE780A01F268597A0FFFFE780E03C5E
:101C00005C48420A135A0A01D2975CC42318640143
:101C1000814763983A0146054D8133062541933744
:101C2000160013F5F70F1703FFFF6700E34C1703C8
:101C3000FFFFE702434889692A8BAE8B328AB68A56
:101C400081440144314CFD199790FFFFE78000402B
:101C500063CDA4009790FFFFE7804042018D33B52C
:101C6000AA001703FFFF6700834833898403832793
:101C70000B003E9963170A008347890085043E9450
:101C8000E1B703560A00DE854A8533F6C90097009E
:101C90000000E780E0F16DD10545E1B71703FFFFD4
:101CA000E702E34301112A847C000355E5003ECAA4
:101CB000B70707003ECC7C003ECE97200000E780AF
:101CC00020082A898545480897A0FFFFE78020392A
:101CD0009945480897A0FFFFE780E015AA844A8548
:101CE00097200000E780A0082380A4009747FF1FEB
:101CF000938707249C434166130606F09396870159
:101D000013D78701558F93D68700F18E558FA20781
:101D1000B706FF00F58FD98F11462C0013851400EC
:101D20003EC497D00000E78020CF5008A382040073
:101D30008945228597000000E780E0E019C9AA855F
:101D40001305840397A0FFFFE780E0313C4085073F
:101D50003CC005611703FFFF6700A33A1703FFFFAD
:101D6000E702E3379790FFFFE78040312A840504BC
:101D70009790FFFFE780802F3305A402F14791453C
:101D80003305F50297200000E78020BA11E565557C
:101D90001703FFFF6700E3369747FF1F23A6A7003F
:101DA0009790FFFFE780802D2A8405049790FFFF1E
:101DB000E780C02B3305A402894506059720000063
:101DC000E780A0B669D59747FF1F23A7A7FC979088
:101DD000FFFFE780A02A2A8405049790FFFFE78091
:101DE000E0283304A4029747FF1F239987FA9790AE
:101DF000FFFFE780A0282A849790FFFFE780002755
:101E0000930714003385A7029747FF1F2399A7F86C
:101E100097F700009387C77F1747FF1F2324F7F822
:101E20000145BDB71703FFFFE702C329AA842E8926
:101E300001449749FF1F9389A90F130A80069790C1
:101E4000FFFFE780A0226347A40001451703FFFFBF
:101E50006700832A3305440383A709024A86A685BF
:101E60003E9597000000E780E0B919E10504C1BF85
:101E70000545E9BF1703FFFFE702E323AA8A2E8B7C
:101E8000B28B368C3A8A814401448149974CFF1FBA
:101E9000938C0C0A130D80069790FFFFE780001DBE
:101EA00063C9A40011E085494E851703FFFF670051
:101EB00003243389A40383A70C025E86D6853E994A
:101EC0004A8597000000E780E0B31DC19790FFFFAF
:101ED000E780C01A0544636D4501D2866286DA85C3
:101EE0001305090397000000E780A0D411C18549BC
:101EF00085045DB71703FFFFE702C31CC1644111EE
:101F00002A8901449749FF1F93898902130A800691
:101F1000FD1436C632C42EC29790FFFFE78000152D
:101F200092452246B2466348A40001454101170389
:101F3000FFFF6700631C3305440383A709023E9536
:101F400009C683473500C18B9DC791C683473500BD
:101F500093F707028DC3630699008357E500639CDE
:101F600027010357050001CB63E7E50083478500A0
:101F7000BA97E3CDF5FA050469BF1703FFFFE7023F
:101F80006314C1642A8901449749FF1F938949FA60
:101F9000130A8006FD149790FFFFE780200D63462B
:101FA000A4001703FFFF670023153305440383A72D
:101FB00009023E958357E500638A97006304990000
:101FC0006396270197000000E780E0970504E1B7DA
:101FD0001703FFFFE702A30D89692A8AAE8A328BB5
:101FE000B68B8144174CFF1F130C8CF4930C8006A6
:101FF000314DFD199790FFFFE780400763C6A400AD
:102000001703FFFF6700630E3389940383270C02D5
:102010008355CA015A863E994A8597000000E78099
:10202000609E31C1814D15A03384AD038327090320
:1020300003D60B00D68533F6C9003E94228597005F
:102040000000E780E0B609E9850D9790FFFFE78083
:10205000E0FFE3CBADFC01A8228597000000E780FC
:10206000E08A23040400850471B71703FFFFE70229
:1020700083044169AA8A014A174BFF1F130B4BEBDC
:102080007D19C14B054C9790FFFFE78020FE63460A
:10209000AA001703FFFF6700830593098006B307B3
:1020A0003A0383290B02BE9983D7E900638E270187
:1020B00063842A01639A570103A4890301E84E85CA
:1020C00097000000E780C0BD050A75BF8357040173
:1020D000639977099304C400268597A0FFFFE780E2
:1020E00060D385452A8D2685835C040197A0FFFF78
:1020F000E780C0CF268597A0FFFFE780A0E76205B5
:102100006185635905048D45268597A0FFFFE7800B
:10211000E0CD8945268597A0FFFFE78020CD894542
:10212000268597A0FFFFE78060CC8545268597A090
:10213000FFFFE780E0CC83470500094793F7F707E7
:10214000639AE7009945268597A0FFFFE78040CB7B
:10215000A30285014848337D2D01231894016A9517
:1021600048C40040A1BF1703FFFFE70243F737E46D
:1021700004008327041D82979747FF1F83C747C822
:102180001715FF1F1305853AA300F5008327441C8C
:1021900082978327841C81461306F00F81450145F1
:1021A00082971703FFFF6700C3F51747FF1F130749
:1021B00027B518439745FF1F83C585C49747FF1F61
:1021C000938787C283468703034697036397D500A7
:1021D0009747FF1F2386C7C2828083C587010347B5
:1021E000A7036317B6009747FF1F238BE7C08280C2
:1021F00003C687016317C7009747FF1F2382D7C015
:10220000828083C68701130750026319D7009307A2
:1022100060021747FF1F2305F7BE828083C6870130
:10222000130660026315D60093077002DDB783C7FB
:10223000870155BF9747FF1F938707BBD44B0947BB
:10224000638DE6081703FFFFE70263E91749FF1FE5
:102250001309C9B63E8483470900918B9DCFB7E42B
:10226000040083A7041D829783A7441C1745FF1F02
:10227000130545B5829783A7841C81461746FF1F27
:10228000034646B681450145829721C5834709002B
:10229000ED9B1747FF1F2303F7B28347040093F713
:1022A000F70F85CB91471747FF1F2329F7B49700F6
:1022B0000000E78080EB97000000E78040EFB7E781
:1022C0000400BC4F414691451745FF1F034545B2E9
:1022D00082971703FFFF6700C3E282801703FFFFA7
:1022E000E702E3DF8D4741116306F504C547630844
:1022F000F50285476310F5029747FF1F2384A7B0B7
:10230000B7E70400BC4B930500101745FF1F0345BA
:1023100025AE829741011703FFFF670083DE8547E3
:102320001747FF1F2300F7AEB7E70400BC4B930528
:102330000020E1BF9747FF1F938707ABD44B11479E
:10234000638DE600B7E7040083A7071D8297B7E710
:102350000400BC4B930500044DBF05491747FF1F00
:10236000232E27A983C7070032C62E8493F7F70FC1
:10237000D5D3B7E4040083A7041D7D141374F40FB0
:102380008297E37689FCB245994703C61500E3F0CE
:10239000C7FCFC4409061745FF1F1305E5A68297F5
:1023A000BC48930500081745FF1F034565A48297A5
:1023B00079BF1703FFFFE70283D21747FF1F1307F9
:1023C000A7A24047184B1C409746FF1F23A4F6A224
:1023D0006316E4001747FF1F2320F7A2130584FEAE
:1023E0009790FFFFE78060A6035564FF9780FFFF8B
:1023F000E780E06E97A0FFFFE78060D01703FFFF44
:10240000670023D01703FFFFE70263CD9747FF1F45
:102410009387879DD84BDC4789C797000000E780EA
:1024200080F985471747FF1F232AF79C9747FF1F0F
:102430009387078D9C43930500021745FF1F0345B3
:10244000259B83C787031747FF1F230BF79AB7E71F
:102450000400BC4B82971703FFFF670083CA9747AE
:10246000FF1F23A5A79882801703FFFFE70283C5FC
:1024700037E404007C4CA1451745FF1F03454597F1
:1024800082977C48A1451745FF1F034565969744F1
:10249000FF1F938464958297DC4489EB97000000CA
:1024A000E78080D91703FFFF670003C503D567FFE7
:1024B0009780FFFFE780A062AA896DD1D848914735
:1024C0006310F7027C4C91451745FF1F0345459269
:1024D00082977C4891451745FF1F03456591829778
:1024E00003A9490103D409018947B7E90400174743
:1024F000FF1F2325F79083A7091D2104420482971B
:1025000083C784011715FF1F1305450261191717AB
:10251000FF1FA30DF70083A7491C418082979747AF
:10252000FF1F2381078E83A7C91C81460946937527
:10253000F40F4A85829711E99747FF1F83C7C79C0D
:1025400089C79700FF1FE780E06AB7E70400BC4F28
:102550002146A1451745FF1F03458589829799B7F5
:102560001703FFFFE702A3B793F7052001112E849D
:1025700081CF97000000E78020E913450420056122
:102580001703FFFF6700E3B793F70510A9CF974440
:10259000FF1F93846485DC4897000000E78020C11A
:1025A0001737FF1F1307C775184383C784010347F5
:1025B00087036318F700DC4489C797000000E780B1
:1025C00080DF85471747FF1F232AF782B7E70400FC
:1025D000BC4B930500021745FF1F03456581829799
:1025E0001345041069BF93F70508BDC79747FF1F40
:1025F00083C79781E91719469745FF1F9385E580A3
:102600001305D10093F4F70F1739FF1F0349C97F52
:1026100097C00000E780404093970401C1831737BB
:10262000FF1F1307E77E231DF100231CF1009737DE
:10263000FF1F9387677B3ACE3ACAD843230601002F
:1026400009CBDC439315890154080D46E1856800E8
:1026500082971345040825B793F72500A5C397373C
:10266000FF1F93876778D84B89476306F702973730
:10267000FF1F83C7A77413F7270011EF918B99CF22
:10268000B7E70400BC4F1306000A89451735FF1F42
:1026900003450576829713452400D5B59737FF1F6C
:1026A000938707669C4383C787031737FF1F230958
:1026B000F77497000000E78060DBF1BF93F7050235
:1026C00081CB97000000E78060DA1345040245BD26
:1026D00093F7850081CB97000000E780E0D2134597
:1026E000840071BD93F7150081CB97000000E7804F
:1026F000A0B41345140061B593F7450081CB970052
:102700000000E78060B31345440095BD93F70504CE
:1027100095C39737FF1F83C7276D91CB97000000A4
:10272000E780A0A491471737FF1F2329F76C1345B3
:102730000404B1B593F705010145E38207E4973737
:10274000FF1F9387676AD84B91476310F704973749
:10275000FF1F9387A7669C4313D727008583D98FD4
:10276000858B91E7B7E7040083A7071D8297B7E73A
:102770000400FC4F91451735FF1F0345656782979D
:1027800085471737FF1F232BF76613450401C5BB89
:102790009737FF1F238AA77682801703FFFFE70280
:1027A00003949737FF1F23A707649737FF1F23A5BD
:1027B000076485471734FF1F130484541737FF1F1E
:1027C000232EF7621C4083C787031737FF1F230997
:1027D000F7629790FFFFE780A08F29C59717FF1F2B
:1027E00023AAA7D41C40170500001305A5D783C74B
:1027F00087031737FF1F2305F7601717FF1FA3076E
:10280000F7D29737FF1FA381075EB7E7040083A7BE
:10281000070882979737FF1F238CA75C1703FFFFDA
:102820006700238EB7C7898E938767ED1717FF1F41
:102830002322F7D045BF1737FF1F0347E75A7955C3
:1028400055E79737FF1F9387275A03C717000507D8
:102850009736FF1FA38AE65803C717008D463377C4
:10286000D7029736FF1FA381E65883C61700173794
:10287000FF1F1307E748184393F6F60FA9EE8347A7
:1028800087031737FF1F230DF75685471737FF1F9D
:10289000230CF7549737FF1F938747529C430145FA
:1028A000998BA9E71703FFFFE702638337E404006E
:1028B0007C48C1451735FF1F0345855382973C4827
:1028C00085451735FF1F0345A5528297014517031C
:1028D000FFFF6700038383C7170085466395F600F3
:1028E0008347970379BF8347A70361BF82809737E8
:1028F000FF1F83C7674FA1CF17F3FEFFE702237EB9
:1029000037E404009737FF1F2380074E7C48854536
:102910001735FF1F0345C54D82977C4C91451735F0
:10292000FF1F0345E54C82977C4891451735FF1FF3
:102930000345054C82973C48C1451735FF1F0345A9
:10294000254B8297014517F3FEFF6700837B79557E
:10295000828017F3FEFFE70283782A84035565FF20
:102960009780FFFFE780A0179737FF1F9387C74720
:10297000D847BE841DEF9790FFFFE78080779C4883
:10298000232004009DEB9737FF1F23A78746973727
:10299000FF1F23A18746B7E70400BC4B89451735C5
:1029A000FF1F0345E5448297014517F3FEFF6700CB
:1029B0004375630A8700184375BF80C39737FF1FAD
:1029C00023AC8742C9BF7955CDB717F3FEFFE702A5
:1029D00003719737FF1F93876753884323260500AA
:1029E00023240500510597A00000E780C03317F3AA
:1029F000FEFF6700037117F3FEFFE702436E173413
:102A0000FF1F1304A4501C40411199CF9C4723027F
:102A1000B5002AC61CC197000000E78040FB1C409F
:102A20009C4B99C332458297410117F3FEFF670023
:102A3000436D17F3FEFFE702836A4111444D32856F
:102A400032842EC69790FFFFE780C0522AC42285A9
:102A50009790FFFFE780205403A84400630C080010
:102A6000B245835744001840224683D54500AA86C4
:102A700026850298410117F3FEFF6700836817F36C
:102A8000FEFFE702C365404D1DC808C09705000062
:102A9000938565031305440197A00000E780401665
:102AA0009737FF1F938787469C43014589E79737F0
:102AB000FF1F23AD874417F3FEFF670083647D5536
:102AC000DDBF17F3FEFFE702836101116800930584
:102AD000F00F02C602C802CA02CC02CE9700000064
:102AE000E780A0F1056117F3FEFF67008361973768
:102AF000FF1F9387A7419C43D847A1679D07631990
:102B0000F70217F3FEFFE702835D0111328597900C
:102B1000FFFFE7802046230AA10081456800970057
:102B20000000E78080ED056117F3FEFF6700635D3D
:102B300082809737FF1F9387673D9C43D847A167E3
:102B4000938777036319F70217F3FEFFE702235910
:102B5000011132859790FFFFE780C041230AA10051
:102B60008145680097000000E78020E9056117F3C0
:102B7000FEFF6700035982809737FF1F938707394D
:102B80009C43D84795476316F70417F3FEFFE70207
:102B900003550111328532849790FFFFE780803D15
:102BA000230AA10022859790FFFFE780C03E83574C
:102BB0004400231BA10081453ECC1C4068003ECE52
:102BC00097000000E78060E3056117F3FEFF6700F0
:102BD00043538280930785FF8DC38327C5FF91CF21
:102BE000DC4B81CF17F3FEFFE702634F032585FF20
:102BF000829717F3FEFF6700C350828017F3FEFF32
